:0200000480007A
:100000009705000093850502130540006B10B500AD
:10001000EF000001EF001034130500006B00050035
:10002000130540006B000500F32610029396A6010D
:10003000732600029315A6001316260037F1FF6FF2
:100040003301B1403301D1403301C100F326100226
:1000500063860600130500006B0005006780000042
:10006000130101FD2326810213040103232EA4FCA6
:10007000232CB4FC232AC4FC8327C4FD83A70700D8
:100080002326F4FE8327C4FE032744FD23A0E700B4
:100090008327C4FE938747002326F4FE232404FE0F
:1000A0006F004003832784FE032784FDB307F70016
:1000B00003C707008327C4FE2380E7008327C4FE0D
:1000C000938717002326F4FE832784FE9387170067
:1000D0002324F4FE032784FE832744FDE344F7FC36
:1000E0008327C4FD0327C4FE23A0E70013000000FC
:1000F0000324C1021301010367800000130101FD05
:100100002326810213040103232EA4FC232CB4FC18
:100110008327C4FD83A707002326F4FE8327C4FE9C
:1001200083A707002322F4FE8327C4FE938747009A
:100130002326F4FE232404FE6F004003832784FE5D
:10014000032784FDB307F7000327C4FE0347070016
:100150002380E7008327C4FE938717002326F4FE3D
:10016000832784FE938717002324F4FE032784FE4D
:10017000832744FEE344F7FC8327C4FD0327C4FE22
:1001800023A0E700130000000324C10213010103B0
:1001900067800000130101FF232611002324810042
:1001A00013040101B707008113850704EF00403AEB
:1001B000130000008320C10003248100130101010A
:1001C00067800000130101F723261108232481080A
:1001D00013040109232EA4F6232CB4F6B7070071EB
:1001E0002326F4FE930760002324F4FE130784FE05
:1001F0009307C4FE1306400093050700138507000C
:10020000EFF01FE61307C4F79307C4FE1306400080
:100210009305070013850700EFF09FE4B7270081DF
:1002200083A7C797E7800700B70700722322F4FE71
:10023000130784F7930744FE93050700138507000F
:10024000EFF0DFEB832784F783A747009385070050
:10025000B707008113854705EF00803F832784F7A8
:100260008397070093850700B7070081138507066A
:10027000EF00003E832784F783D72700938507008C
:10028000B70700811385C706EF00803C832784F7FA
:1002900083D7A70093850700B707008113858707D9
:1002A000EF00003B832784F783D7C70093850700BF
:1002B000B707008113854708EF008039832784F74B
:1002C0008397E70093850700B70700811385070927
:1002D000EF000038832784F783A707019385070081
:1002E000B70700811385C709EF008036832784F79D
:1002F00083A7470493850700B70700811385870A02
:10030000EF000035832784F783A7870493850700D0
:10031000B70700811385870BEF0080339307000038
:10032000138507008320C1080324810813010109F4
:1003300067800000130101FE232E1100232C810091
:10034000130401022326A4FEB70700811385470C7E
:10035000EF00002093071000138507008320C101E0
:10036000032481011301010267800000130101FFD2
:10037000232611002324810013040101B707008103
:100380001385870DEF00C01C130000008320C100FF
:10039000032481001301010167800000130101FFA4
:1003A000232611002324810013040101B7070081D3
:1003B0001385C70EEF00C019130000008320C10091
:1003C000032481001301010167800000130101FD76
:1003D000232611022324810213040103232EA4FCEB
:1003E000232CB4FC232AC4FCB70700712326F4FE97
:1003F000930750002324F4FE130784FE9307C4FEE2
:10040000130640009305070013850700EFF05FC552
:100410001307C4FD9307C4FE1306400093050700AD
:1004200013850700EFF0DFC39307C4FE032644FDE6
:10043000832584FD13850700EFF09FC2B727008155
:1004400083A7C797E7800700130000001385070004
:100450008320C1020324810213010103678000008D
:10046000130101FD2326810213040103232EA4FCA2
:100470008327C4FD63D807008327C4FDB307F0407A
:10048000232EF4FC0327C4FDB737000093870780B1
:1004900063D8E700B737000093870780232EF4FC6A
:1004A000B727008183A707982326F4FEB72700818A
:1004B00003A707988327C4FD3307F700B7270081F8
:1004C00023A0E7988327C4FE138507000324C102F5
:1004D00013010103678000006B10B5006780000006
:1004E0006B000500678000006B40B500678000006E
:1004F0006B200500678000006B3000006780000003
:1005000073251002678000007325000267800000D9
:10051000130540006B000500F32610029396F600C9
:10052000732600029315A6001316260037F1FF6FFD
:100530003301B1403301D1403301C100F326100231
:1005400063860600130500006B000500678000004D
:10055000130141FF232011002322B1008345050030
:1005600063880500EF00C001130515006FF01FFF41
:1005700083200100832541001301C1006780000032
:10058000B702010023A0B20067800000130101FD43
:10059000232611022324810213040103232EA4FC29
:1005A0000327C4FD9307F00063E4E702B717008157
:1005B0000327C4FD13172700938707F1B307F7003C
:1005C00083A7070013850700EFF09FF86F0040072F
:1005D000930700022326F4FEA30504FE8327C4FE2E
:1005E0009387C7FF0327C4FDB357F70093F7F700BE
:1005F0002322F4FE832744FE63860700930710003E
:10060000A305F4FE8347B4FE63820702B717008197
:10061000032744FE13172700938707F1B307F7005A
:1006200083A7070013850700EFF09FF28327C4FE1E
:100630009387C7FF2326F4FE8327C4FEE340F0FA26
:100640008320C1020324810213010103678000009B
:10065000130101FE232E1100232C8100130401023B
:100660002326A4FE2324B4FE0325C4FEEFF05FEE90
:10067000032584FEEFF09FF1B7070081138507146F
:10068000EFF01FED130000008320C101032481015E
:100690001301010267800000130101FE232E1100E7
:1006A000232C810013040102B727008183A7C79977
:1006B00013850700EFF0DFE2B727008103A78799D2
:1006C000B727008183A7479913850700E700070034
:1006D000EFF01FE32326A4FE8327C4FE63880700F0
:1006E00013050000EFF0DFDF6F00C00013051000FE
:1006F000EFF01FDF130000008320C10103248101FC
:100700001301010267800000130101FE232E110076
:10071000232C8100130401022326A4FE2324B4FE0B
:100720002322C4FE2320D4FEB7270081032744FEE2
:1007300023ACE798B7270081032704FE23AAE79894
:10074000B7270081032784FE23AEE798B707008010
:1007500093878769938507000325C4FEEFF0DFD7F1
:10076000EFF09FF3130000008320C10103248101F7
:100770001301010267800000130101FE232E110006
:10078000232C810013040102B70700811385471849
:10079000EFF01FDC13054000EFF09FD4EFF0DFD641
:1007A0002326A4FE0327C4FEB71700818326C4FEB8
:1007B00093962600938707F9B387F60023A0E700F6
:1007C00013051000EFF0DFD1B717008183A707F9F9
:1007D00013850700EFF09FDBB707008113854719EA
:1007E000EFF01FD7B7170081938707F983A747005A
:1007F00013850700EFF09FD9B707008113854719CC
:10080000EFF01FD5B7170081938707F983A78700FB
:1008100013850700EFF09FD7B707008113854719AD
:10082000EFF01FD3B7170081938707F983A7C7009D
:1008300013850700EFF09FD5B7070081138547198F
:10084000EFF01FD1130000008320C10103248101B8
:100850001301010267800000130101FE232E110025
:10086000232C810013040102EFF01FCA2326A4FEEB
:100870008327C4FE93B72700A305F4FE8347B4FE85
:1008800013850700EFF0DFC68347B4FE63840706D5
:100890008327C4FE93B717002305F4FE8347A4FE05
:1008A00013850700EFF0DFC48347A4FE63820702CD
:1008B000B72700810327C4FE131727009387079BE0
:1008C000B307F7001307A00023A0E7006F000002A2
:1008D000B72700810327C4FE131727009387079BC0
:1008E000B307F7001307B00023A0E700EFF0DFC065
:1008F0006F0040068327C4FE93B73700A304F4FEBD
:10090000834794FE13850700EFF09FBE834794FE54
:1009100063820702B72700810327C4FE131727004D
:100920009387079BB307F7001307C00023A0E700D6
:100930006F000002B72700810327C4FE13172700AA
:100940009387079BB307F7001307D00023A0E700A6
:10095000EFF09FBAEFF05FBAB727008183A7079B3C
:1009600013850700EFF09FC2B70700811385471971
:10097000EFF01FBEB72700819387079B83A747002F
:1009800013850700EFF09FC0B70700811385471953
:10099000EFF01FBCB72700819387079B83A78700D1
:1009A00013850700EFF09FBEB70700811385471935
:1009B000EFF01FBAB72700819387079B83A7C70073
:1009C00013850700EFF09FBCB70700811385471917
:1009D000EFF01FB8130000008320C1010324810140
:1009E0001301010267800000130101FE232E110094
:1009F000232C810013040102EFF09FB02326A4FEF4
:100A0000B72700810327C4FE131727009387079A8F
:100A1000B307F7000327C4FE23A0E7008327C4FE23
:100A20006386070013050000EFF09FAB1300000082
:100A30008320C101032481011301010267800000AA
:100A4000130101FE232E1100232C81001304010247
:100A5000B71700809387879E2326F4FE8325C4FE64
:100A600013054000EFF05FA7EFF01FF8B7270081F4
:100A700083A7079A13850700EFF05FB1B7070081DE
:100A800013854719EFF0DFACB72700819387079AEA
:100A900083A7470013850700EFF05FAFB70700811A
:100AA00013854719EFF0DFAAB72700819387079ACC
:100AB00083A7870013850700EFF05FADB7070081BC
:100AC00013854719EFF0DFA8B72700819387079AAE
:100AD00083A7C70013850700EFF05FABB70700815E
:100AE00013854719EFF0DFA6130000008320C10132
:100AF000032481011301010267800000130101FF3B
:100B0000232611002324810013040101EFF0DFC626
:100B1000B707008113858719EFF09FA313054000E5
:100B2000EFF01F9CEFF05FD313051000EFF05F9B19
:100B3000B70700811385C71AEFF09FA1EFF05FF0B0
:100B4000130000008320C100032481001301010170
:100B500067800000130101FF232611002324810078
:100B60001304010113051000EFF09F979305801CFB
:100B7000B70700811385871FEF00C00593070000AA
:100B8000138507008320C1000324810013010101A4
:100B900067800000130101FC2324C1022326D10237
:100BA0002328E102232AF102232C0103232E11031F
:100BB000138605008325850093068102232E1100EC
:100BC0002326D100EF0000068320C1011301010498
:100BD00067800000130101FC232AF102B72700817E
:100BE00083A787982324C1022326D1022322B1029E
:100BF0002328E102232C0103232E110383A5870060
:100C0000930641021306050013850700232E1100E9
:100C10002326D100EF0000018320C101130101044C
:100C200067800000130101E2232E111C232A911C6E
:100C30002328211D2326311D232C811B1389050008
:100C400093040600138C0600232C811C2324411DD1
:100C50002322511D2320611D232E711B232A911B4A
:100C60002328A11B2326B11B93090500EF40103B4D
:100C700083270500138507002328F102EF60C06475
:100C8000232EA1002320010E2322010E2324010E76
:100C90002326010E638A090083A789036396070050
:100CA00013850900EF2000588317C9001397270107
:100CB00063420702B726000003274906B3E7D700BF
:100CC0002316F900B7E7FFFF9387F7FFB377F70025
:100CD0002322F9068357C90093F78700638007042E
:100CE00083270901638C07028357C9001307A000FB
:100CF00093F7A7016390E7088317E90063CC070621
:100D000093060C001386040093050900138509005F
:100D1000EF10D0772320A1026F00C00193050900D6
:100D200013850900EF204002E30005FC9307F0FF64
:100D30002320F1028320C11D0324811D032501020C
:100D40008324411D0329011D8329C11C032A811C01
:100D5000832A411C032B011C832BC11B032C811BE9
:100D6000832C411B032D011B832DC11A1301011E6E
:100D700067800000B7070081938707212324F104CF
:100D8000B7070081930AC10F9387C738232A510DF3
:100D9000232E010C232C010C130A0000938B0A0054
:100DA000232E0102232C0102232401002326010209
:100DB000232A0102232001022328F10013840400C6
:100DC000130750028347040063840700639CE70A0B
:100DD000330B9440630A0B048327C10D23A09B00AF
:100DE00023A26B01B3876701232EF10C8327810DAA
:100DF00013077000938B8B0093871700232CF10C43
:100E0000635EF7001306410D930509001385090081
:100E1000EF804050631C0572938B0A008327010208
:100E2000B38767012320F10283470400639407001E
:100E30006F10106093071400A30B010A930DF0FFCD
:100E400023220102130400009306A005930CA000C6
:100E5000130D900003CB070013871700232CE1002C
:100E60001306A00293070BFE63F4F6006F108028B0
:100E70000327810493972700B387E70083A7070020
:100E800067800700130414006FF0DFF31385090077
:100E9000EF40D0188327450013850700232AF1026D
:100EA000EF6080422326A10213850900EF4010174E
:100EB000832785009306A0052324F1008327C10220
:100EC000638C0700832781006388070083C70700BE
:100ED0006384070013640440832781016FF09FF748
:100EE0008347710BE39A07FE93070002A30BF10AF5
:100EF0006FF09FFE136414006FF01FFE83270C0039
:100F0000130C4C002322F102E3D807FCB307F04096
:100F10002322F102136444006FF01FFC9307B00218
:100F20006FF0DFFC0327810183278101034B07005A
:100F3000938717006310CB04832D0C0013074C001C
:100F400063D40D00930DF0FF130C0700232CF10068
:100F50006FF09FF833839D039387170003CBF7FF50
:100F6000B30DE30013070BFDE376EDFE232CF10038
:100F70006FF05FEF930D00006FF0DFFE1364040865
:100F80006FF09FF58327810123220102032741028D
:100F9000130B0BFD93871700330797033307EB0001
:100FA00003CBF7FF2322E10213070BFDE370EDFEF5
:100FB0006FF0DFFB136484006FF01FF28327810161
:100FC00003C7070093078006631CF700832781018E
:100FD0001364042093871700232CF1006FF0DFEFD8
:100FE000136404046FF05FEF8327810103C70700D8
:100FF0009307C006631CF7008327810193871700BE
:10100000232CF100136404026FF01FED136404013C
:101010006FF09FEC93074C00232AF10083270C000C
:10102000A30B010A230EF112130C0000930D100004
:101030001307000023260100930C0000130D00008D
:101040009304C1132324E1026354B7012324B103A1
:101050008346710B638806008327810293871700FC
:101060002324F102937724002320F10463880700EE
:1010700083278102938727002324F1029377440872
:101080002322F1046390070883274102832681020B
:10109000B386D7406358D006B7070081130E00010E
:1010A0001388C737930E70000326810D23A00B0110
:1010B0008325C10D1306160013858B006354DE00D3
:1010C0006F10800423A2DB00B386B600232ED10C60
:1010D000232CC10C93067000930B050063D4C60249
:1010E0001306410D93050900138509002326E10429
:1010F000EF804022630405006F10902D0327C10488
:10110000938B0A008346710B638E06049306710B62
:1011100023A0DB009306100023A2DB008326C10D71
:1011200013067000938B8B0093861600232ED10C30
:101130008326810D93861600232CD10C6354D6028E
:101140001306410D93050900138509002326E104C8
:10115000EF80401C630405006F1090270327C10433
:10116000938B0A0083270104638E07049306810B87
:1011700023A0DB009306200023A2DB008326C10D01
:1011800013067000938B8B0093862600232ED10CC0
:101190008326810D93861600232CD10C6354D6022E
:1011A0001306410D93050900138509002320E1046E
:1011B000EF804016630405006F109021032701049F
:1011C000938B0A008327410493060008639CD7068B
:1011D0008327410283268102B386D7406354D00619
:1011E00013080001130E7000832701010326810DEF
:1011F0008325C10D23A0FB001306160013858B0069
:10120000E340D87623A2DB00B386B600232ED10CB0
:10121000232CC10C93067000930B050063D4C60207
:101220001306410D93050900138509002320E104ED
:10123000EF80400E630405006F109019032701042E
:10124000938B0A003307B7416350E006130800018F
:10125000130E7000832701018326810D0326C10D23
:1012600023A0FB009386160093858B00E342E8746D
:1012700023A2EB003307C700232EE10C232CD10C53
:1012800013077000938B05006350D7021306410DBE
:101290009305090013850900EF80C007630405006A
:1012A0006F101013938B0A00937604100327C10D5F
:1012B000E39406748327810D3383ED0023A09B0004
:1012C0009387170023A2BB01232E610C232CF10C62
:1012D00013077000938B8B006344F7006F10400678
:1012E0001306410D9305090013850900EF80800264
:1012F000630405006F10D00D938B0A006F1040043B
:10130000136404019377040263860706130C7C00C0
:10131000137C8CFF832C0C00032D4C0093078C0056
:10132000232AF10063440D006F109012330890419E
:1013300033370001B307A041338DE7401307D002D4
:10134000A30BE10A930C0800130710009306F0FFAB
:10135000E38ADD409306040033E6AC011374F4F72E
:10136000E3120640E38A0D5693061000E310D740BF
:101370006F10500F93074C00232AF100937704015C
:1013800063880700832C0C0013DDFC416FF09FF98C
:101390009377040403280C0063880700931C08015A
:1013A00093DC0C416FF05FFE93770420930C0800F0
:1013B000E38C07FC931C880193DC8C416FF0DFFC0D
:1013C000937784006388070A93074C00232AF1006F
:1013D00083270C0003A6070083A6470003A7870006
:1013E00083A7C7002320C10E2322D10E2324E10EA0
:1013F0001305010E2326F10EEF40803B232EA10A98
:1014000093072000631EF50A8327010E9305010947
:101410001305010A2320F10A8327410E232801081E
:10142000232A01082322F10A8327810E232C010895
:10143000232E01082324F10A8327C10E2326F10A53
:10144000EFB09041635605009307D002A30BF10A59
:101450009307700463D06707B70400819384043A4C
:101460001374F4F7130C0000930D30001307000001
:101470006F009035130C7C00137C8CFF83250C00CF
:1014800003264C0093078C001305010A232AF10060
:10149000EFE050588327010A2320F10E8327410AE9
:1014A0002322F10E8327810A2324F10E8327C10A08
:1014B0006FF01FF4B70400819384C4396FF05FFAB2
:1014C00093071000631AF5028327C10E63D6070045
:1014D0009307D002A30BF10A9307700463D8670146
:1014E000B70400819384843A6FF09FF7B7040081BA
:1014F0009384443A6FF0DFF6937CFBFD930710046E
:10150000639EFC0493070003230CF10A13071006E3
:10151000930780076304EB0093078005A30CF10A8F
:10152000930730061364240063D2B74D93851D00E2
:1015300013850900EF40404B93040500631E054AE4
:101540008357C90093E707042316F9008357C9009E
:1015500093F70704638007FE6FF04FFD9307F0FFDA
:101560006380FD4A93077004130C00006398FC002D
:1015700063960D00138C0D00930D1000032AC10E0D
:10158000936704102324F10223200104032F010E8A
:10159000832E410E032E810E635A0A00B707008086
:1015A00033CA47019307D0022320F10493071004A4
:1015B0006392FC4A1305010A2320E10B2322D10B7D
:1015C0002324C10B2326410BEFE050681306C10B07
:1015D000EF50901D13860500930505001305010AC1
:1015E000EFE050438327010A130601079305010822
:1015F0002320F1088327410A130501092328010646
:101600002322F1088327810A232A0106232C0106BD
:101610002324F1088327C10A2326F108B707FC3FDA
:10162000232EF106EFB010380328010903264109E3
:10163000832681090327C109930501091305010ABE
:101640002320010B232801052322C10A2326C104DC
:101650002324D10A2322D1042326E10A2326E100F0
:1016600023280108232A0108232C0108232E01081E
:10167000EFB000770327C100832641040326C1048D
:10168000032801056316050093071000232EF10AB5
:1016900093071006630CFB36370D008193070D3C52
:1016A0002326F100138EFDFF138D0400B7070340BE
:1016B00093050109232AC1081305010A130601082D
:1016C000232CC1052326F10823280109232CD10846
:1016D000232EE108232001082322010823240108E6
:1016E000EFB0502C0328010A0326410A8326810A01
:1016F0000327C10A1305010A232A01052328C1046F
:101700002326D1042322E104EFE0C07993050500EC
:10171000130A05001305010AEFE01017032741041F
:1017200003260105032841052326E1080327010AB2
:101730008326C1042322C1082328E1060327410A86
:101740009305010813060107232AE1060327810AEE
:101750001305010923200109232CE1060327C10AEF
:101760002324D108130D1D00232EE106EFC0904E57
:101770008327C100032E810583220109B385470118
:1017800083C50500832F4109032F8109832EC109D9
:101790002322C105A30FBDFE9307F0FF6300FE08DF
:1017A000130EFEFF930501091305010A2326D10735
:1017B0002324E1072322F10723205106232EC1050C
:1017C0002320510A232C51042322F10B232AF10553
:1017D0002324E10B2328E1052326D10B2326D10561
:1017E00023280108232A0108232C0108232E01089D
:1017F000EFB0005F0327C1048326010503264105DE
:1018000003288105032EC10583220106832F41068B
:10181000032F8106832EC106E31A05E83707FE3F32
:10182000930501091305010A2320510A232C5104B1
:101830002322F10B232AF1052324E10B2328E105C0
:101840002326D10B2326D10523280108232A0108AA
:10185000232C0108232EE108EFB0406B6348A0045D
:1018600083228105832F4105032F0105832EC104A7
:101870003707FE3F930501091305010A2320510A8A
:101880002322F10B2324E10B2326D10B232801086B
:10189000232A0108232C0108232EE108EFB040542D
:1018A0006310051A137A1A00630C0A188327C10003
:1018B0002326A10D9305000303C6F7008326C10C60
:1018C0001387F6FF2326E10C03C7F6FF6306C71450
:1018D000130690036316C7148327C10003C7A7002C
:1018E000A38FE6FE130A0D0013077004330A9A4013
:1018F000032DC10B6390EC2C1307D0FF6344ED0064
:1019000063DAAD33130BEBFF9306FDFF232ED10AF1
:101910001376FBFD130510041377FB0F93050000EE
:101920006318A6001307F7001377F70F930510004D
:101930002302E10C9307B00263D80600930610005F
:10194000B386A6419307D002A302F10C930790003F
:1019500063D8D72A1307310D130507009305A0009C
:1019600013083006B3E7B6021306F7FF93870703A1
:10197000A30FF7FEB3C7B6026344D82693870703C5
:10198000A30FF6FE1307E7FF1306610C6360A7269B
:101990009307410CB307F640232CF102B38D4701A6
:1019A0009307100063C6470193771400638607000E
:1019B0008327C101B38DFD001374F4BF9367041036
:1019C0002324F10223260100930C0000130D0000D4
:1019D00083270104638607001307D002A30BE10AE3
:1019E00003248102130700006FF0CFE5130C000001
:1019F0009304C1136FF09FB8130C05006FF01FB86C
:101A0000130C0000930D60006FF05FB7370D00817D
:101A10009307CD3A6FF0DFC8A38FB6FE6FF01FEAD1
:101A2000130717001377F70F6FF09FEB130A1A00D5
:101A3000A30FDAFE33874741E35A07FE6FF0DFEA70
:101A400083274104130A0D0093060003B307FD002A
:101A50006FF05FFE93076004638EFC0093075004F1
:101A6000138D1D006384FC00138D0D0013062000F0
:101A70006F00C000138D0D00130630009307010C9A
:101A80001308C10C1307C10B93060D009305010A3F
:101A9000138509002320E10B2326E1052322D10B26
:101AA0002322D1052324C10B2326C1012326410B68
:101AB000EF30C0109307700493040500032EC1009B
:101AC000832E4104032FC104639AFC009377140012
:101AD00063960700032AC10C6FF01FE1130760042F
:101AE000B387A401639AEC0683C6040013070003BE
:101AF0006390E606930501091305010A2328F10402
:101B00002320E10B2326E1052322D10B2322D1053B
:101B10002324C10B2326C1012326410B23280108BE
:101B2000232A0108232C0108232E0108EFB0402BA3
:101B3000032EC100832E4104032FC1048327010516
:101B40006308050013071000330DA741232EA10BD6
:101B50000327C10BB387E700930501091305010AA9
:101B60002326F1002320E10B2322D10B2324C10BD8
:101B70002326410B23280108232A0108232C0108CE
:101B8000232E0108EFB0C0258327C1006314050090
:101B90002326F10C930600036F00000113061700C3
:101BA0002326C10C2300D7000327C10CE368F7FEEE
:101BB0006FF05FF213076004E398ECD4137714001E
:101BC0003367B7016350A0076300070C8327C10187
:101BD0003307FD00B38DED00130B60066F000009A5
:101BE00013070600938607006FF0DFD7130717006F
:101BF0008347F7FF13061600A30FF6FE6FF01FD9F9
:101C00001307610C63980500930700032303F10C8D
:101C10001307710C93870603130617002300F700C0
:101C20006FF01FD7630607068327C10113871700CC
:101C30006FF05FFA63404D0313771400930D0D00AE
:101C4000630607008327C101B30DFD00130B700667
:101C50006F00C0018327C101130B7006B30DFA009A
:101C60006346A0013383AD41930D1300937C044080
:101C700023260100E38E0CD4930C0000E35AA0D578
:101C80009306F00F6F008003930D0D006FF0DFF4EB
:101C9000130B6006930D10006FF05FFD6356A703F2
:101CA00083278100330DED4003C71700630A070245
:101CB00093871700938C1C002324F1008327810055
:101CC00003C70700E31CD7FC8327C1003387FC0050
:101CD0008327C1023307F702B30DB7016FF05FCF5F
:101CE0008327C100938717002326F1006FF01FFDA3
:101CF00013074C00232AE1001377040283270C000A
:101D0000630007020327010223A0E7001357F741EE
:101D100023A2E700032C4101832481016FF00F8A85
:101D200013770401630807000327010223A0E700DB
:101D30006FF05FFE137704046308070003270102B6
:101D40002390E7006FF01FFD13740420E30E04FCE2
:101D5000032701022380E7006FF0DFFB1364040117
:101D60009377040263860702130C7C00137C8CFFBC
:101D7000832C0C00032D4C0093078C00232AF100C8
:101D80001374F4BF13070000A30B010A6FF00FDCFC
:101D900093074C00232AF100937704016386070020
:101DA000832C0C006F000001937704046388070004
:101DB000835C0C00130D00006FF09FFC93770420F0
:101DC000E38007FE834C0C006FF0DFFE3787FFFFD8
:101DD0001347078393074C00231CE10A3707008150
:101DE000232AF1009307C73A832C0C00130D00003F
:101DF00013642400232EF10213072000130B800725
:101E00006FF09FF893074C00232AF100A30B010AFF
:101E10009307F0FF83240C006384FD0213860D00FA
:101E20009305000013850400EF404023130C0500C8
:101E3000630E05E2B30D9540130C00006FF00FE345
:101E400013850400EF504048930D05006FF0DFFE4E
:101E5000136404019377040263820702130C7C006D
:101E6000137C8CFF832C0C00032D4C0093078C00FB
:101E7000232AF100130710006FF01FF193074C00A5
:101E8000232AF1009377040163860700832C0C005A
:101E90006F0000019377040463880700835C0C00E3
:101EA000130D00006FF01FFD93770420E38007FE01
:101EB000834C0C006FF0DFFEB70700819387073C6F
:101EC000232EF10293770402638A0704130C7C002B
:101ED000137C8CFF832C0C00032D4C0093078C008B
:101EE000232AF10013771400630E070033E7AC01D7
:101EF000630A070013070003230CE10AA30C610B1C
:101F0000136424001374F4BF130720006FF0DFE79D
:101F1000B70700819387C73A6FF09FFA93074C0089
:101F2000232AF1009377040163860700832C0C00B9
:101F30006F0000019377040463880700835C0C0042
:101F4000130D00006FF01FFA93770420E38007FE63
:101F5000834C0C006FF0DFFE9306040013071000A3
:101F60006FF08FBF93061000E308D74E9306200052
:101F70006308D7121307011A1316DD0193F67C00CC
:101F800013D83C0093860603B36C0601135D3D0035
:101F9000A30FD7FE33E6AC019304F7FF631E0602DE
:101FA00093771400638A0700930700036386F600A3
:101FB000A38FF4FE9304E7FF9307011A13870D0024
:101FC000130C0000B38D974023260100930C0000F2
:101FD000130D00006FF00F87138704006FF0DFF917
:101FE00093770440130A00001307011A2326F10017
:101FF000130C90001306A0009306000013850C003C
:1020000093050D009304F7FF2324E102EFA0501C79
:10201000032781028327C10013050503A30FA7FE31
:10202000130A1A00638807048327810003C7070087
:102030006312EA049307F00F630EFA0263140D00B3
:10204000637A9C038327C10283254103130A00009E
:10205000B384F4401386070013850400EF508028F2
:102060008327810003C717006306070093871700C3
:102070002324F1001306A0009306000013850C0032
:1020800093050D00EFA0805163140D00E3769CF3DF
:10209000930C0500138D0500138704006FF09FF566
:1020A0009304011A8327C10313F7FC009384F4FF00
:1020B0003387E7000347070013D84C002380E40070
:1020C0001317CD01B36C0701135D4D0033E7AC016D
:1020D000E31A07FC6FF05FEE9304011AE31E07ECAE
:1020E00093F61600E38A06EC93070003A30FF1189A
:1020F0006F00D037E30E0B32230E6113A30B010ADE
:10210000232A81016FE05FF29385050123A2CB01B1
:10211000232EB10C232CC10C63DECE021306410D1D
:1021200093050900138509002328E1042326D1041F
:10213000EF70401EE31E0528032701058326C10416
:10214000B707008113850A00930E70001388C73704
:10215000130E0001938606FF930B05006FE0DFF47A
:102160009385050123A20B01232EB10C232CC10C56
:10217000635ACE021306410D930509001385090029
:102180002322E1042320D104EF70C018E3120524B8
:10219000032741048326010413850A00130E7000EF
:1021A00013080001938606FF930B05006FF0CF83A1
:1021B0001306060123A20B01232EC10C232CD10CE4
:1021C0006356DE021306410D9305090013850900CD
:1021D0002320E104EF700014E31C051E0327010413
:1021E00093850A00130E700013080001130707FF00
:1021F000938B05006FF00F869306500663D86677C1
:102200008326010E930501091305010A2320D10A33
:102210008326410E2320E104232801082322D10A2A
:102220008326810E232A0108232C01082324D10AA6
:102230008326C10E232E01082326D10AEFA0503A8F
:102240000327010463120518B70700819387473DF0
:1022500023A0FB009307100023A2FB008327810D1E
:1022600013071700232EE10C93871700232CF10C82
:1022700013077000938B8B00635EF7001306410D0C
:102280009305090013850900EF70C008E3120514D7
:10229000938B0A008327C10B63C647019377140011
:1022A0006380070A832701030327C101938B8B00F7
:1022B00023ACFBFE8327C10123AEFBFE8327C10DA8
:1022C000B387E700232EF10C8327810D13077000DD
:1022D00093871700232CF10C635EF7001306410D62
:1022E0009305090013850900EF70C002E312050E83
:1022F000938B0A009304FAFF63549004130B0001BC
:10230000930C7000032601018327810D0327C10D63
:1023100023A0CB009387170093868B00634A9B060C
:1023200023A29B00B384E400232E910C232CF10CF8
:1023300013077000938B06006354F7006FE05FFA99
:1023400013744400E3160402032B41028327810225
:102350006354FB00138B070083270102B3876701D7
:102360002320F1028327C10D638C07001306410D62
:102370009305090013850900EF60D079E31A05047D
:10238000232C010CE31E0C08938B0A006FF09F981E
:102390001307070123A26B01232EE10C232CF10C60
:1023A00063DEFC001306410D930509001385090047
:1023B000EF605076E31E050093860A00938404FFC5
:1023C000938B06006FF01FF48326C10B634ED0166B
:1023D000B70700819387473D23A0FB0093071000B8
:1023E00023A2FB008327810D13071700232EE10C86
:1023F00093871700232CF10C13077000938B8B002D
:10240000635EF7001306410D93050900138509006B
:10241000EF605070631E057A938B0A008327C10B0F
:10242000937614000327C10DB367FA00B3E7D70012
:10243000E38807F08327010393888B0023A0FB0028
:102440008327C10123A2FB00B387E700232EF10CF1
:102450008327810D1307700093871700232CF10C3D
:10246000635EF7001306410D93050900138509000B
:10247000EF60506A631E057493880A00032BC10B3A
:1024800063500B06330B604113870800930C000167
:10249000130D7000032601018327810D8326C10DD2
:1024A0002320C700938717009388880063C26C07B6
:1024B00023226701330BDB00232E610D232CF10C4B
:1024C00013077000635EF7001306410D93050900C2
:1024D00013850900EF601064631C056E93880A0081
:1024E0008327C10D23A0980023A24801B387470189
:1024F000232EF10C8327810D13077000938B880026
:1025000093871700232CF10CE35CF7E26FE05FDDAB
:102510009386060123229701232ED10C232CF10C44
:10252000635EFD001306410D930509001385090044
:10253000EF60505E631E056893880A00130B0BFF63
:10254000138708006FF01FF5130B0D006354AA01E9
:10255000130B0A00635260053307EB00232EE10CD6
:102560000327810D23A09B0023A26B0113071700F3
:10257000232CE10C93067000938B8B0063DEE60046
:102580001306410D9305090013850900EF6090586B
:1025900063100564938B0A0063540B00130B000057
:1025A000330B6D41635E6005930D000113037000F2
:1025B000832701010327810D8326C10D23A0FB0082
:1025C0001307170013868B0063C06D1B23A26B01DA
:1025D000330BDB00232E610D232CE10C93067000DE
:1025E000930B060063DEE6001306410D9305090018
:1025F00013850900EF601052631C055C938B0A0081
:1026000093770440338BA40163840702B3874401AA
:10261000930D7000138D07008327C10063940C187D
:1026200063940718B387440163F46701138B0700B1
:102630008327C10B63C6470193771400638A07049D
:10264000832701030327C101938B8B0023ACFBFE7F
:102650008327C10123AEFBFE8327C10DB387E700AB
:10266000232EF10C8327810D130770009387170029
:10267000232CF10C635EF7001306410D930509004E
:1026800013850900EF60104963140554938B0A0009
:10269000B3844401B38764418324C10BB3049A40DB
:1026A00063D4970093840700635490048327C10D7B
:1026B00023A06B0123A29B00B387F400232EF10C0F
:1026C0008327810D13077000938B8B00938717006E
:1026D000232CF10C635EF7001306410D93050900EE
:1026E00013850900EF6010436314054E938B0A00B5
:1026F0009387040063D40400930700008324C10B74
:10270000B3049A40B384F440E35C90C2130B00011D
:10271000930C7000032601018327810D0327C10D4F
:1027200023A0CB009387170093868B0063449B20E4
:1027300023A29B00B384E400232E910C232CF10CE4
:1027400013077000938B0600E35CF7BE1306410D80
:102750009305090013850900EF60D03B631A054615
:10276000930BC10F6FF0DFBD9386060123A2BB015F
:10277000232ED10C232CE10C6350E3021306410DF0
:102780009305090013850900EF60D03863120544F2
:1027900013860A0013037000130B0BFF930B060044
:1027A0006FF01FE16386070E8327C1009387F7FF51
:1027B0002326F100832741030327C102938B8B005B
:1027C00023ACFBFE8327C10223AEFBFE8327C10D92
:1027D000B387E700232EF10C8327810D9387170021
:1027E000232CF10C63DEFD001306410D9305090057
:1027F00013850900EF601032631C053C938B0A00BF
:102800008327810033076D4183C707006354F700B6
:10281000930707006356F0040327C10D23A06B0143
:1028200023A2FB003387E700232EE10C0327810D51
:10283000938B8B0013071700232CE10C63D2ED025E
:102840001306410D93050900138509002320F104A7
:10285000EF60502C631E053683270104930BC10FD4
:102860001387070063D40700130700008327810044
:102870001308000183C70700B387E7406344F006ED
:102880008327810083C70700330BFB006FF0DFD87D
:1028900083278100938CFCFF9387F7FF2324F100AB
:1028A0006FF05FF19386060123A20B01232ED10C5A
:1028B000232CE10C63D4ED021306410D93050900AE
:1028C000138509002320F104EF60D0246312053042
:1028D000832701041306C10F13080001938707FF24
:1028E000930B0600832501010327810D8326C10D6B
:1028F00023A0BB001307170013868B00E344F8FAEC
:1029000023A2FB00B387D700232EF10C232CE10C6C
:10291000930B0600E3D6EDF61306410D930509006F
:1029200013850900EF60101F6314052A930BC10F74
:102930006FF01FF51307070123A26B01232EE10C93
:10294000232CF10C63DEFC001306410D93050900F6
:1029500013850900EF60101C631C05269306C10F48
:10296000938404FF938B06006FF0DFDA8327810DD9
:102970009306100023A09B001307170093871700EE
:10298000938C8B0063C64601137614006306061C05
:1029900093061000232EE10C23A2DB00232CF10C64
:1029A00013077000635EF7001306410D93050900DD
:1029B00013850900EF601016631C0520938C0A0034
:1029C000832701030327C101938C8C0023ACFCFEF9
:1029D0008327C10123AEFCFE8327C10DB387E70027
:1029E000232EF10C8327810D1307700093871700A6
:1029F000232CF10C635EF7001306410D93050900CB
:102A000013850900EF6010116314051C938C0A00F4
:102A10008327010E930501091305010A2320F10AFA
:102A20008327410E130BFAFF232801082322F10A02
:102A30008327810E232A0108232C01082324F10A6D
:102A40008327C10E232E01082326F10AEFA0403967
:102A5000630605088327C10D0327810D93841400A5
:102A60009387F7FFB38747011307170023A09C0044
:102A700023A26C01232EF10C232CE10C9307700090
:102A8000938C8C0063DEE7001306410D930509006B
:102A900013850900EF601008631C0512938C0A006F
:102AA0009307410C23A0FC008327810303278103A4
:102AB000938B8C0023A2FC008327C10DB387E70012
:102AC000232EF10C8327810D1307700093871700C5
:102AD000232CF10CE356F7866FE09F80E35260FDF4
:102AE00093040001130D7000032601010327810DDB
:102AF0008327C10D23A0CC001307170093868C00F9
:102B000063C06403B307FB0023A26C01232EF10C06
:102B1000232CE10C93077000938C06006FF09FF656
:102B20009387070123A29C00232EF10C232CE10C98
:102B3000635EED001306410D93050900138509003E
:102B4000EF60407D6316050893860A00130B0BFFA8
:102B5000938C06006FF05FF9232EE10C23A2DB00BB
:102B6000232CF10C13077000E35CF7F26FF0DFF138
:102B700083274102032781023384E740635680FCA8
:102B8000B7070081130B00019384C737930C7000C3
:102B90008327810D23A09B000327C10D9387170076
:102BA00063448B0423A28B003304E400232E810CA6
:102BB000232CF10C130770006358F7F81306410D2E
:102BC0009305090013850900EF60C074630E05F6D4
:102BD00063140C006FE09F9793050C0013850900A8
:102BE000EF0050106FE09F961307070123A26B01BF
:102BF000232EE10C232CF10C938B8B0063DEFC0065
:102C00001306410D9305090013850900EF608070DC
:102C1000E31005FC938B0A00130404FF6FF05FF7C9
:102C200093050C0013850900EF00D00B6FF0CFF572
:102C30008327C10D639407006FE05F911306410D78
:102C40009305090013850900EF60C06C6FE01F90C9
:102C50001307F0FF6392EDB063140DB813079000F3
:102C6000636097B913880C03A30F01199304F1193A
:102C70006FF08FB4B7270081930606001386050016
:102C80009305050003A587986FD0DFF983D7C500AA
:102C9000130101B8232C814693F7D7FF231AF100C3
:102CA00083A7450613840500232A91462326F106AF
:102CB00083D7E50023282147232E1146231BF1004B
:102CC00083A7C50113090500232001022322F10275
:102CD00083A74502930581002326F102930701078C
:102CE0002324F100232CF100930700402328F10056
:102CF000232EF100EFD01FF393040500634C050071
:102D00009305810013050900EF00003863040500F6
:102D10009304F0FF8357410193F70704638807008A
:102D20008357C40093E707042316F4008320C147A8
:102D30000324814713850400032901478324414765
:102D40001301014867800000130101FFB7270081CC
:102D5000232291009304050003A587982324810072
:102D600023261100138405006308050083278503CB
:102D700063940700EF00004B0317C400931707018B
:102D800093D7070193F68700639E060693F6070123
:102D9000639606029307900023A0F40013670704CC
:102DA0002316E4001305F0FF8320C10003248100F3
:102DB00083244100130101016780000093F747005D
:102DC000638C070283250403638C050093070404C6
:102DD0006386F50013850400EF00C0702328040209
:102DE0008357C4002322040093F7B7FD2316F40091
:102DF000832704012320F4008357C40093E787004E
:102E00002316F40083270401639007028357C4004C
:102E10001307002093F707286388E7009305040051
:102E200013850400EF20502D8357C40013F71700BB
:102E3000630C07028327440123240400B307F040F6
:102E4000232CF4008327040113050000E39E07F4FC
:102E50008317C40013F70708E30807F493E7070490
:102E60002316F4006FF01FF493F7270013070000F8
:102E700063940700032744012324E4006FF09FFCC0
:102E80008397C500130101FE232C810013970701CE
:102E900013570701232A9100232E11002328210113
:102EA00023263101937687009304050013840500DF
:102EB000639C06163717000013070780B3E7E70087
:102EC00003A745002396F5006346E00203A7C50368
:102ED0006342E002130500008320C1010324810145
:102EE00083244101032901018329C1001301010247
:102EF0006780000003278402E30E07FC03A9040097
:102F00009396370123A0040063D8060C032604051A
:102F10008357C40093F74700638E0700832744005C
:102F20003306F64083270403638607008327C40320
:102F30003306F640832784028325C40193060000EC
:102F400013850400E78007009307F0FF8356C40051
:102F50006312F50283A704001307D001636EF70A1A
:102F600037074020130717003357F7001377170070
:102F70006304070AB7F7FFFF9387F77F032704016E
:102F8000B3F7D7009397070193D707412320E400B5
:102F90002316F4002322040013973701635C070013
:102FA0009307F0FF6316F50083A7040063940700FE
:102FB0002328A4048325040323A02401E38C05F023
:102FC000930704046386F50013850400EF00805125
:102FD000232804026FF01FF08325C40113060000AC
:102FE0009306100013850400E70007009307F0FF25
:102FF00013060500E31EF5F083A70400E38A07F03B
:103000001307D0016386E700130760016392E706A8
:1030100023A024016FF01FEC93E706042316F400AD
:103020001305F0FF6FF05FEB83A90501E38409EA64
:1030300003A905001377370023A03501330939416F
:10304000930700006314070083A745012324F400BD
:10305000E35220E9832744028325C4019306090033
:103060001386090013850400E78007006348A00069
:103070008357C40093E707046FF05FFAB389A90090
:103080003309A9406FF0DFFC130101FE232C8100FE
:10309000232E110013040500630C0500832785030C
:1030A000639807002326B100EF00C0178325C100F5
:1030B0008397C500638C0700130504000324810176
:1030C0008320C101130101026FF09FDB8320C10146
:1030D0000324810113050000130101026780000031
:1030E00093050500631C0500B717008103A547E79A
:1030F000B7350080938585086F00006FB727008182
:1031000003A587986FF05FF8130500006780000043
:10311000130101FF2324810023261100130405005D
:103120002316B5002317C500232005002322050020
:10313000232405002322050623280500232A050051
:10314000232C050013068000930500001305C50518
:10315000EF201073B7770080938707172320F402BE
:10316000B77700809387871C2322F402B77700800B
:103170009387C7242324F402B77700809387472AD4
:10318000232E84002326F4028320C100032481001F
:103190001301010167800000B7A500809385452ACF
:1031A0006F0080641305000067800000130101FFB9
:1031B00023229100130680069384F5FFB384C40292
:1031C00023202101138905002324810023261100D7
:1031D00093854407EF2050011304050063000502A6
:1031E00023200500232225011305C5002324A40064
:1031F0001386840693050000EF20906813050400F1
:103200008320C1000324810083244100032901009D
:103210001301010167800000B717008103A547E78C
:103220006FF09FF783278503639E0706130101FF55
:10323000B737008023261100232481009387871944
:10324000232EF502930730002322F52E9307C52E77
:10325000130405002324F52E2320052E0325450005
:103260001306000093054000EFF09FEA0325840059
:103270001306100093059000EFF09FE90325C400AA
:103280001306200093052001EFF09FE8930710003C
:10329000232CF4028320C1000324810013010101C7
:1032A0006780000067800000130101FFB7170081ED
:1032B0002322910083A447E7232021012326110024
:1032C00083A7840323248100130905006396070064
:1032D00013850400EFF01FF59384042E03A48400EB
:1032E00083A744009387F7FF63DA070083A70400EE
:1032F0006380070883A404006FF05FFE0317C40017
:1033000063140706B707FFFF9387170023220406FD
:103310002320040023220400232404002326F40095
:1033200023280400232A0400232C04001306800011
:10333000930500001305C405EF20905423280402D0
:10334000232A040223220404232404041305040072
:103350008320C1000324810083244100032901004C
:103360001301010167800000130484066FF09FF7CA
:103370009305400013050900EFF05FE323A0A400CC
:10338000E31A05F69307C0002320F9001304000098
:103390006FF0DFFB6780000067800000678000003F
:1033A00067800000B727008103A58798B7350080A4
:1033B000938585106F004039B727008103A5879852
:1033C000B73500809385451A6F000038130101FE60
:1033D0002328210137190081232C8100232A910001
:1033E0002326310113840500232E110093090500C3
:1033F00013098940EF209056832789003717000072
:1034000083A447009307F7FE3384874093F4C4FFF7
:10341000330494001354C4001304F4FF1314C400C1
:103420006356E40213850900EF2090531305000052
:103430008320C10103248101832441010329010167
:103440008329C10013010102678000009305000079
:1034500013850900EF30903F83278900B3879700D9
:10346000E312F5FCB305804013850900EF30103EF0
:103470009307F0FF6310F50493050000138509001E
:10348000EF30D03C032789009306F000B307E540F6
:10349000E3DAF6F8B726008183A6C69893E717000B
:1034A0002322F7003305D540B726008123A0A69C30
:1034B0006FF05FF783278900B3848440372700814A
:1034C00093E4140023A297008327079C1385090027
:1034D000338487402320879CEF20904813051000F9
:1034E0006FF01FF563800526130101FF232481007F
:1034F0002322910013040500938405002326110064
:10350000EF20D04503A5C4FF37160081938684FFC2
:103510009377E5FF13088640B385F60003A74500BF
:1035200003288800130686401377C7FF137515001C
:103530006314B806B387E7006310050203A784FF8E
:10354000B386E64083A58600B387E70003A7C600DD
:1035500023A6E5002324B70013E7170023A2E60003
:1035600037270081032707992324D60063EAE70061
:10357000B727008183A5479F13050400EFF01FE5DF
:1035800013050400032481008320C100832441002B
:10359000130101016F20D03C23A2E50013080000B5
:1035A0006316050203A584FFB718008193880841BC
:1035B000B386A640B387A70003A586006306150B54
:1035C00083A8C6002326150123A4A8003385E5009F
:1035D000032545001375150063180502B387E7003E
:1035E00003A78500631608083715008113050541F8
:1035F0006310A708232AD6002328D60023A6E600B6
:1036000023A4E6001308100013E7170023A2E60026
:103610003387F6002320F700E31408F61307F01FA2
:103620006360F70693D7370093D527401307100040
:103630003317B70083254600938717009397370009
:10364000B307F6003367B7002322E60003A707009D
:10365000138687FF23A6C60023A4E60023A0D70075
:103660002326D7006FF0DFF1130810006FF01FF66C
:1036700083A5C5002326B70023A4E5006FF0DFF87B
:1036800093D59700130740006368B70413D767000A
:10369000130787039305170093953500B305B6000C
:1036A000138585FF83A505006314B50893071000F3
:1036B000135727403397E700832746003367F70007
:1036C0002322E60023A6A60023A4B6002324D500C7
:1036D00023A6D5006FF0DFEA130740016366B70049
:1036E0001387B5056FF01FFB130740056368B7002C
:1036F00013D7C7001307E7066FF0DFF9130740156C
:103700006368B70013D7F700130777076FF09FF8C8
:10371000130540551307E007E36EB5F613D72701ED
:103720001307C7076FF01FF783A585006308B5006F
:1037300003A745001377C7FFE3E8E7FE03A5C5002D
:103740006FF05FF867800000130101FD2324810200
:1037500023202103232C4101232A51012326110276
:1037600023229102232E31011304052E1309000098
:10377000130A1000930AF0FF631604028320C102AB
:103780000324810213050900832441020329010255
:103790008329C101032A8101832A41011301010305
:1037A0006780000083248400832944009389F9FF03
:1037B00063D60900032404006FF01FFC83D7C40004
:1037C0006370FA028397E400638C57011385040049
:1037D0002326B100E78005008325C1003369A900D5
:1037E000938484066FF09FFC130101FD2324810262
:1037F00023202103232C4101232A51012328610185
:10380000232671012326110223229102232E310146
:10381000130A0500938A05001304052E13090000FE
:10382000130B1000930BF0FF631A04028320C102F4
:1038300003248102130509008324410203290102A4
:103840008329C101032A8101832A4101032B01013C
:10385000832BC100130101036780000083248400CF
:10386000832944009389F9FF63D6090003240400E7
:103870006FF09FFB83D7C400637EFB008397E40057
:10388000638A77019385040013050A00E7800A0024
:103890003369A900938484066FF0DFFC9307450128
:1038A00013052500231F05FEE31CF5FE67800000BD
:1038B0009307000013074001B306F50003D6060086
:1038C000B386F500938727002390C600E396E7FEB2
:1038D000678000009307A50113052500231F05FE3F
:1038E000E31CF5FE678000009307000013078001CA
:1038F000B306F50003D60600B386F50093872700CC
:103900002390C600E396E7FE239C05006780000035
:10391000930740001306A0013307F5008356070004
:103920003387F50003570700638AE600130510008C
:10393000636CD7001305F0FF6780000093872700B2
:10394000E39CC7FC13050000678000009306450058
:10395000930700001305A5013786FFFF03D7060074
:10396000937517006384050093E7170093F527000C
:103970001357170063900502939717002390E600F2
:10398000939707019386260093D70701E318D5FC88
:10399000678000003367C7006FF01FFE9306650164
:1039A0001307000083D7260013960701135606411C
:1039B0006354060013671700939717009397070146
:1039C0001376270093D70701631006021317170019
:1039D0002391F600131707019386E6FF135707019B
:1039E000E312D5FC6780000093E717006FF01FFE1D
:1039F00093074500130700001305A50183D60700B0
:103A00009387270013D686003367C700239FE7FEFE
:103A1000139786001317070113570701E310F5FEEC
:103A200067800000930765011307000083D6270015
:103A30009387E7FF139686003367C7002392E7005A
:103A400013D78600E314F5FE678000009307450056
:103A5000130785019387270083D60700239FD7FE8E
:103A6000E31AF7FE231C0500678000009307850119
:103A7000130745009387E7FF83D607002391D700FC
:103A8000E31AF7FE23120500678000009385850185
:103A900013076501930600008357270003D605002E
:103AA0001307E7FF9385E5FFB387C700B387D70008
:103AB0002391F50093D7070193F61700E31EE5FC69
:103AC0006780000093858501130765019306000058
:103AD00083D705001307E7FF9385E5FFB387D7403A
:103AE00083564700B387D7402391F50093D707014A
:103AF00093F61700E31EE5FC67800000130101FE4A
:103B00003703010093888501231D0100231E010056
:103B1000938545009306C1011303F3FF03D7080003
:103B20009386E6FF9388E8FF631C0702239F06FE47
:103B3000E39615FF930740001307A001930541008A
:103B4000B385F50083D50500B306F60093872700FB
:103B50002390B600E394E7FE1301010267800000A2
:103B60003307A70203D82600B3776700B38707019E
:103B700013D807012391F6009357070103D70600D6
:103B8000B387E700B38707012390F60093D70701B7
:103B9000239FF6FE6FF0DFF98357250193C7F7FFE8
:103BA00013971701631C07009307250113052500D0
:103BB0000357E5FF63180700E39AA7FE130500000B
:103BC000678000001305100067800000130101FFEB
:103BD000232481002326110013040500EFF0DFFBEE
:103BE000631E0500031524011355F5018320C10050
:103BF0000324810013010101678000001305000008
:103C00006FF0DFFE83172501130101FF232611004A
:103C100023248100232291002320210163D8070659
:103C20009307F0FF2390F50003572501B7870000A5
:103C30009387F7FF33F7E7002391E50013090501A8
:103C40006316F7061384050093040500EFF0DFF414
:103C50006302050493076400231204001385C4FF64
:103C60001309E9FF0357290093872700239FE7FEE5
:103C7000E318A9FE8320C1000324810083244100AE
:103C80000329010013010101678000002390050052
:103C90006FF09FF9930744009305A40193872700D1
:103CA000239F07FEE39CB7FE6FF0DFFC9387650060
:103CB000239205001305E5FF1309E9FF03572900C7
:103CC00093872700239FE7FEE318A9FE239C0500A6
:103CD0006FF05FFA130101FB2322910423202105D9
:103CE000232611042324810413090500938405006D
:103CF000EFF09FEA6310050E13850400EFF0DFE993
:103D0000130405006318050C9305810013050900D1
:103D1000EFF05FEF9305410213850400EFF09FEE93
:103D200003578100835741026380E7069307200011
:103D300093068001130681003306F6000356060041
:103D4000631C0602130641023306F6000356060002
:103D50006314060293872700E39ED7FC1305040033
:103D60008320C10403248104832441040329010422
:103D7000130101056780000013041000E30007FE33
:103D80001304F0FF6FF09FFD13071000638407001A
:103D90001307F0FF9307000093058001930681004D
:103DA000B386F60003D6060093064102B386F600FA
:103DB00083D60600630AD60013040700E3E0C6FAC0
:103DC0003304E0406FF09FF993872700E398B7FC36
:103DD0006FF0DFF81304E0FF6FF05FF88357250101
:103DE00093C7F7FF1397170163100702130101FF31
:103DF00023261100EFF05FDA8320C1001335150090
:103E000013010101678000001305000067800000B6
:103E1000130725019307050093872700239F07FEBB
:103E2000E39CE7FE83572501378700001307F7FF60
:103E3000B3E7E7002319F50067800000130101FED6
:103E4000232C810023263101232E1100232A9100E7
:103E50002328210123244101232251019309050034
:103E60001384050063D205103309B040130A09001A
:103E700093040000930AF00063CE4A0313594900EB
:103E8000930500FFB305B902130A7000338485401F
:103E900013090400634C2A0393553400930780FFF1
:103EA000B385F50233848500631E04023335900028
:103EB0006F00400983D7890113850900130A0AFF9F
:103EC000B3E4F400EFF09FBA6FF01FFB83C78901E2
:103ED00013850900130989FFB3E49700EFF05FB180
:103EE0006FF05FFB83D78901138509001304F4FF8A
:103EF00093F71700B3E49700EFF05FA56FF0DFFAD8
:103F000013850900EFF09FB4938404FFE34A99FE00
:103F100093554400930700FFB385F5021309700021
:103F20003304B400930404006346990493553400A9
:103F3000930780FFB385F5023304B40063140404CF
:103F4000130500008320C101032481018324410162
:103F5000032901018329C100032A8100832A41002A
:103F60001301010267800000938405001309F0002B
:103F70006FF0DFF913850900EFF0DFAA938484FF67
:103F80006FF09FFA13850900EFF05FA11304F4FFAF
:103F90006FF0DFFA83574500130101FF23229100E0
:103FA00023261100232481002320210193040500EE
:103FB0006380070293F707F013040000638607008D
:103FC000EFF01FA3130480FF1309F0F66F00400900
:103FD00083176500130400001309000A63D8070261
:103FE000130504008320C1000324810083244100C1
:103FF00003290100130101016780000013850400FB
:1040000013040401EFF09FA4E30C24FD83D76400A4
:10401000E38607FE83D7640093F707F06382070205
:104020001309000A83976400E3CC07FA13850400A0
:1040300013041400EFF09F96E35689FE6FF05FFAC9
:1040400013850400EFF01F9E130484006FF09FFCA3
:10405000138504001304F4FFEFF05F8FE30224F9EB
:1040600083D74400E39607FE6FF09FF7130705011F
:104070009307050093872700239F07FEE39CE7FE35
:10408000B7C7FF7F2328F5006780000013070500EE
:1040900083560700138505008357270063860600B3
:1040A000B786FFFFB3E7D7002319F50003562700B3
:1040B000B78600009386F6FF93076700631ED6005D
:1040C0001307A70183D6070063980602938727008A
:1040D000E39AE7FE6FF0DFD31305050113078701AD
:1040E0009387270083D6E7FF1305E5FF2311D5004B
:1040F000E398E7FE678000006FF05FF7130101FDB2
:104100002322910293040500130541002324810218
:104110002326110213840500EFF0CFFB03D7E40040
:104120009317070193D7074163C2070423120100C5
:10413000B78600009386F6FF3377D7009387E400B5
:10414000631CD706138704008356070063860602A4
:1041500013050400EFF09FF18320C10203248102C4
:104160008324410213010103678000009307F0FFDD
:104170002312F1006FF0DFFB13072700E396E7FC43
:1041800013050400EFF08FF113050400EFF05FC892
:104190008397E400E3D207FC13050400EFF0DF9FF0
:1041A000E31C05FA835724013787FFFFB3C7E700F5
:1041B0002319F4006FF05FFA2313E1009306410026
:1041C0009387E7FF03D60700938626002392C60055
:1041D000E398F4FE631C0700231401009305040018
:1041E00013054100EFF09FEA6FF01FF793071000EF
:1041F0009305F0FF130541002314F100EFF01FC4F5
:104200006FF0DFFD130101FE232C8100232A9100B2
:104210002328210123263101232441012322510196
:104220001389060013840700232E11009304050050
:1042300093890500130A0600930A0700EFF09FD543
:10424000930700093309A94063D4A704B787000086
:104250009387E7FF63CC2705938724009384A40109
:1042600093872700239F07FEE39C97FE8320C101CD
:104270000324810183244101032901018329C10011
:10428000032A8100832A4100130101026780000094
:10429000635E0900930700F76344F918930509006A
:1042A00013850400EFF09FB96318051863800A14A2
:1042B00003274400832704006306F7061305A401BF
:1042C000EFF04FE183274400130780036386E71C68
:1042D0006348F71613078001638EE71E1307500328
:1042E000638AE71C1307C0002324E400370701801A
:1042F0001307F7FF232AE40013071000231CE40030
:104300001307B0002326E4000327C400835684016A
:1043100013078700131717003307E4002315D7008E
:104320002320F4006342200303274400930700097D
:10433000630CF70083D784011385040093F71700FB
:10434000B3E9F900EFF08FE08326840003564401BF
:1043500083254400139716003387E4008357070032
:10436000B3F7C7001306F008634AB6009386160039
:10437000130607009305C00063D2D5168356440187
:104380000356070093C6F6FFB3F6C6002310D70006
:1043900003576401B376F700638406026310F716CF
:1043A000639C09148327C400035784019397170063
:1043B000B387F40083D70700B3F7E70063900714CF
:1043C000634C200103274400930700096306F700AC
:1043D00013850400EFF08FDC83D744006388070067
:1043E00013850400EFF08FD613091900B78700007A
:1043F000239C04009387E7FF63DA2711B787FFFF49
:1044000093C7F7FF2391F4009387440093848401BA
:104410002390070093872700E39CF4FE6FF01FE5CD
:10442000938724009384A40193872700239F07FE8A
:10443000E39C97FE6FF09FE3930910006FF01FE776
:10444000130700046388E70213071007E39CE7E8FB
:10445000378700401307F7FF9306A000232AE400E4
:104460002324D4003787FFFF231CE4002326D40035
:104470006FF09FE9130770002324E40037070180E1
:104480001307F7FF232AE40013071000231CE4009E
:10449000130760006FF01FE7930660003707800086
:1044A0001307F70F232AE4002324D4001307001076
:1044B0006FF09FFB370700041307F77F9306600038
:1044C000232AE400371700002324D40013070780B1
:1044D0006FF09FF9930640006FF05FFC03552600D4
:1044E0006304050093E71700231106009386160066
:1044F000130626006FF05FE8E3140AEC93850400CE
:104500001305A401EFF08FD86FF09FEB63560900FD
:10451000239104006FF09FD5239124016FF01FD5E4
:10452000130101FE23244101035A2500232C81009D
:1045300013840500232E1100232A91002328210132
:10454000232251012320610113090600130B4603A6
:1045500023263101930A0500EFF0DFA383542400E2
:10456000330AAA4013050400EFF0DFA2B384A4408D
:1045700013050B00EFF00FB663D2440513050400DA
:10458000032481018320C1018329C100032A810002
:10459000832A4100032B010093070900938604003E
:1045A00003290101832441011307000013060000C1
:1045B00093050000130101026FF0DFC493050400AE
:1045C00013850A00EFF0CFB493090000634AA000FE
:1045D0009305040013850A00EFF0CFCE9309100075
:1045E00013050B00EFF08FBB8357C90413050400BC
:1045F0009384F4FFB3E9F90023163905EFF00FBAFD
:104600006FF09FF7130101F72324810823229108FB
:1046100023202109232C410723261108232E3107AB
:10462000232A5107232861072326710723248107A2
:10463000130905001384050093040600138A06007D
:10464000EFF08FD56300050493850400130509007E
:10465000EFF00FA68320C1080324810883244108BA
:10466000032901088329C107032A8107832A4107F7
:10467000032B0107832BC106032C810613010109BB
:104680006780000013050400EFF00FD163080500F8
:1046900093850400130504006FF09FFB13050900C8
:1046A000EFF0CFF36314050613050400EFF00FF3EA
:1046B000630C0500B70500819385853D130509004E
:1046C000EFF04FE1630E050413050900EFF00FF161
:1046D0006318050013050400EFF04FF0630C0504A8
:1046E00013050900EFF08FCE130905001305040030
:1046F000EFF0CFCD630CA902B787FFFF2399F40039
:1047000013850400EFF0CFF06FF0DFF4B705008100
:104710009385853D13050400EFF0CFDBE31605F824
:1047200013850400EFF09F946FF0DFF223990400EB
:104730006FF01FFD9305C10013050900EFF08FCC4A
:104740001305040093058102EFF0CFCB8359E100FC
:104750000354A102638A090E8357A102130B0400BC
:10476000638007108327810213094A03930BEA042D
:10477000232AFA0293078A032390070093872700CE
:10478000E39C77FF1304C100130C81FF930A000020
:1047900003558401630E050093058102130641044D
:1047A000EFF0CFB59305090013054104EFF00FAE0C
:1047B0008357CA04130509001304E4FFB3EAFA009F
:1047C000EFF0CFAAE3168CFC930509009307810252
:1047D00003D705009385250093872700239FE7FED5
:1047E000E39875FFB7C6FFFFB3896901938626007A
:1047F00093070A0013070004B386D90013060000CC
:1048000093850A0013058102EFF0DF9F0357C10073
:1048100083578102631AF70623140102938504006B
:1048200013058102EFF09F866FF0DFE29387270088
:1048300083D62700638E06001305C100EFF08FF5C5
:10484000B309A0406FF05FF19307C10013070102A5
:10485000E39EE7FC13850400EFF04F846FF09FDFC9
:10486000930781021307C103E386E7FE93872700BE
:1048700083D62700E38A06FE13058102EFF08FF14D
:10488000330BA4406FF01FEE9307F0FF2314F102E7
:104890006FF0DFF8130101F7232481082322910828
:1048A00023202109232A510723261108232E31070B
:1048B000232C41072328610723267107232481071E
:1048C00023229107130905001384050093040600B1
:1048D000938A0600EFF04FAC630205049385040051
:1048E00013050900EFE0DFFC8320C10803248108E1
:1048F00083244108032901088329C107032A81076A
:10490000832A4107032B0107832BC106032C810651
:10491000832C410613010109678000001305040080
:10492000EFF08FA7630805009385040013050400CA
:104930006FF05FFBB70900819385893D130509007E
:10494000EFF04FB96306050413050900EFF00FC936
:104950009309050013050400EFF04FC8639809049C
:10496000630E050413050900EFF04FA613090500B7
:1049700013050400EFF08FA5630AA920B787FFFF96
:104980002399F40013850400EFF08FC86FF0DFF572
:104990009385893D13050400EFF0CFB3E31605FAC4
:1049A00013850400EFF08FEC6FF01FF4E31A05FE9F
:1049B00013850400EFE09FEE6FF01FF3130509006D
:1049C0009305C100EFF00FA41305040093058102C5
:1049D000EFF04FA30359A1020354E100630A091445
:1049E0008357E100930B04006386071803278102B5
:1049F00093878A03138BEA0423AAEA0293890700A8
:104A000093872700239F07FEE39C67FF130581021E
:104A1000EFE0DFF3035C2101370A0100130AFAFF1C
:104A2000B30C4C038357C1020354E102939707016F
:104A3000B387870013040A0063E8FC0033D48703BC
:104A400013140401135404019305C1001305040059
:104A500013064104EFF08F8A930581021305410488
:104A6000EFE01FEB6356A002930541041305C1005C
:104A7000EFF04F859305810213054104EFE05FE9F4
:104A8000634AA0101304F4FF131404011354040127
:104A90009305810213054104EFF0CF8213058102D3
:104AA0002390890093892900EFE05FFAE31C3BF72C
:104AB000130781029306E1039307070093050000A3
:104AC00003D6470093872700B3E5C500E39AF6FEB7
:104AD000B335B00093874A0383D607009387270036
:104AE00013072700231FD7FEE318FBFEB74600007D
:104AF000330979419386F6FF93870A001307000470
:104B0000B306D9001306000013058102EFF08FEF02
:104B10000357C10083578102631CF7082314010265
:104B20009385040013058102EFF04FD66FF0DFDBB1
:104B3000930781021307C103E38CE7E693872700FD
:104B400083D62700E38A06FE13058102EFF08FC4A7
:104B50003309A0406FF0DFE89387270083D6270052
:104B6000638E06001305C100EFF0CFC2B30BA44063
:104B70006FF0DFE79307C10013070102E39EE7FC34
:104B80000357C10083578102E31AF7DE239904001B
:104B90006FF05FDF1304E4FF131404019305410475
:104BA0001305C10013540401EFE0DFF16FF05FEE75
:104BB0009307F0FF2314F1026FF09FF603AE050098
:104BC00003A3450083A8850083A5C500130101E266
:104BD000232C811C2326B10213840700832505049E
:104BE0009307F0FF2328F114930700092324411DA4
:104BF0002320611D232A911B2328A11B232E111C76
:104C0000232A911C2328211D2326311D2322511DD7
:104C1000232E711B232C811B2326B11B232801016A
:104C20002320C1032322610223241103232AF11428
:104C3000130A0500130B0600938C0600130D0700E2
:104C40006380050283274504130710003317F7001C
:104C500023A2F50023A4E500EF10405B23200A0403
:104C60001305010293050105EFF04FC91305010576
:104C7000EFE0DFF56300050E930710002320F4003A
:104C800093073000630CFB0C93094001630A0B008F
:104C90009389FCFF9307A00263D437019309A00214
:104CA0008327411513050105232AF100EFE0DFEE0C
:104CB000930B05006308050AB70500819385C5625B
:104CC0001305411137240000EF2040431304F47012
:104CD000832741011305010523208116232AF1149E
:104CE000EFF0CF8F1309411163180500130501057B
:104CF000EFE09FEAE30E0514B72700009387F770F3
:104D00002320FD0093070900130600029306D0023A
:104D100003C70700E30CC718E30AD7189304090078
:104D20009387170003C7F7FF93861400A38FE6FE4F
:104D3000E312071813072000930710006308EB0025
:104D40009387090063D48900930704009306000346
:104D50006F005017232004006FF09FF293890C001E
:104D60006FF05FF3930700099305C1061305010572
:104D7000232AF114EFE0DFB38357E107232001007A
:104D80001397070113570741635E070093971701B5
:104D900093D71701231FF106B70701009387F7FF89
:104DA0002320F100370400811305843D9305810819
:104DB00013058511EFE0DFAF0357E10737090081E5
:104DC000232481009304843D1309094FE312071C37
:104DD0009307C1061307E10783D607006394061003
:104DE00093872700E31AF7FE130400009305010CD4
:104DF00013058108EFE01FE1930581081305010CFD
:104E0000EFE09FAE9305010C1305C106EFE09FDFB5
:104E10009305C1061305010CEFE01FAD1306011544
:104E20009305C10613058108EFF08FEF8354C11974
:104E3000639C0400832781001305C1069385873D89
:104E4000EFE05FE9631C056683270100638E076A54
:104E50009307D002230AF110930730001389090049
:104E6000631AFB00338989009307A00263D42701EA
:104E70001309A0029307A000639CF4689307100332
:104E8000A30AF1109307E002230BF11093047111B0
:104E9000635A200193070003A30BF1101309F9FFD4
:104EA0009304811113041400635E0966B705008141
:104EB000130604009385056513850400EF20002484
:104EC0006FF01FE1B7050081938505646FF05FDF28
:104ED0008317C10763C80700B70500819385C564C0
:104EE0006FF01FDE9305C10613050900EFE09FDE9A
:104EF000E30C05EE635A05429305410A1305C1060A
:104F0000EFE01F9BB74700009387E708231BF10AD8
:104F1000930700012322F100B78700009387F7FF72
:104F2000232CF100B7C7FFFF93872700130400006D
:104F3000138C440B232EF1009306011513068108F0
:104F40009305410A13050C00EFF0DF949305C103AC
:104F500013058108EFE0DF9583278101835AE1047F
:104F6000B3FDFA008327C101B38DFD00634AB0058C
:104F70001305010CEFE09F92939A0A0193DA0A411C
:104F800063D40A10930700001307C1033307F70027
:104F9000835607001307010C3307F7000357070078
:104FA000638CE63613050900EFE01FBF63020508B6
:104FB0009305010C13050900EFE09F8F6F00C00CF3
:104FC00093070009B38DB7419305010C1305C10385
:104FD000EFE01F8E635AB00B1307010C93870D008F
:104FE0009306F00063CEF60293D74D001397170097
:104FF0009306010C3387E600930600FFB387D702C0
:1050000083560700B387B70193971700B387F4005F
:1050100083D7C712B3F7D7002310F7006FF0DFF57F
:1050200023100700938707FF130727006FF09FFBEC
:105030001305010CEFE05FB6630805009305010C52
:10504000138505006FF05FF713050900EFE01FD926
:10505000930A05001305010CEFE05FD8930D0500DE
:1050600063840A14630C051013050900EFE01FB6F2
:10507000930A05001305010CEFE05FB56390AA10D9
:105080001305010CEFE09FFE930700001307810852
:105090003307F700835607001307010C3307F700A7
:1050A000035707006392E602938727001307200146
:1050B000E39EE7FC9305410A13058108EFE04FFFEB
:1050C000832741003304F40083274100130C4C0173
:1050D000938D440193D717002322F1009387841105
:1050E000E31CFCE48357610B0357E1079305C106FA
:1050F0001305410AB387E70037C7FFFF130727F7F8
:10510000B387E700231BF10AEFE08FFA93058108CC
:1051100013050C00EFE0CFF9B71A00009384441098
:105120009305410A13850400EFE0DFBAE340A0CC09
:105130009305410A13850D00EFE0DFB96348A00233
:105140001306410A930506009306011513850D0009
:10515000EFF04FF41306810893060115930506003E
:1051600013850D00EFF00FCA3304540193DA1A00CF
:10517000E38E9DC6938D4D016FF09FFA13050900D4
:105180009305010CEFE0CFF21305010CEFE0DFA077
:10519000E31C05EE8357210D3787FFFFB3C7E700F8
:1051A0002319F10C6FF05FEEE31A05E89305C10DCA
:1051B00013050900EFE01FA59305810F1305010CEE
:1051C000EFE05FA48357C10D835AA10F93C7F7FF88
:1051D000231EF10C8357E10DB38557412326F100BF
:1051E000635AB002930541111305810FEFE0CFEF31
:1051F0009305810F1305C10DEFE00FEF9305C10D6E
:1052000013054111EFE04FEE8327C100B385FA404B
:10521000835AA10F638805049307F0F663C4F50869
:105220001305C10DEFE09FC12326A1000357C10D57
:105230008357810F9305810F1305C10D6318F70C78
:10524000EFE0DF848325C1009307011513070004F5
:1052500093860A0013860D001305810FEFE09FFA75
:105260006F0040049305810F1305C10DEFE04FEA75
:10527000631605060357C10D8357810F6308F700B6
:105280001305010CEFE08FE16FF01FE08357A10FD2
:10529000639207028317E10F63CE07001305810FA6
:1052A000EFE0CFEF9305010C1305810FEFE01FDE58
:1052B0006FF09FDD9307810F1307E11083D627005E
:1052C00063880600938A1A00231D510F6FF09FFD1B
:1052D00093872700E314F7FE6FF01FFF23260100DA
:1052E000E356A0F4930541111305810FEFE0CFDFE2
:1052F0009305810F1305C10DEFE00FDF9305C10D7D
:1053000013054111EFE04FDE6FF05FF2EFE08FFB2E
:10531000930D10006FF01FF39387270013072001F0
:10532000E394E7C66FF05FD68357E10713040000EC
:10533000938A44106388070A9305010C1305C1067C
:10534000B74A0000EFE01F8C938AEAFF130C50FD70
:105350008357810D93F77700639207069305410AFF
:105360001305010CEFE04FD81305410AEFE00FDE03
:105370001305410AEFE08FDD9305410A1305010C87
:10538000EFE0CFF08357610A938737002313F10AC8
:105390008357810A639A07108357C10B63900702F2
:1053A0008357610A63ECFA009305010C1305410A67
:1053B0001304F4FFEFE04FD3E31C84F99305C10617
:1053C0001305010CEFE09FCC6F0040021306C106ED
:1053D000930601159305060013850A00EFF08FA2CE
:1053E0001304F4FF8317C107E3D207FE9305010CF2
:1053F0001305C106EFE0CFCB930581081305090023
:10540000EFE00FCB93874401130C0000B7FAFFFFC6
:105410002322F100930D2000B70700819387875264
:1054200033878701832741009305010C1305090089
:105430002326E100B3848701EFE0DF890327C10061
:105440006358A0049305010C13050700EFE09F8843
:10545000634805021306010C930506009306011527
:1054600013850400EFF00F9A1306810893060115C7
:105470009305060013850400EFF0CF983304540120
:10548000130C4C0193074010B3CABA03E316FCF89F
:1054900013068108930601159305090013050600FC
:1054A000EFF04FBF6FF09F941305410AEFE00FCA72
:1054B0008357610A938717006FF05FED1305C106EC
:1054C000EFE0CFCD9305410A1305C106EFE0CFC150
:1054D0001305410AEFE08FCC1305410AEFE00FCC32
:1054E0009305C1061305410AEFE04FDA13060115D3
:1054F0009305C10613058108EFF08F821304F4FFB2
:105500008354C1196FF0DF92930700026FF09F94EC
:10551000938404039307E002A30A9110230BF11074
:1055200093047111B38A7401635679058357C119C5
:10553000130740009384FAFFE35AF79613075000CD
:105540006384E708938704001306E0029305800351
:10555000930600039387F7FF03C707001377F70746
:105560006358090A130710032380E700130414008B
:105570006FF0DF931305C106EFE04FC29305410AB8
:105580001305C106EFE04FB61305410AEFE00FC166
:105590001305410AEFE08FC09305C1061305410AC8
:1055A000EFE0CFCE130601159305C1061305810860
:1055B000EFE01FF78347C119938B1B009387070305
:1055C0002380FA006FF01FF6930581081305C106CA
:1055D000EFE0DFAB83278100130581089385873DCA
:1055E000EFE04FEFE31005F6E342098C83C7EAFFD3
:1055F000938727FD93B7170093C7F7FFB387F4008E
:1056000083C7070093F71700E39E07F26FF01F8A26
:105610006314C70203C7F7FF9306800363E8E6003D
:1056200013071700A38FE7FE6FF05F8813041400C1
:10563000130710036FF01FFF63E8E500130717005F
:105640002380E7006FF09F862380D7006FF09FF0E4
:10565000930714002320FD009306E002930709003E
:1056600003C7070063160700130750046F00C0024A
:10567000138617006306D700930706006FF05FFEDE
:1056800003C7170093871700A38FE7FEE31A07FEEF
:105690006FF09FFD9387F7FF83C607006384E600E2
:1056A000E36AF9FE238007006FF0CFE593871700C8
:1056B0006FF00FE6938406006FF08FE69384F4FF9B
:1056C0002380040003C7F4FF6316D7003387244107
:1056D000E3C6E7FE1307300093879C006312EB02DA
:1056E0003384890063580400230A011023200D002D
:1056F0009304090083270D00B38CFC0093873C00C2
:1057000023220A04130740009306470183254A0415
:1057100063F8D70613050A00EF00D0242320AA045B
:105720009305090013040500EF1050388327010189
:1057300063880700B3842441B304940023A0970036
:10574000130504008320C11D0324811D8324411DF2
:105750000329011D8329C11C032A811C832A411CA2
:10576000032B011C832BC11B032C811B832C411B8E
:10577000032D011B832DC11A1301011E6780000038
:10578000938515002322BA04131717006FF0DFF773
:10579000B78700009387F7FF631CF7F283270100A8
:1057A000638207F2B7050081938545636FF04FD19F
:1057B00083270500130101FC930541012320F1001B
:1057C00083274500232E11022322F1008327850021
:1057D0002324F1008327C500130501002326F100CF
:1057E000EFE0DF91835761021305000093C7F7FFD5
:1057F00013971701631A070013054101EFE0CFB9B2
:1058000013351500130515008320C103130101048E
:10581000678000001305050F67800000B72700812F
:1058200083A7879803A547036316050037250081E2
:10583000130505811305050F67800000B727008158
:1058400083A7879803A547036316050037250081C2
:10585000130505811305050F67800000130101F88A
:10586000232A9106938405008395E500232C810665
:10587000232E11061304060063DE050083D7C4003F
:1058800023A0060093F707086398070493070040D6
:105890006F00C004130681012326D100EF40D048D9
:1058A0008326C100E34C05FC0327C101B7F70000C4
:1058B00037150000B3F7E70037E7FFFFB387E700CE
:1058C00093B7170023A0F600930700402320F400AD
:1058D000130505806F000001930700042320F400E6
:1058E000130500008320C107032481078324410797
:1058F000130101086780000083D7C500130101FE72
:10590000232C8100232E1100232A9100232821011A
:1059100093F7270013840500638807029307340474
:105920002320F4002328F40093071000232AF40016
:105930008320C10103248101832441010329010142
:1059400013010102678000009306C1001306810065
:1059500093040500EFF09FF08325810013090500F3
:1059600013850400EF004008631005028317C4008C
:1059700013F70720E31E07FA93F7C7FF93E7270003
:105980002316F4006FF09FF9B737008093878719CB
:1059900023AEF4028357C4002320A4002328A400CC
:1059A00093E707082316F40083278100232AF400D5
:1059B0008327C100638207028315E4001385040076
:1059C000EF508001630A05008357C40093F7C7FFB7
:1059D00093E717002316F4008357C4003369F900D6
:1059E000231624016FF0DFF4130101FD23261102B9
:1059F000232481022322910223202103232E31011B
:105A0000232C4101232A51012328610123267101FE
:105A100023248101232291019387B500130760019C
:105A20006376F70493F487FF63D404049307C000FC
:105A30002320F500130500008320C1020324810206
:105A400083244102032901028329C101032A810120
:105A5000832A4101032B0101832BC100032C810008
:105A6000832C4100130101036780000093040001AF
:105A7000E3EEB4FA93090500EF00406E3719008198
:105A80009307701F1309894063EA97041387840002
:105A90003307E90003244700930687FF93D73400B8
:105AA0006318D4000324C700938727006300870886
:105AB000832744000327C4008326840093F7C7FF8D
:105AC000B307F40023A6E6002324D70003A747006A
:105AD0001367170023A2E7006F00800A13D7940012
:105AE0009307F003630A07009307400063E2E70AA5
:105AF00093D7640093878703138717001317370022
:105B00003307E90003244700930587FF1305F000DE
:105B1000630CB400032744001377C7FF3306974094
:105B20006350C50C9387F7FF93871700032409017F
:105B3000B715008193068900938505416308D41247
:105B4000032744001306F0001377C7FF330597407F
:105B5000635AA60A93E714002322F4003306940044
:105B6000232AC9002328C900936715002326D600DD
:105B70002324D6002322F6003307E4002320A700C5
:105B800013850900EF00C05D130584006FF0DFEAA4
:105B90009307400163E6E7009307B7056FF0DFF571
:105BA0009307400563E8E70093D7C4009387E706AF
:105BB0006FF09FF49307401563E8E70093D7F40074
:105BC000938777076FF05FF3930640559307E007DD
:105BD000E3E4E6F293D724019387C7076FF0DFF180
:105BE0008326C400634C06008327840023A6D700C5
:105BF00023A4F600B307E4006FF05FED1384060002
:105C00006FF01FF1232AD9002328D900634C050027
:105C10003307E4008327470093E717002322F700A8
:105C20006FF01FF69306F01F0328490063E0E618A3
:105C30001357370013562740930610001307170019
:105C4000B396C600131737003307E900B3E6060121
:105C50002322D90083260700130687FF2326C400CA
:105C60002324D4002320870023A6860013D72740AF
:105C7000130310003313E30003274900636A670628
:105C8000B3766700639C060093F7C7FF13131300F6
:105C9000B376670093874700E38A06FE130EF00091
:105CA00093963700B306D9001388060013850700C2
:105CB0000324C800631C041B13051500137735006B
:105CC00013088800E31607FE13F73700631E07204A
:105CD000032749009347F3FFB377F7002322F90026
:105CE0000327490013131300636467006312032240
:105CF000832B890003A44B00937AC4FF63E89A00C6
:105D000033879A409307F00063CEE732B7270081CC
:105D1000372A008103A4479F0327CA989307F0FFFF
:105D2000B38C5B01338484006318F71E13040401F1
:105D30009305040013850900EF1040319307F0FF2D
:105D4000130B05006306F5286374950163922B29F4
:105D5000372C008193060C9C03A70600130C0C9CA7
:105D60003307E40023A0E60063946C1D93974C0175
:105D70006390071C8327890033848A00136414000E
:105D800023A287003727008183270C008326079FE3
:105D900063F4F6002328F79E372700818326C79EE9
:105DA00063F8F6222326F79E6F0080221356970091
:105DB0009306400063E6C604935667009386860305
:105DC00013861600131636003306C900130586FF26
:105DD000032606006312C50893D626401307100059
:105DE000B316D700B3E606012322D9002326A40068
:105DF0002324C40023248500232686006FF01FE798
:105E00009306400163E6C6009306B6056FF05FFB9C
:105E10009306400563E8C6009356C7009386E606DE
:105E20006FF01FFA9306401563E8C6009356F7001B
:105E3000938676076FF0DFF8130540559306E00769
:105E4000E360C5F8935627019386C6076FF05FF7A6
:105E5000032686006308C5008326460093F6C6FF26
:105E6000E368D7FE0325C6006FF05FF80327440000
:105E70000326C4001377C7FFB308974063501E057D
:105E800093E714002322F40083278400B3069400D0
:105E90003307E40023A6C7002324F600232AD900F1
:105EA0002328D90093E7180023A6B60023A4B60040
:105EB00023A2F600232017016FF09FCC63C20802D3
:105EC0003307E4008327470093E717002322F700F6
:105ED0008327840023A6C7002324F6006FF05FCA3F
:105EE000130406006FF01FDD938686FF03A786006C
:105EF0009387F7FFE30AD7DC6FF09FDE93874700B5
:105F000013131300B3766700E38A06FE6FF05FD9C0
:105F1000930705006FF01FFF371700001307F70006
:105F20003304E400B7F7FFFF3374F4006FF05FE071
:105F30008326CA989307F0FF6390F60C23266A998C
:105F4000937C7B009307000063880C00930780001C
:105F5000B3879741330BFB0037150000338AA70046
:105F600033048B001305F5FFB377A400330AFA401E
:105F7000337AAA0093050A0013850900EF10000D7B
:105F80009307F0FF631CF5001305040063860C0003
:105F900013858CFF3305A400130A000083270C002F
:105FA0003305654123246901B3874701330A45015D
:105FB000136A1A002320FC0023224B01E3842BDD0B
:105FC0001307F00063625705930710002322FB00BC
:105FD0008327890083A7470093F7C7FF338797403C
:105FE00063E697009307F00063CEE704138509008A
:105FF000EF0000176FF01FA4B3079B41B387E700C2
:106000002320FC006FF0DFF383A74B0013844AFFCB
:10601000137484FF93F71700B3E7870023A2FB00F4
:1060200093065000B3878B0023A2D70023A4D70088
:10603000E37A87D493858B0013850900EFD08FCA4C
:106040006FF05FD40324890093E714002322F40047
:10605000B30794002324F9006FF09FA793F5F50F81
:106060003306C5006316C5001305000067800000F5
:1060700083470500E38CB7FE130515006FF09FFE04
:106080001303F00013070500637EC3029377F70044
:106090006390070A63920508937606FF1376F6006D
:1060A000B386E6002320B7002322B7002324B700DD
:1060B0002326B70013070701E366D7FE6314060023
:1060C00067800000B306C340939626009702000045
:1060D000B38656006780C6002307B700A306B70043
:1060E0002306B700A305B7002305B700A304B70034
:1060F0002304B700A303B7002303B700A302B7002C
:106100002302B700A301B7002301B700A300B70023
:106110002300B7006780000093F5F50F9396850084
:10612000B3E5D50093960501B3E5D5006FF0DFF632
:106130009396270097020000B386560093820000D2
:10614000E78006FA93800200938707FF3307F74042
:106150003306F600E378C3F66FF0DFF367800000E4
:10616000678000008327C504130101FF23229100EB
:1061700023202101232611002324810093040500FC
:10618000138905006382070403A7C4049317290039
:10619000B307F70003A507006310050613041000FA
:1061A000331424011306540013162600930510001F
:1061B00013850400EF4080006302050223222501BD
:1061C000232485006F00C0031306100293054000CE
:1061D000EF30D07E23A6A404E31805FA13050000CF
:1061E0008320C1000324810083244100032901008E
:1061F00013010101678000000327050023A0E700C9
:1062000023280500232605006FF09FFD638005020B
:1062100083A74500139727008327C504B387E700AA
:1062200003A7070023A0E50023A0B70067800000B4
:10623000130101FD232E31019309050037050100EB
:1062400023248102232291021384050083A40501E3
:106250002326110223202103938545011308000002
:106260001305F5FF83A70500938545001308180063
:1062700033F7A7003307C70293D70701B387C702D5
:106280003307D700935607013377A700B387D700AA
:1062900093D6070193970701B387E70023AEF5FE76
:1062A000E34298FC638406068327840063C4F404F5
:1062B00083254400138509002326D100938515000A
:1062C000EFF05FEA032604019305C40013090500FB
:1062D00013062600131626001305C500EF40900E86
:1062E0009305040013850900EFF05FF28326C100D7
:1062F000130409009387440093972700B307F40021
:1063000023A2D700938414002328940013050400CB
:106310008320C10203248102832441020329010254
:106320008329C1011301010367800000130101FDEE
:1063300093878600232C4101138A06009306900060
:106340002324810223229102232E3101138405008C
:10635000B3C7D7022326110223202103232A510188
:1063600093090500930406009306100093050000AE
:1063700063C4F608138509002326E100EFF09FDED1
:106380000327C100930710002328F500232AE50006
:106390009307900063D89706930A940013890A0024
:1063A00033049400130919008346F9FF930505008F
:1063B0001306A000938606FD13850900EFF05FE742
:1063C000E31289FE138484FF33848A001389040056
:1063D000634049058320C1020324810283244102D2
:1063E000032901028329C101032A8101832A410172
:1063F0001301010367800000939616009385150032
:106400006FF01FF71304A400930490006FF01FFCBB
:10641000B3079940B307F40083C60700930505004E
:106420001306A000938606FD13850900EFF05FE0D8
:10643000130919006FF0DFF93707FFFF3377E50025
:1064400093070500130500006316070093970701E3
:1064500013050001370700FF33F7E7006316070055
:106460001305850093978700370700F033F7E7009F
:10647000631607001305450093974700370700C0D0
:1064800033F7E700631607001305250093972700ED
:1064900063CA07001397170013051500634407002C
:1064A00013050002678000008327050013F77700BB
:1064B000630E070293F6170013070000639C0600A3
:1064C00013F72700630C070093D717002320F5006C
:1064D00013071000130507006780000093D72700FB
:1064E0002320F500130720006FF0DFFE93960701CD
:1064F00093D60601130700006396060093D70701A1
:106500001307000193F6F70F639606001307870041
:1065100093D7870093F6F7006396060013074700AA
:1065200093D7470093F637006396060013072700BA
:1065300093D7270093F617006398060093D71700A8
:1065400013071700638607002320F5006FF09FF8FC
:10655000130700026FF01FF8130101FF23248100CD
:10656000138405009305100023261100EFF09FBF50
:10657000232A85008320C100032481001307100013
:106580002328E500130101016780000003A705012E
:1065900083270601130101FD232291022326110204
:1065A0002324810223202103232E3101938405001B
:1065B0006356F700930406001386050083A90401BF
:1065C0000329060183A7840083A54400338429019D
:1065D00063D48700938515002326C100EFF09FB890
:1065E0000326C10013084501131324003303680078
:1065F0009307080063EC670493854401939829008E
:1066000013064601131E2900B7060100B3881501C1
:10661000330EC6019386F6FF6360C605635880009B
:106620001303C3FF83270300638E0710232885000D
:106630008320C10203248102832441020329010231
:106640008329C101130101036780000023A0070013
:10665000938747006FF01FFA832F0600B3FFDF0018
:1066600063840F06130F0800938205009304000053
:1066700003A7020083230F00130F4F00B37ED70040
:10668000B38EFE03B3F7D30093D30301938242008A
:10669000B38EFE0093570701B387F703B38E9E00B6
:1066A00013D70E01B3FEDE00B3877700B387E70090
:1066B00093D4070193970701B3E7D701232EFFFE79
:1066C000E3E812FB23209F00835226006386020624
:1066D00083270800930E0800138F0500930F000016
:1066E00003270F0083D32E00B3F7D7003377D700EB
:1066F00033075702938E4E00130F4F003307770076
:106700003307F701931F0701B3E7FF0023AEFEFE37
:106710008357EFFF83AF0E0013570701B38757026C
:10672000B3FFDF00B387F701B387E70093DF07010B
:10673000E3681FFB23A0FE00130646001308480071
:106740006FF09FED1304F4FF6FF05FED130101FE96
:10675000232A91002328210123263101232E110011
:10676000232C81002324410193773600130905006F
:106770009304060093890500638407029387F7FF5B
:10678000370700811307876593972700B307F70042
:1067900003A6070093060000EFF09FA993090500E8
:1067A00093D424406380040803248904631E0400F6
:1067B0009305102713050900EFF01FDA2324A9041D
:1067C000130405002320050093F7140063840702D7
:1067D000938509001306040013050900EFF01FDB81
:1067E000130A05009385090013050900EFF01FA2A5
:1067F00093090A0093D4144063860402032504001D
:10680000631E050013060400930504001305090028
:10681000EFF0DFD72320A400232005001304050098
:106820006FF09FFA8320C1010324810113850900C1
:1068300083244101032901018329C100032A810026
:106840001301010267800000130101FD2322910260
:1068500093840500232E310183A90401232481029E
:1068600083A545001354564083A78400B30934011F
:1068700023202103232A510123261102232C410125
:10688000930A05001389190063C6270D13850A00B2
:106890002326C100EFF01F8D0326C1009307450199
:1068A000130A05009386070013070000938646002D
:1068B0006348870A635404001304000083A604019C
:1068C000131424003387870093962600938744018E
:1068D0001376F601B386D700630A06081308000290
:1068E0003308C8409305000003A5070013074700BD
:1068F000938747003315C500B365B500232EB7FE57
:1069000083A5C7FFB3D50501E3E0D7FE2320B70079
:1069100063840500138929001309F9FF23282A013C
:1069200013850A0093850400EFF05F8E8320C10277
:106930000324810213050A00832441020329010272
:106940008329C101032A8101832A41011301010323
:106950006780000093851500939717006FF0DFF2B2
:1069600023AE06FE130717006FF05FF4938747000E
:1069700003A6C7FF13074700232EC7FEE3E8D7FE91
:106980006FF09FF98327050103A70501B387E7404F
:10699000639C0702131727001305450193854501E2
:1069A000B306E500B385E5009386C6FF9385C5FF72
:1069B00003A6060003A70500630CE6009307F0FF9B
:1069C0006364E600930710001385070067800000EA
:1069D000E36CD5FC6FF05FFF130101FE232A9100E9
:1069E00093840500232631019305060093090500D1
:1069F00013850400232C8100232E1100232821015C
:106A000013040600EFF01FF8631C05029305000055
:106A100013850900EFF00FF5930710002328F50008
:106A2000232A05008320C10103248101832441011D
:106A3000032901018329C1001301010267800000BD
:106A400013091000634A05009307040013090000AE
:106A500013840400938407008325440013850900F0
:106A6000EFF04FF00323040183A80401130644014F
:106A7000131E23001388440193982800B70E0100C9
:106A800023262501330EC601B308180193064501DC
:106A9000130F0000938EFEFF03270600832F0800CC
:106AA00093864600B375D701B3F7DF01B385E501DF
:106AB000B385F54093DF0F0193570701B387F74183
:106AC00013D70541B387E70013DF0741B3F5D501BD
:106AD00093970701B3E7B7001308480023AEF6FE0B
:106AE00013064600E36A18FBB70501009385F5FF1E
:106AF000636CC6019386C6FF83A706006382070402
:106B0000232865006FF01FF2832706009386460056
:106B10001306460033F7B7003307E7011358074160
:106B200093D70701B387070113DF07413377B70016
:106B300093970701B3E7E70023AEF6FE6FF05FFB24
:106B40001303F3FF6FF01FFBB707F07FB3F5B70038
:106B5000B707C0FCB385F5006358B0009307000089
:106B60001385070067800000B305B04093D7454107
:106B7000130730016348F700B7050800B3D5F540A7
:106B80006FF0DFFD1387C7FE9306E0019305000059
:106B900093071000E3C6E6FCB7070080B3D7E70011
:106BA0006FF01FFC130101FD2322910283240501D4
:106BB000232E31019309450193942400B384990055
:106BC0002324810203A4C4FF232021032326B10030
:106BD0001305040023261102EFF01F868325C10050
:106BE00093070002B387A74023A0F5009307A000F6
:106BF0001389C4FF63CCA7049307B000B387A740F1
:106C00003707F03FB356F400B3E6E6001307000081
:106C100063F4290103A784FF130555013315A4006C
:106C2000B357F700B367F5008320C1020324810244
:106C300083244102032901028329C101138507002E
:106C4000938506001301010367800000930700008D
:106C500063F6290183A784FF138984FF130555FF79
:106C6000630E0502130700023306A74033D7C7009F
:106C70003314A4003364E400B706F03FB366D400D5
:106C80001307000063F429010327C9FFB397A70086
:106C90003357C700B3E7E7006FF01FF9B706F03FBF
:106CA000B366D4006FF05FF8130101FD2324810265
:106CB0001384050093051000232291022320210351
:106CC00093040600232E3101232C410113090700F0
:106CD00023261102138A0600EFF0CFC837071000F1
:106CE0009307F7FFB3F7970093D4440193F4F47F2D
:106CF00093090500639A04082326F100630E040833
:106D00001305810023248100EFF00FFA8326810010
:106D1000630005080327C10093070002B387A7405B
:106D2000B317F700B3E7D7003357A70023AAF9003A
:106D30002326E1000324C10023AC89003334800002
:106D40001304140023A88900638A04069384D4BC26
:106D5000B384A4009307500323209A003385A740EF
:106D60002320A9008320C102032481021385090086
:106D700083244102032901028329C101032A8101DD
:106D80001301010367800000B3E7E7006FF0DFF64F
:106D900023AAD9006FF01FFA1305C100EFF0CFF05E
:106DA0008327C100130505021304100023AAF9006C
:106DB0009307100023A8F9006FF01FF99317240020
:106DC0001305E5BCB387F9002320AA0003A507013A
:106DD00013145400EFF04FE63304A440232089003D
:106DE0006FF05FF8130101FD2322910293840500E7
:106DF00093058101232611022324810223202103EC
:106E000013090500EFF01FDA2320A1002322B100AF
:106E100013840500138504009305C101EFF09FD88A
:106E200003A70401832709018326C1012324A100AC
:106E3000B387E74003278101939757002326B100CA
:106E40003307D740B387E7006350F00493974701B7
:106E5000B38787002322F1008737010007378100BD
:106E60008320C10203248102D3F7E71A832441025D
:106E7000032901022730F100032501008325410089
:106E800013010103678000003707F0FFB387E702B3
:106E9000B387B7002326F1006FF01FFC9307700142
:106EA000130101FF63C6A702B70700811315350060
:106EB000938787653385A700873705012734F1005D
:106EC000032581008325C1001301010167800000B3
:106ED000B717008187B787E7B717008107B707E8BB
:106EE0001305F5FFD3F7E712E31C05FE6FF01FFD56
:106EF0009387F5FF0327060193D757409387170021
:106F0000939727009306460113172700B307F50050
:106F10003387E60063E6E600636EF50067800000F5
:106F20009386460003A6C6FF13054500232EC5FE23
:106F30006FF05FFE13054500232E05FE6FF0DFFDA9
:106F40008326050193D755401307450163C0F60416
:106F500063D4D70293F5F501638005029396270069
:106F6000B306D70003A6060013051000B356B600FB
:106F7000B395B6006318B60293972700B307F700DE
:106F8000636AF7001305000067800000938706001E
:106F90006FF09FFE9387C7FF83A60700E38206FE7C
:106FA0001305100067800000130101FF2326B100C4
:106FB0000327C100B706008093C6F6FF2324A10073
:106FC000B3F7E60023200600B705F07F63D8B706C5
:106FD0000325810033E5A70063020506B375B700FA
:106FE00063940502B717008187B787E807378100E8
:106FF000D377F7122734F1000327C100B3F7E60077
:107000009306A0FC2320D6008326060093D7474191
:10701000938727C0B387F6002320F600B7071080B8
:107020009387F7FF832581003377F700B707E03FA9
:10703000B367F7002324B1002326F1000325810064
:107040008325C1001301010167800000130101FFC6
:10705000232481002322910037240081930405001A
:1070600013850500232611002324049EEF904FBFB3
:107070009307F0FF6318F5008327849E638407005D
:1070800023A0F4008320C100032481008324410055
:107090001301010167800000130101F6232AF108A2
:1070A000B707008093C7F7FF232EF1002328F100D4
:1070B000B707FFFF2326D1082324B100232CB100FA
:1070C000938787209306C10893058100232E11061C
:1070D000232AF1002328E108232C0109232E11097A
:1070E0002322D100EF008023832781002380070023
:1070F0008320C1071301010A67800000130101F614
:10710000232AF108B707008093C7F7FF232EF10069
:107110002328F100B707FFFF93878720232AF10078
:10712000B72700812324A100232CA10003A5879861
:107130002324C1082326D10813860500930681085D
:1071400093058100232E11062328E108232C010931
:10715000232E11092322D100EF00401C8327810038
:10716000238007008320C1071301010A6780000004
:10717000130101FF23248100138405008395E5009A
:1071800023261100EF3050376340050283270405A2
:10719000B387A7002328F4048320C10003248100BF
:1071A00013010101678000008357C40037F7FFFF18
:1071B0001307F7FFB3F7E7002316F4006FF0DFFDC6
:1071C000130500006780000083D7C500130101FE8E
:1071D000232C8100232A9100232821012326310119
:1071E000232E110093F70710930405001384050064
:1071F0001309060093890600638A07008395E5005A
:107200009306200013060000EF30D00E8357C40011
:1072100037F7FFFF1307F7FFB3F7E7002316F40074
:107220008315E400032481018320C10193860900B2
:10723000130609008329C1000329010113850400F5
:1072400083244101130101026F201072130101FF19
:1072500023248100138405008395E5002326110073
:10726000EF3050099307F0FF0357C4006312F50293
:10727000B7F7FFFF9387F7FFB3F7E7002316F40094
:107280008320C100032481001301010167800000F5
:10729000B7170000B367F7002316F4002328A404EF
:1072A0006FF01FFE8395E5006F20107B93070500AC
:1072B00003C705009387170093851500A38FE7FE8A
:1072C000E31807FE67800000930705009387170007
:1072D00003C7F7FFE31C07FE3385A7401305F5FF3F
:1072E0006780000093070500630E06009385150074
:1072F00003C7F5FF938717001306F6FFA38FE7FE7A
:10730000E31407FE3386C7006394C700678000005C
:1073100093871700A38F07FE6FF01FFF130101E291
:10732000232E111C232A911C2328211D2326311DC5
:10733000232C811B9389050093040600138C0600FF
:10734000232C811C2324411D2322511D2320611D38
:10735000232E711B232A911B2328A11B2326B11B3B
:1073600013090500EFE08FCB832705001385070085
:107370002328F102EFF05FF583D7C900232EA10087
:107380002320010E2322010E2324010E2326010EA9
:1073900093F707086380070483A70901639C07022A
:1073A0009305000413050900EFE00FE423A0A900F2
:1073B00023A8A900631C05009307C0002320F9003F
:1073C0009307F0FF2320F1026F00407F9307000432
:1073D00023AAF900B7070081938707782324F104D3
:1073E000B7170081930AC10F9387C78F232A510DC6
:1073F000232E010C232C010C130A0000938B0A008E
:10740000232E0102232C0102232401002326010242
:10741000232A0102232001022328F10013840400FF
:10742000130750028347040063840700639CE70A44
:10743000330B9440630A0B048327C10D23A09B00E8
:1074400023A26B01B3876701232EF10C8327810DE3
:1074500013077000938B8B0093871700232CF10C7C
:10746000635EF7001306410D9385090013050900BB
:10747000EF404010631E0572938B0A0083270102C0
:10748000B38767012320F102834704006394070058
:107490006F10106493071400A30B010A130DF0FF83
:1074A00023220102130400009306A005930CA00000
:1074B000930D900003CB070013871700232CE100E6
:1074C0001306A00293070BFE63F4F6006F10802CE6
:1074D0000327810493972700B387E70083A707005A
:1074E00067800700130414006FF0DFF31305090031
:1074F000EFE0CFB28327450013850700232AF1026E
:10750000EFF09FDC2326A10213050900EFE00FB185
:10751000832785009306A0052324F1008327C10259
:10752000638C0700832781006388070083C70700F7
:107530006384070013640440832781016FF09FF781
:107540008347710BE39A07FE93070002A30BF10A2E
:107550006FF09FFE136414006FF01FFE83270C0072
:10756000130C4C002322F102E3D807FCB307F040D0
:107570002322F102136444006FF01FFC9307B00252
:107580006FF0DFFC0327810183278101034B070094
:10759000938717006310CB04032D0C0013074C00D6
:1075A00063540D00130DF0FF130C0700232CF100A2
:1075B0006FF09FF833039D039387170003CBF7FF0A
:1075C000330DE30013070BFDE3F6EDFE232CF10072
:1075D0006FF05FEF130D00006FF0DFFE136404081F
:1075E0006FF09FF5832781012322010203274102C7
:1075F000130B0BFD93871700330797033307EB003B
:1076000003CBF7FF2322E10213070BFDE3F0EDFEAE
:107610006FF0DFFB136484006FF01FF2832781019A
:1076200003C7070093078006631CF70083278101C7
:107630001364042093871700232CF1006FF0DFEF11
:10764000136404046FF05FEF8327810103C7070011
:107650009307C006631CF7008327810193871700F7
:10766000232CF100136404026FF01FED1364040176
:107670006FF09FEC93074C00232AF10083270C0046
:10768000A30B010A230EF112130C0000130D1000BE
:107690001307000023260100930C0000930D000047
:1076A0009304C1132324E1026354A7012324A103FB
:1076B0008346710B63880600832781029387170036
:1076C0002324F102937724002320F1046388070028
:1076D00083278102938727002324F10293774408AC
:1076E0002322F10463900708832741028326810245
:1076F000B386D7406358D006B7170081130E000138
:107700001388C78E930E70000326810D23A00B01F2
:107710008325C10D1306160013858B006354DE000C
:107720006F10800823A2DB00B386B600232ED10C95
:10773000232CC10C93067000930B050063D4C60282
:107740001306410D93850900130509002326E10462
:10775000EF305062630405006F1090310327C104BD
:10776000938B0A008346710B638E06049306710B9C
:1077700023A0DB009306100023A2DB008326C10DAB
:1077800013067000938B8B0093861600232ED10C6A
:107790008326810D93861600232CD10C6354D602C8
:1077A0001306410D93850900130509002326E10402
:1077B000EF30505C630405006F10902B0327C10469
:1077C000938B0A0083270104638E07049306810BC1
:1077D00023A0DB009306200023A2DB008326C10D3B
:1077E00013067000938B8B0093862600232ED10CFA
:1077F0008326810D93861600232CD10C6354D60268
:107800001306410D93850900130509002320E104A7
:10781000EF305056630405006F10902503270104D4
:10782000938B0A008327410493060008639ED706C2
:107830008327410283268102B386D7406356D00650
:1078400013080001130E7000832701010326810D28
:107850008325C10D23A0FB001306160013858B00A2
:107860006354D8006F00D07923A2DB00B386B60042
:10787000232ED10C232CC10C93067000930B050012
:1078800063D4C6021306410D938509001305090050
:107890002320E104EF30104E630405006F10501DEB
:1078A00003270104938B0A003307A7416350E006C6
:1078B00013080001130E7000832701018326810D38
:1078C0000326C10D23A0FB009386160093858B0031
:1078D000E340E87823A2EB003307C700232EE10C36
:1078E000232CD10C13077000938B05006350D70233
:1078F0001306410D9385090013050900EF309047E9
:10790000630405006F10D016938B0A009376041061
:107910000327C10DE39206788327810D3303ED0021
:1079200023A09B009387170023A2AB01232E610C99
:10793000232CF10C13077000938B8B006344F7002A
:107940006F10000A1306410D938509001305090005
:10795000EF305042630405006F109011938B0A00C2
:107960006F1000081364040193770402638607060E
:10797000130C7C00137C8CFF832C0C00832D4C009B
:1079800093078C00232AF10063C40D006F1050167A
:107990003308904133370001B307B041B38DE7405E
:1079A0001307D002A30BE10A930C08001307100081
:1079B0009306F0FFE308DD449306040033E6BC01C0
:1079C0001374F4F7E3100644E3080D5A930610000D
:1079D000E31ED7426F10101393074C00232AF100C7
:1079E0009377040163880700832C0C0093DDFC412E
:1079F0006FF09FF99377040403280C006388070055
:107A0000931C080193DC0C416FF05FFE9377042018
:107A1000930C0800E38C07FC931C880193DC8C41D9
:107A20006FF0DFFC937784006388070A93074C00AC
:107A3000232AF10083270C0003A6070083A6470032
:107A400003A7870083A7C7002320C10E2322D10EDE
:107A50002324E10E1305010E2326F10EEFD05FD58E
:107A6000232EA10A93072000631EF50A8327010E27
:107A7000930501091305010A2320F10A8327410E0A
:107A800023280108232A01082322F10A8327810ED3
:107A9000232C0108232E01082324F10A8327C10E79
:107AA0002326F10AEF50405B635605009307D0028E
:107AB000A30BF10A9307700463D06707B704008132
:107AC0009384043A1374F4F7130C0000130D300080
:107AD000130700006F005039130C7C00137C8CFFDF
:107AE00083250C0003264C0093078C001305010A24
:107AF000232AF100EF8000728327010A2320F10E70
:107B00008327410A2322F10E8327810A2324F10EC1
:107B10008327C10A6FF01FF4B70400819384C4392E
:107B20006FF05FFA93071000631AF5028327C10E06
:107B300063D607009307D002A30BF10A93077004E2
:107B400063D86701B70400819384843A6FF09FF78C
:107B5000B70400819384443A6FF0DFF6937CFBFD19
:107B600093071004639CFC0893070003230CF10A9D
:107B700013071006930780076304EB009307800543
:107B8000A30CF10A930730061364240063D0A751B5
:107B900093051D0013050900EFD01FE593040500B0
:107BA000631C054E83D7C90093E707042396F900A9
:107BB00083D7C90093F70704E39407808320C11D8E
:107BC0000324811D032501028324411D0329011D76
:107BD0008329C11C032A811C832A411C032B011CFD
:107BE000832BC11B032C811B832C411B032D011BE9
:107BF000832DC11A1301011E678000009307F0FF57
:107C00006300FD4A93077004130C00006398FC00A6
:107C100063160D00130C0D00130D1000032AC10E86
:107C2000936704102324F10223200104032F010E83
:107C3000832E410E032E810E635A0A00B70700807F
:107C400033CA47019307D0022320F104930710049D
:107C50006392FC4A1305010A2320E10B2322D10B76
:107C60002324C10B2326410BEF80407E1306C10B5A
:107C7000EFF08FB313860500930505001305010A85
:107C8000EF8040598327010A130601079305010875
:107C90002320F1088327410A13050109232801063F
:107CA0002322F1088327810A232A0106232C0106B7
:107CB0002324F1088327C10A2326F108B707FC3FD4
:107CC000232EF106EF50004E032801090326410937
:107CD000832681090327C109930501091305010AB8
:107CE0002320010B232801052322C10A2326C104D6
:107CF0002324D10A2322D1042326E10A2326E100EA
:107D000023280108232A0108232C0108232E010817
:107D1000EF50000D0327C100832641040326C10450
:107D2000032801056316050093071000232EF10AAE
:107D300093071006630CFB36B70D008193870D3C4B
:107D40002326F100130EFDFF938D0400B7070340B7
:107D500093050109232AC1081305010A1306010826
:107D6000232CC1052326F10823280109232CD1083F
:107D7000232EE108232001082322010823240108DF
:107D8000EF5040420328010A0326410A8326810A54
:107D90000327C10A1305010A232A01052328C10468
:107DA0002326D1042322E104EF80C00F93050500B0
:107DB000130A05001305010AEF80002D0327410473
:107DC00003260105032841052326E1080327010AAC
:107DD0008326C1042322C1082328E1060327410A80
:107DE0009305010813060107232AE1060327810AE8
:107DF0001305010923200109232CE1060327C10AE9
:107E00002324D108938D1D00232EE106EF608064AA
:107E10008327C100032E810583220109B385470111
:107E200083C50500832F4109032F8109832EC109D2
:107E30002322C105A38FBDFE9307F0FF6300FE0858
:107E4000130EFEFF930501091305010A2326D1072E
:107E50002324E1072322F10723205106232EC10505
:107E60002320510A232C51042322F10B232AF1054C
:107E70002324E10B2328E1052326D10B2326D1055A
:107E800023280108232A0108232C0108232E010896
:107E9000EF4010750327C104832601050326410521
:107EA00003288105032EC10583220106832F410685
:107EB000032F8106832EC106E31A05E83707FE3F2C
:107EC000930501091305010A2320510A232C5104AB
:107ED0002322F10B232AF1052324E10B2328E105BA
:107EE0002326D10B2326D10523280108232A0108A4
:107EF000232C0108232EE108EF5040016348A00421
:107F000083228105832F4105032F0105832EC104A0
:107F10003707FE3F930501091305010A2320510A83
:107F20002322F10B2324E10B2326D10B2328010864
:107F3000232A0108232C0108232EE108EF40506A70
:107F40006310051A137A1A00630C0A188327C100FC
:107F50002326B10D9305000303C6F7008326C10C49
:107F60001387F6FF2326E10C03C7F6FF6306C71449
:107F7000130690036316C7148327C10003C7A70025
:107F8000A38FE6FE138A0D0013077004330A9A408C
:107F9000832DC10B6390EC2C1307D0FF63C4ED005D
:107FA000635ABD33130BEBFF9386FDFF232ED10ADB
:107FB0001376FBFD130510041377FB0F93050000E8
:107FC0006318A6001307F7001377F70F9305100047
:107FD0002302E10C9307B00263D806009306100059
:107FE000B386B6419307D002A302F10C9307900029
:107FF00063D8D72A1307310D130507009305A00096
:1080000013083006B3E7B6021306F7FF938707039A
:10801000A30FF7FEB3C7B6026344D82693870703BE
:10802000A30FF6FE1307E7FF1306610C6360A72694
:108030009307410CB307F640232CF102338D47011F
:108040009307100063C64701937714006386070007
:108050008327C101330DFD001374F4BF936704102F
:108060002324F10223260100930C0000930D00004D
:1080700083270104638607001307D002A30BE10ADC
:1080800003248102130700006FF0CFE1130C0000FE
:108090009304C1136FF09FB8130C05006FF01FB865
:1080A000130C0000130D60006FF05FB7B70D008177
:1080B0009387CD3A6FF0DFC8A38FB6FE6FF01FEA4B
:1080C000130717001377F70F6FF09FEB130A1A00CF
:1080D000A30FDAFE33874741E35A07FE6FF0DFEA6A
:1080E00083274104138A0D0093060003B387FD0024
:1080F0006FF05FFE93076004638EFC0093075004EB
:10810000930D1D006384FC00930D0D0013062000E9
:108110006F00C000930D0D00130630009307010C93
:108120001308C10C1307C10B93860D009305010AB8
:10813000130509002320E10B2326E1052322D10B9F
:108140002322D1052324C10B2326C1012326410B61
:10815000EFC0DFA69307700493040500032EC1004F
:10816000832E4104032FC104639AFC00937714000B
:1081700063960700032AC10C6FF01FE11307600428
:10818000B387B401639AEC0683C6040013070003A7
:108190006390E606930501091305010A2328F104FB
:1081A0002320E10B2326E1052322D10B2322D10535
:1081B0002324C10B2326C1012326410B23280108B8
:1081C000232A0108232C0108232E0108EF405041E7
:1081D000032EC100832E4104032FC1048327010510
:1081E0006308050013071000B30DB741232EB10B30
:1081F0000327C10BB387E700930501091305010AA3
:108200002326F1002320E10B2322D10B2324C10BD1
:108210002326410B23280108232A0108232C0108C7
:10822000232E0108EF40D03B8327C10063140500D3
:108230002326F10C930600036F00000113061700BC
:108240002326C10C2300D7000327C10CE368F7FEE7
:108250006FF05FF213076004E398ECD41377140017
:108260003367A7016350B0076300070C8327C10180
:108270003387FD00330DED00130B60066F0000091E
:1082800013070600938607006FF0DFD71307170068
:108290008347F7FF13061600A30FF6FE6FF01FD9F2
:1082A0001307610C63980500930700032303F10C87
:1082B0001307710C93870603130617002300F700BA
:1082C0006FF01FD7630607068327C10113871700C6
:1082D0006FF05FFA63C04D0313771400138D0D0028
:1082E000630607008327C101338DFD00130B700661
:1082F0006F00C0018327C101130B7006330DFA0014
:108300006346B0013303BD41130D1300937C044059
:1083100023260100E38E0CD4930C0000E35AB0D561
:108320009306F00F6F008003138D0D006FF0DFF4E4
:10833000130B6006130D10006FF05FFD6356B7035B
:1083400083278100B38DED4003C71700630A07023E
:1083500093871700938C1C002324F100832781004E
:1083600003C70700E31CD7FC8327C1003387FC0049
:108370008327C1023307F702330DA7016FF05FCFE8
:108380008327C100938717002326F1006FF01FFD9C
:1083900013074C00232AE1001377040283270C0003
:1083A000630007020327010223A0E7001357F741E8
:1083B00023A2E700032C4101832481016FF00F8683
:1083C00013770401630807000327010223A0E700D5
:1083D0006FF05FFE137704046308070003270102B0
:1083E0002390E7006FF01FFD13740420E30E04FCDC
:1083F000032701022380E7006FF0DFFB1364040111
:108400009377040263860702130C7C00137C8CFFB5
:10841000832C0C00832D4C0093078C00232AF10041
:108420001374F4BF13070000A30B010A6FF04FD8B9
:1084300093074C00232AF100937704016386070019
:10844000832C0C006F0000019377040463880700FD
:10845000835C0C00930D00006FF09FFC9377042069
:10846000E38007FE834C0C006FF0DFFE3787FFFFD1
:108470001347078393074C00231CE10A3707008149
:10848000232AF1009307C73A832C0C00930D0000B8
:1084900013642400232EF10213072000130B80071E
:1084A0006FF09FF893074C00232AF100A30B010AF9
:1084B0009307F0FF83240C006304FD0213060D00F4
:1084C0009305000013850400EFD05FB9130C05007D
:1084D000630005E0330D9540130C00006FF04FDF93
:1084E00013850400EFE05FDE130D05006FF0DFFE83
:1084F000136404019377040263820702130C7C0067
:10850000137C8CFF832C0C00832D4C0093078C0074
:10851000232AF100130710006FF01FF193074C009E
:10852000232AF1009377040163860700832C0C0053
:108530006F0000019377040463880700835C0C00DC
:10854000930D00006FF01FFD93770420E38007FE7A
:10855000834C0C006FF0DFFEB70700819387073C68
:10856000232EF10293770402638A0704130C7C0024
:10857000137C8CFF832C0C00832D4C0093078C0004
:10858000232AF10013771400630E070033E7BC01C0
:10859000630A070013070003230CE10AA30C610B15
:1085A000136424001374F4BF130720006FF0DFE797
:1085B000B70700819387C73A6FF09FFA93074C0083
:1085C000232AF1009377040163860700832C0C00B3
:1085D0006F0000019377040463880700835C0C003C
:1085E000930D00006FF01FFA93770420E38007FEDD
:1085F000834C0C006FF0DFFE93060400130710009D
:108600006FF0CFBB93061000E308D74E930620000F
:108610006308D7121307011A1396DD0193F67C0045
:1086200013D83C0093860603B36C060193DD3D002E
:10863000A30FD7FE33E6BC019304F7FF631E0602C7
:1086400093771400638A0700930700036386F6009C
:10865000A38FF4FE9304E7FF9307011A13070D009D
:10866000130C0000338D974023260100930C00006B
:10867000930D00006FF00F83138704006FF0DFF994
:1086800093770440130A00001307011A2326F10010
:10869000130C90001306A0009306000013850C0035
:1086A00093850D009304F7FF2324E102EF4040324D
:1086B000032781028327C10013050503A30FA7FE2B
:1086C000130A1A00638807048327810003C7070081
:1086D0006312EA049307F00F630EFA0263940D002D
:1086E000637A9C038327C10283254103130A000098
:1086F000B384F4401386070013850400EFE09FBEA7
:108700008327810003C717006306070093871700BC
:108710002324F1001306A0009306000013850C002B
:1087200093850D00EF30906763940D00E3769CF322
:10873000930C0500938D0500138704006FF09FF5DF
:108740009304011A8327C10313F7FC009384F4FFF9
:108750003387E7000347070013D84C002380E40069
:108760001397CD01B36C070193DD4D0033E7BC01D6
:10877000E31A07FC6FF05FEE9304011AE31E07ECA7
:1087800093F61600E38A06EC93070003A30FF11893
:108790006F00D037E30E0B32230E6113A30B010AD7
:1087A000232A81016FE05FEE9385050123A2CB01AF
:1087B000232EB10C232CC10C63DECE021306410D17
:1087C00093850900130509002328E1042326D10419
:1087D000EF20505AE31E0528032701058326C10414
:1087E000B717008113850A00930E70001388C78E97
:1087F000130E0001938606FF930B05006FE0DFF078
:108800009385050123A20B01232EB10C232CC10C4F
:10881000635ACE021306410D938509001305090022
:108820002322E1042320D104EF20D054E3120524B5
:10883000032741048326010413850A00130E7000E8
:1088400013080001938606FF930B05006FE0DFFF1E
:108850001306060123A20B01232EC10C232CD10CDD
:108860006356DE021306410D9385090013050900C6
:108870002320E104EF201050E31C051E0327010410
:1088800093850A00130E700013080001130707FFF9
:10889000938B05006FF04F829306500663D866777E
:1088A0008326010E930501091305010A2320D10A2D
:1088B0008326410E2320E104232801082322D10A24
:1088C0008326810E232A0108232C01082324D10AA0
:1088D0008326C10E232E01082326D10AEF404050E3
:1088E0000327010463120518B70700819387473DEA
:1088F00023A0FB009307100023A2FB008327810D18
:1089000013071700232EE10C93871700232CF10C7B
:1089100013077000938B8B00635EF7001306410D05
:108920009385090013050900EF20D044E3120514D4
:10893000938B0A008327C10B63C64701937714000A
:108940006380070A832701030327C101938B8B00F0
:1089500023ACFBFE8327C10123AEFBFE8327C10DA1
:10896000B387E700232EF10C8327810D13077000D6
:1089700093871700232CF10C635EF7001306410D5B
:108980009385090013050900EF20D03EE312050E80
:10899000938B0A009304FAFF63549004130B0001B5
:1089A000930C7000032601018327810D0327C10D5D
:1089B00023A0CB009387170093868B00634A9B0606
:1089C00023A29B00B384E400232E910C232CF10CF2
:1089D00013077000938B06006354F7006FE09FF657
:1089E00013744400E3160402032B4102832781021F
:1089F0006354FB00138B070083270102B3876701D1
:108A00002320F1028327C10D638C07001306410D5B
:108A10009385090013050900EF20D035E31A0504FA
:108A2000232C010CE31E0C08938B0A006FF09F9817
:108A30001307070123A26B01232EE10C232CF10C59
:108A400063DEFC001306410D938509001305090040
:108A5000EF205032E31E050093860A00938404FF42
:108A6000938B06006FF01FF48326C10B634ED01664
:108A7000B70700819387473D23A0FB0093071000B1
:108A800023A2FB008327810D13071700232EE10C7F
:108A900093871700232CF10C13077000938B8B0026
:108AA000635EF7001306410D938509001305090065
:108AB000EF20502C631E057A938B0A008327C10B8D
:108AC000937614000327C10DB367FA00B3E7D7000C
:108AD000E38807F08327010393888B0023A0FB0022
:108AE0008327C10123A2FB00B387E700232EF10CEB
:108AF0008327810D1307700093871700232CF10C37
:108B0000635EF7001306410D938509001305090004
:108B1000EF205026631E057493880A00032BC10BB7
:108B200063500B06330B604113870800930C000160
:108B3000930D7000032601018327810D8326C10D4B
:108B40002320C700938717009388880063C26C07AF
:108B500023226701330BDB00232E610D232CF10C44
:108B600013077000635EF7001306410D938509003B
:108B700013050900EF201020631C056E93880A007E
:108B80008327C10D23A0980023A24801B387470182
:108B9000232EF10C8327810D13077000938B88001F
:108BA00093871700232CF10CE35CF7E26FE09FD969
:108BB0009386060123229701232ED10C232CF10C3E
:108BC00063DEFD001306410D9385090013050900BE
:108BD000EF20501A631E056893880A00130B0BFFE1
:108BE000138708006FF01FF5138B0D006354BA0153
:108BF000130B0A00635260053307EB00232EE10CD0
:108C00000327810D23A09B0023A26B0113071700EC
:108C1000232CE10C93067000938B8B0063DEE6003F
:108C20001306410D9385090013050900EF209014E8
:108C300063100564938B0A0063540B00130B000050
:108C4000338B6D41635E6005130D000113037000EB
:108C5000832701010327810D8326C10D23A0FB007B
:108C60001307170013868B0063406D1B23A26B0153
:108C7000330BDB00232E610D232CE10C93067000D7
:108C8000930B060063DEE6001306410D9385090091
:108C900013050900EF20100E631C055C938B0A007E
:108CA00093770440338BB40163840702B387440194
:108CB000130D7000938D07008327C10063940C1877
:108CC00063940718B387440163F46701138B0700AB
:108CD0008327C10B63C6470193771400638A070497
:108CE000832701030327C101938B8B0023ACFBFE79
:108CF0008327C10123AEFBFE8327C10DB387E700A5
:108D0000232EF10C8327810D130770009387170022
:108D1000232CF10C635EF7001306410D93850900C7
:108D200013050900EF20100563140554938B0A0006
:108D3000B3844401B38764418324C10BB3049A40D4
:108D400063D4970093840700635490048327C10D74
:108D500023A06B0123A29B00B387F400232EF10C08
:108D60008327810D13077000938B8B009387170067
:108D7000232CF10C635EF7001306410D9385090067
:108D800013050900EF20007F6314054E938B0A0042
:108D90009387040063D40400930700008324C10B6D
:108DA000B3049A40B384F440E35C90C2130B000117
:108DB000930C7000032601018327810D0327C10D49
:108DC00023A0CB009387170093868B0063449B20DE
:108DD00023A29B00B384E400232E910C232CF10CDE
:108DE00013077000938B0600E35CF7BE1306410D7A
:108DF0009385090013050900EF20C077631A054623
:108E0000930BC10F6FF0DFBD9386060123A2AB0168
:108E1000232ED10C232CE10C6350E3021306410DE9
:108E20009385090013050900EF20C07463120544FF
:108E300013860A0013037000130B0BFF930B06003D
:108E40006FF01FE16386070E8327C1009387F7FF4A
:108E50002326F100832741030327C102938B8B0054
:108E600023ACFBFE8327C10223AEFBFE8327C10D8B
:108E7000B387E700232EF10C8327810D938717001A
:108E8000232CF10C635EFD001306410D9385090050
:108E900013050900EF20006E631C053C938B0A004C
:108EA0008327810033876D4183C707006354F70030
:108EB000930707006356F0040327C10D23A06B013D
:108EC00023A2FB003387E700232EE10C0327810D4B
:108ED000938B8B0013071700232CE10C6352ED02D8
:108EE0001306410D93850900130509002320F104A1
:108EF000EF204068631E053683270104930BC10FE2
:108F00001387070063D4070013070000832781003D
:108F10001308000183C70700B387E7406344F006E6
:108F20008327810083C70700330BFB006FF0DFD876
:108F300083278100938CFCFF9387F7FF2324F100A4
:108F40006FF05FF19386060123A20B01232ED10C53
:108F5000232CE10C6354ED021306410D93850900A7
:108F6000130509002320F104EF20C06063120530CF
:108F7000832701041306C10F13080001938707FF1D
:108F8000930B0600832501010327810D8326C10D64
:108F900023A0BB001307170013868B00E344F8FAE5
:108FA00023A2FB00B387D700232EF10C232CE10C66
:108FB000930B0600E356EDF61306410D9385090069
:108FC00013050900EF20005B6314052A930BC10F02
:108FD0006FF01FF51307070123A26B01232EE10C8D
:108FE000232CF10C63DEFC001306410D9385090070
:108FF00013050900EF200058631C05269306C10FD6
:10900000938404FF938B06006FF0DFDA8327810DD2
:109010009306100023A09B001307170093871700E7
:10902000938C8B0063C64601137614006306061CFE
:1090300093061000232EE10C23A2DB00232CF10C5D
:1090400013077000635EF7001306410D9385090056
:1090500013050900EF200052631C0520938C0A00C1
:10906000832701030327C101938C8C0023ACFCFEF2
:109070008327C10123AEFCFE8327C10DB387E70020
:10908000232EF10C8327810D13077000938717009F
:10909000232CF10C635EF7001306410D9385090044
:1090A00013050900EF20004D6314051C938C0A0082
:1090B0008327010E930501091305010A2320F10AF4
:1090C0008327410E130BFAFF232801082322F10AFC
:1090D0008327810E232A0108232C01082324F10A67
:1090E0008327C10E232E01082326F10AEF30504FAB
:1090F000630605088327C10D0327810D938414009F
:109100009387F7FFB38747011307170023A09C003D
:1091100023A26C01232EF10C232CE10C9307700089
:10912000938C8C0063DEE7001306410D93850900E4
:1091300013050900EF200044631C0512938C0A00FC
:109140009307410C23A0FC0083278103032781039D
:10915000938B8C0023A2FC008327C10DB387E7000B
:10916000232EF10C8327810D1307700093871700BE
:10917000232CF10CE356F7866FE0CFFCE35260FD41
:1091800093040001930D7000032601010327810D54
:109190008327C10D23A0CC001307170093868C00F2
:1091A00063C06403B307FB0023A26C01232EF10C00
:1091B000232CE10C93077000938C06006FF09FF650
:1091C0009387070123A29C00232EF10C232CE10C92
:1091D00063DEED001306410D9385090013050900B8
:1091E000EF2040396316050893860A00130B0BFF26
:1091F000938C06006FF05FF9232EE10C23A2DB00B5
:10920000232CF10C13077000E35CF7F26FF0DFF131
:1092100083274102032781023384E740635680FCA1
:10922000B7170081130B00019384C78E930C700055
:109230008327810D23A09B000327C10D938717006F
:1092400063448B0423A28B003304E400232E810C9F
:10925000232CF10C130770006358F7F81306410D27
:109260009385090013050900EF20C030630E05F651
:1092700063140C006FE0DF9393050C0013050900E5
:10928000EFA04FA66FE0DF921307070123A26B0147
:10929000232EE10C232CF10C938B8B0063DEFC005E
:1092A0001306410D9385090013050900EF20802C5A
:1092B000E31005FC938B0A00130404FF6FF05FF7C3
:1092C00093050C0013050900EFA0CFA16FF0CFF5B7
:1092D0008327C10D639407006FE09F8D1306410D36
:1092E0009385090013050900EF20C0286FE05F8C0B
:1092F0001307F0FF6312EDB063940DB813079000ED
:10930000636097B913880C03A30F01199304F11933
:109310006FF08FB483278600130101FD232481029F
:10932000232611022322910223202103232E31011F
:10933000232C4101232A5101232861012326710195
:109340002324810113040600639E070223220600E2
:10935000130500008320C1020324810283244102FB
:10936000032901028329C101032A8101832A4101C2
:10937000032B0101832BC100032C81001301010386
:109380006780000083A7450693890500139727018E
:109390006358070683240600930A0500130BF0FFA9
:1093A00003A9440003AC0400130A0000935B2900E6
:1093B00063467A03832784001379C9FF938484006A
:1093C000B38727412324F400E39C07FC1305000026
:1093D00023240400232204006FF0DFF793172A00F0
:1093E000B307FC0083A507001386090013850A0054
:1093F000EF10400B630A6501130A1A006FF05FFB60
:10940000EF1080176FF0DFFC1305F0FF6FF05FFCCB
:10941000130101ED2324811223202113232E311166
:10942000232A51112326111223229112232C411198
:1094300023286111232671112324811123229111E4
:109440002320A111232EB10F9309050013840500D9
:10945000930A060013890600630805008327850325
:1094600063940700EF901FDC8317C4001397270154
:1094700063420702B726000003274406B3E7D7007C
:109480002316F400B7E7FFFF9387F7FFB377F700E2
:109490002322F4068357C40093F7870063800704F0
:1094A00083270401638C07028357C4001307A000BD
:1094B00093F7A701639EE7068317E40063CA0706D4
:1094C0009306090013860A0093050400138509001A
:1094D000EF00D03D130C05006F00800193050400E0
:1094E00013850900EF905F86E30005FC130CF0FF85
:1094F0008320C1120324811213050C00832441121E
:10950000032901128329C111032A8111832A4111E0
:10951000032B0111832BC110032C8110832C4110CC
:10952000032D0110832DC10F13010113678000006B
:10953000B71700819387C7902324F102B7170081E2
:10954000938787A8232AF100B7170081930BC104E2
:10955000938787A723207105232401042322010474
:10956000938D0B00232601002324010023280100F2
:10957000232E0100130C0000232CF10093840A0019
:109580009306500283C70400638407006392D70ADE
:10959000338A544163060A048327810423A05D01B2
:1095A00023A24D01B38747012324F10483274104FB
:1095B00093067000938D8D00938717002322F1048A
:1095C00063DEF60013060104930504001385090009
:1095D000EFF05FD4E31C0522938D0B00330C4C019C
:1095E00083C70400E388072693861400A30D0102B5
:1095F0009304F0FF130A0000130D0000130BA000EA
:10960000930C900003C60600938A16001305A0056C
:109610001308A002930606FEE36CD50A8327810295
:1096200093962600B386F60083A6060067800600A0
:10963000938414006FF01FF5B70600819387C63A34
:109640002326F10093760D02638C066813097900D6
:10965000137989FF03230900032B4900930C890028
:1096600093761D00638E0600B3666301638A06006D
:1096700093060003230ED102A30EC102136D2D0029
:10968000137DFDBF6F00C02F13850900EFC00F9938
:109690008327450013850700232EF100EFD0DFC29A
:1096A0002328A10013850900EFC04F978327850069
:1096B0002324F10083270101638C070083278100A5
:1096C0006388070083C6070063840600136D0D409E
:1096D00093860A006FF01FF38346B103E39A06FEF8
:1096E00093060002A30DD1026FF09FFE136D1D00C3
:1096F0006FF01FFE032A090013094900E35A0AFC10
:10970000330A4041136D4D006FF09FFC9306B00289
:109710006FF05FFD03C60A0093861A00631006050A
:10972000832409001306490063D404009304F0FF66
:1097300013090600938A06006FF09FF9B38464034F
:109740009386160003C6F6FFB384B400930506FDA6
:10975000E3F6BCFE938A06006FF0DFEB9304000093
:109760006FF0DFFE136D0D086FF09FF693860A0011
:10977000130A0000330A6A03130606FD93861600D7
:10978000330A460103C6F6FF930506FDE3F4BCFE6B
:109790006FF05FFC03C60A00930680066318D600CC
:1097A000938A1A00136D0D206FF09FF2136D0D0454
:1097B0006FF01FF203C60A009306C0066318D600B6
:1097C000938A1A00136D0D026FF09FF0136D0D0157
:1097D0006FF01FF083260900930C4900A30D0102CE
:1097E0002306D10893041000130B00001309C108CD
:1097F0006F00801C136D0D0193760D0263800606C9
:1098000013097900137989FF03230900032B490009
:10981000930C8900E35E0B0433036040B3366000B1
:1098200033086041330BD8409306D002A30DD10218
:10983000930610001306F0FF6386C44E13060D0056
:10984000B3656301137DFDF7639E054C6384046675
:1098500013061000639CC64C6F00D00293760D0176
:10986000930C49006388060003230900135BF3414E
:109870006FF05FFA93760D040323090063880600F6
:1098800013130301135303416FF05FFE93760D2012
:10989000E38E06FC13138301135383416FF01FFD06
:1098A00013760D028326090013094900630A060096
:1098B0009357FC4123A0860123A2F6006FF01FCC32
:1098C00013760D016306060023A086016FF01FCBFF
:1098D00013760D0463060600239086016FF01FCAFD
:1098E00093770D20E38207FE238086016FF01FC966
:1098F000136D0D0193760D0263840602130979003E
:10990000137989FF03230900032B4900930C890075
:10991000137DFDBF93060000A30D01026FF09FF1C0
:1099200093760D01930C490063860600032309001A
:109930006F00000193760D0463880600035309004D
:10994000130B00006FF0DFFC93760D20E38006FE22
:10995000034309006FF0DFFEB786FFFF93C606835F
:10996000231ED10203230900B70600819387C63A5C
:10997000930C4900130B0000136D2D002326F100FA
:10998000930620006FF05FF9A30D01029306F0FF2C
:10999000930C4900032909006384D42C1386040026
:1099A0009305000013050900EFC04FEB130B0000F7
:1099B00063040500B30425412322610163549B0025
:1099C000232291008346B103638806008327410068
:1099D000938717002322F10093772D002320F102B3
:1099E0006388070083274100938727002322F10023
:1099F00093774D082322F1026394070683274100E1
:109A0000B306FA40635ED0041308000193087000A7
:109A100083278101032641048325810423A0FD00BF
:109A20001306160013858D00634ED84A23A2DD006D
:109A3000B386B6002324D1042322C1049306700008
:109A4000930D050063DEC6001306010493050400B0
:109A500013850900EFF01F8C631A055A938D0B00D4
:109A60008346B103638806041306B10323A0CD0027
:109A7000130610008326410423A2CD00032681048F
:109A8000938616002322D104130616002324C10452
:109A900013067000938D8D00635ED60013060104DB
:109AA0009305040013850900EFF0DF866310055667
:109AB000938D0B0083270102638807041306C103FB
:109AC00023A0CD00130620008326410423A2CD004D
:109AD00003268104938616002322D1041306260050
:109AE0002324C10413067000938D8D00635ED6009D
:109AF000130601049305040013850900EFF09F810C
:109B000063160550938D0B008327410293060008CE
:109B10006394D70683274100B306FA40635ED004FE
:109B200013080001930870008327410103264104B4
:109B30008325810423A0FD001306160013858D00E4
:109B40006346D83E23A2DD00B386B6002324D104A9
:109B50002322C10493067000930D050063DEC60046
:109B6000130601049305040013850900EFF08FFA32
:109B7000631E0548938D0B00330B9B40635E6005AD
:109B800013080001930870008327410183264104D4
:109B90000326810423A0FD009386160093858D0083
:109BA000634A683D23A26D01330BCB00232461057A
:109BB0002322D10413067000938D0500635ED60046
:109BC000130601049305040013850900EFF08FF4D8
:109BD000631E0542938D0B008326810423A29D0002
:109BE00023A02D01B38496008326410423249104ED
:109BF00013067000938616002322D10413878D006C
:109C0000635ED60013060104930504001385090062
:109C1000EFF04FF0631C053E13870B0093774D0068
:109C2000639A0738832741006354FA00138A0700B8
:109C300083278104330C4C01638C07001306010455
:109C40009305040013850900EFF0CFEC6310053C89
:109C50002322010413890C00938D0B006FF01F92D7
:109C600013050900EFD04FE693040500130B000025
:109C70006FF09FD4136D0D0193760D026380060281
:109C800013097900137989FF03230900032B490085
:109C9000930C8900930610006FF01FC893760D0196
:109CA000930C490063860600032309006F0000013E
:109CB00093760D046388060003530900130B00001C
:109CC0006FF05FFD93760D20E38006FE03430900ED
:109CD0006FF0DFFEB70600819387063C6FF05F965A
:109CE00093760D01930C4900638606000323090057
:109CF0006F00000193760D0463880600035309008A
:109D0000130B00006FF0DF9593760D20E38006FEC5
:109D1000034309006FF0DFFE13060D0093061000E9
:109D20006FF01FB2130610006388C63413062000BC
:109D30006386C6149306010F9315DB011376730037
:109D4000135333001306060333E36500135B3B0034
:109D5000A38FC6FEB36563011389F6FF6396050200
:109D600093751D00638A0500930500036306B60022
:109D7000A30FB9FE1389E6FF9307010F138B0400AD
:109D8000B38427416FF05FC3930609006FF0DFFAD9
:109D900093770D4093080000130E010F2322F1006A
:109DA000130503001306A0009306000093050B00A3
:109DB000232611031309FEFF2322C103232061027E
:109DC000EF201041032E41028328C1028327410066
:109DD00013050503A30FAEFE9388180003230102A9
:109DE000638E07048327810083C6070063981605E6
:109DF0009307F00F6384F80463160B009307900039
:109E000063FE6702832701018325C10123206102CC
:109E10003309F9401386070013050900EFD08FCCF2
:109E200083278100930800000323010283C61700E3
:109E300063860600938717002324F10013050300AF
:109E40001306A0009306000093050B0023221103C4
:109E500023206102EF208074032301028328410242
:109E600063160B0093079000E3F867F013030500F7
:109E7000138B0500130E09006FF09FF21309010FF9
:109E80008327C1009376F3001309F9FFB386D70047
:109E900083C60600135343002300D9009316CB0159
:109EA00033E36600135B4B00B3666301E39A06FC81
:109EB0006FF09FEC1309010FE39006EC1376160088
:109EC000E30C06EA93060003A307D10E6F00001C03
:109ED000630206182306C108A30D0102930C0900B2
:109EE0006FF05F909385050123A20D012324B10437
:109EF0002322C10463D6C80213060104930504009B
:109F0000138509002326D102EFF0CFC0631005109E
:109F10008326C10213850B0093087000130800010B
:109F2000938606FF930D05006FF09FAE93850501A4
:109F300023A20D012324B1042322C10463D6C80245
:109F40001306010493050400138509002320D102A0
:109F5000EFF04FBC631C050A8326010213850B003A
:109F60009308700013080001938606FF930D050007
:109F70006FF09FBB1306060123A20D012324C10429
:109F80002322D10463D2D8021306010493050400EE
:109F900013850900EFF00FB8631A050693850B00CF
:109FA0009308700013080001130B0BFF938D05003D
:109FB0006FF09FBD83274100B304FA40E35490C67D
:109FC00013090001130B700003268101832741044C
:109FD000832681042320C7009387170063409904D8
:109FE00023229700B384D400232491042322F10474
:109FF00013077000E358F7C2130601049305040029
:10A0000013850900EFF00FB1E30E05C08357C400BC
:10A0100093F70704638E07CC6FF04FCD938606014C
:10A02000232227012324D1042322F10413078700CC
:10A03000635EFB0013060104930504001385090009
:10A04000EFF04FADE31405FC13870B00938404FF7E
:10A050006FF09FF783278104E38A07FA1306010450
:10A060009305040013850900EFF0CFAA6FF01FFAE3
:10A070009306F0FFE392D4CAE31C0BD09306900042
:10A08000E3E866D013030303A307610E1309F10E7F
:10A090006FF09FCEB7270081930606001386050058
:10A0A0009305050003A587986FF08FB683D7C50089
:10A0B000130101B8232C814693F7D7FF231AF1002F
:10A0C00083A7450613840500232A91462326F1061B
:10A0D00083D7E50023282147232E1146231BF100B7
:10A0E00083A7C50113090500232001022322F102E1
:10A0F00083A74502930581002326F10293070107F8
:10A100002324F100232CF100930700402328F100C1
:10A11000232EF100EFF0CFAF93040500634C050050
:10A120009305810013050900EF801FF66304050005
:10A130009304F0FF8357410193F7070463880700F6
:10A140008357C40093E707042316F4008320C14714
:10A1500003248147138504000329014783244147D1
:10A160001301014867800000130101FF23248100CF
:10A1700023229100372400819304050013850500F4
:10A180009305060013860600232611002324049E4F
:10A19000EF60CFA39307F0FF6318F5008327849E39
:10A1A0006384070023A0F4008320C10003248100FE
:10A1B000832441001301010167800000B385C502BB
:10A1C000130101FF2324810023261100EFB0DF815A
:10A1D00013040500630205040326C5FF13074002AC
:10A1E0001376C6FF1306C6FF6362C70693063001E7
:10A1F0009307050063FCC600232005002322050009
:10A200009307B00163E4C7029307850023A007000A
:10A2100023A2070023A40700130504008320C10024
:10A22000032481001301010167800000232405003D
:10A230002326050093070501E31AE6FC2328050001
:10A2400093078501232A05006FF05FFC930500004A
:10A25000EFB01FE36FF05FFC130101FF23248100C7
:10A260002322910037240081930405001385050003
:10A27000232611002324049EEF50DFF19307F0FF03
:10A280006318F5008327849E6384070023A0F400ED
:10A290008320C100032481008324410013010101B4
:10A2A00067800000130101FF232611002324810091
:10A2B000232291002320210163920502130900004B
:10A2C0008320C10003248100130509008324410079
:10A2D00003290100130101016780000093040500B8
:10A2E0001384050063080500832785036394070032
:10A2F000EF805FF38317C400E38207FC930504003B
:10A3000013850400EF80DFB78327C402130905001B
:10A31000638C07008325C40113850400E7800700D0
:10A32000635405001309F0FF8357C40093F707082F
:10A33000638807008325040113850400EF908F9A3A
:10A3400083250403638C0500930704046386F500EA
:10A3500013850400EF900F992328040283254404F9
:10A360006388050013850400EF90CF97232204042F
:10A37000EF904F8223160400EF900F826FF05FF48E
:10A38000B72700819305050003A587986FF09FF11B
:10A39000130101FD2324810223229102232C410178
:10A3A0002326110223202103232E3101232A5101C8
:10A3B00023286101130A0500938405001304060095
:10A3C000EF00806D93071000631AF5049387F4FF84
:10A3D0001307E00F6364F70423069100930910004C
:10A3E00013090000930AF0FF130BA0006312390752
:10A3F000138504008320C1020324810283244102C7
:10A40000032901028329C101032A8101832A410111
:10A41000032B010113010103678000009306C405AB
:10A42000138604009305C10013050A00EF20C0073E
:10A430009307F0FF93090500E314F5FA8357C4006E
:10A4400093E707042316F4001305F0FF6FF09FFA5B
:10A450009307C100B387270183C5070083278400C2
:10A460009387F7FF2324F40063D8070003278401B0
:10A4700063C0E702638E650183270400138717001A
:10A480002320E4002380B700130919006FF01FF6A2
:10A490001306040013050A00EF10D06CE31655FFF5
:10A4A0006FF09FFA8317C6001397270163400702D6
:10A4B00003274606B7260000B3E7D7002316F600A9
:10A4C000B7270000B367F7002322F6066FF05FECB2
:10A4D000130101FEB7270081232C810003A4879874
:10A4E000232A9100232E11009304050013860500F2
:10A4F000630E040083278403639A07001305040096
:10A500002326B100EF801FD20326C10013050400EB
:10A51000032481018320C101938504008324410128
:10A52000130101026FF01FF8130101FF23248100C2
:10A530002322910037240081930405001385050030
:10A5400093050600232611002324049EEF509FC785
:10A550009307F0FF6318F5008327849E6384070048
:10A5600023A0F4008320C100032481008324410040
:10A5700013010101678000008327860063980700AC
:10A5800093070000138507006780000083D7C5008C
:10A59000130101FB2324810423202105232A5103D5
:10A5A0002326110423229104232E3103232C41035B
:10A5B000232861032326710323248103232291038B
:10A5C0002320A103232EB10193F78700930A0600ED
:10A5D00013840500130905006382070E83A7050194
:10A5E000638E070C8357C40003AA0A0013F72700E1
:10A5F000631A071693F7170063840720930B000074
:10A6000013050000130B0000930900006384093652
:10A6100063120502138609009305A00013050B00C1
:10A62000EFB0DFA3938B1900630605001305150037
:10A63000B30B6541138C0B0063F47901138C090093
:10A6400003250400832704018326440163FEA73207
:10A6500083248400B384960063D8843393050B006D
:10A6600013860400EF008063832704009305040031
:10A6700013050900B38797002320F400EF80DFA0C3
:10A6800063160516B38B9B4013051000639A0B00ED
:10A690009305040013050900EF801F9F631805143C
:10A6A00083A78A00330B9B00B3899940B3849740FA
:10A6B00023A49A00E39C04F46F0080069305040031
:10A6C00013050900EF804FE89307F0FFE30C05F056
:10A6D0006F00400583290A0083244A00130A8A0078
:10A6E000E38A04FE9386040063749B0093060B00C8
:10A6F000832744028325C40113860900130509003A
:10A70000E78007006354A00E83A78A00B389A900DD
:10A71000B384A4403385A74023A4AA00E31205FC18
:10A72000930700008320C10403248104832441048F
:10A73000032901048329C103032A8103832A4103D6
:10A74000032B0103832BC102032C8102832C4102C2
:10A75000032D0102832DC10113850700130101059B
:10A7600067800000370B008093090000930400000D
:10A77000134B0BC06FF0DFF6032B0A0083244A0053
:10A78000130A8A00E38A04FE0357C4008327840067
:10A7900003250400937607206388061463E2F40C13
:10A7A00093760748638E060A832D440183250401AE
:10A7B000B38DBC03B309B54093871900B3879700E5
:10A7C000B3CDAD0363F4FD00938D0700137707400D
:10A7D0006304070E93850D0013050900EFB0CFA0A9
:10A7E000631005049307C0002320F9008357C400B9
:10A7F00093E707042316F4009307F0FF6FF09FF22E
:10A80000B70B008013CCEBFF130B00009304000088
:10A8100093CBFBFF930C3000130D20006FF09FF6DD
:10A8200083250401138609002326A100EF00803947
:10A830000357C4008327C1001377F7B713670708CE
:10A840002316E4002328F400232AB401B387370138
:10A85000B38D3D412320F4002324B40193870400E9
:10A860009389040063F4F400938704000325040033
:10A870001386070093050B002326F100EF0000422A
:10A88000032784008327C1003307F7402324E40013
:10A8900003270400B307F7002320F40083A78A00EE
:10A8A000330B3B01B3843441B389374123A43A01CC
:10A8B000E39A09EC6FF0DFE613860D00130509003B
:10A8C000EF00C04893070500E31E05F68325040149
:10A8D00013050900EF801FC18357C40093F7F7F7F2
:10A8E0002316F4006FF01FF0032704016366A7002E
:10A8F0008326440163F6D4049389070063F4F400CB
:10A90000938904001386090093050B00EF000039BA
:10A910008327840003270400B387374133073701B7
:10A920002324F4002320E400E39A07F693050400AF
:10A9300013050900EF804FF5E30205F66FF01FEBFA
:10A940009387040063749C0093870B00B3C7D702FE
:10A95000032744028325C40113060B0013050900D5
:10A96000B386D702E700070093090500E348A0F289
:10A970006FF0DFE7032B0A0083294A00130500006C
:10A98000130A8A006FF09FC86342DC0283274402E7
:10A990008325C40113060B0013050900E780070097
:10A9A00093040500E340A0CE6FF05FE413060C00B3
:10A9B00093050B00EF00802E8327840093040C0086
:10A9C000B38787412324F40083270400B3878701DA
:10A9D0002320F4006FF01FCB130101FF232481001B
:10A9E000232291003724008193040500138505007C
:10A9F000232611002324049EEF50DF939307F0FFDA
:10AA00006318F5008327849E6384070023A0F40065
:10AA10008320C1000324810083244100130101012C
:10AA200067800000130101FF2322910023261100FB
:10AA300023248100B7140081631E0600138584A9B6
:10AA40008320C100032481008324410013010101FC
:10AA500067800000B71500819385C5A9130506001E
:10AA600013040600EF005019E30A05FC938584A93E
:10AA700013050400EF005018E30205FCB705008140
:10AA80009385053D13050400EF001017E30805FA50
:10AA9000130500006FF0DFFAB727008183A78798BE
:10AAA00083A7470363960700B72700819387078131
:10AAB00003C58712678000000325C50E678000006C
:10AAC000B727008183A7879883A74703639607006A
:10AAD000B72700819387078103A5C70E6780000011
:10AAE000B7270081138605009305050003A5879805
:10AAF0006FF05FF3130101FF2324810023229100F3
:10AB00003724008193040500138505009305060092
:10AB100013860600232611002324049EEF501F8570
:10AB20009307F0FF6318F5008327849E6384070072
:10AB300023A0F4008320C10003248100832441006A
:10AB40001301010167800000B727008183A7879860
:10AB500083A7470363960700B72700819387078180
:10AB600003A3470E67000300639A0502130101FF68
:10AB70009305C10013050000630E06001305E0FFF6
:10AB8000638A06008347060023A0F50003450600FC
:10AB90003335A00013010101678000001305000098
:10ABA000630006021305E0FF638C0600834706007E
:10ABB00023A0F500034506003335A00067800000A0
:10ABC00067800000B3C7A50093F737003307C500BF
:10ABD000639607009307300063E2C70293070500FE
:10ABE000637CE50A83C605009387170093851500EB
:10ABF000A38FD7FEE3E8E7FE678000009376350079
:10AC000093070500638E060083C60500938717002F
:10AC100093851500A38FD7FE93F637006FF09FFE44
:10AC20009376C7FF138606FE63F4C70683A3050069
:10AC300083A2450083AF850003AFC50083AE050145
:10AC400003AE450103A3850183A8C5019385450291
:10AC500023A0770003A8C5FF23A2570023A4F70170
:10AC600023A6E70123A8D70123AAC70123AC6700C5
:10AC700023AE17019387470223AE07FF6FF0DFFA79
:10AC800003A60500938747009385450023AEC7FEC2
:10AC9000E3E8D7FEE3E8E7F46780000063FAA50481
:10ACA000B386C5006376D5049345F6FF930700008D
:10ACB0009387F7FF6394F500678000003387F60001
:10ACC000034807003387C7003307E5002300070167
:10ACD0006FF01FFE3387F500834607003307F5004A
:10ACE000938717002300D700E316F6FE6780000065
:10ACF000930700006FF05FFF130101FF2324810021
:10AD00002322910037240081930405001385050058
:10AD10009305060013860600232611002324049EB3
:10AD2000EF50CFE79307F0FF6318F5008327849E69
:10AD30006384070023A0F4008320C1000324810062
:10AD4000832441001301010167800000130101FC0D
:10AD5000232C8102232E110213840500232A910241
:10AD600023282103232631032324410323225103D3
:10AD700023206103232E7101232C810193050600FA
:10AD8000631A0402032481038320C1038324410343
:10AD9000032901038329C102032A8102832A410274
:10ADA000032B0102832BC101032C81011301010438
:10ADB0006FA09FC3930A05002326C100EFB00FBA0E
:10ADC0008325C100930760019389B50063F63705B9
:10ADD00013FB89FF63540B049307C00023A0FA0000
:10ADE000130A00008320C1030324810313050A0012
:10ADF00083244103032901038329C102032A810219
:10AE0000832A4102032B0102832BC101032C810100
:10AE10001301010467800000130B0001E36EBBFA0D
:10AE20008326C4FF930B84FF13F9C6FF635C694557
:10AE3000371C008113078C4003268700B3872B0142
:10AE400003A74700130C8C40630CF6001375E7FF53
:10AE50003385A70003254500137515006314050607
:10AE60001377C7FFB309E9006310F60413050B015C
:10AE700063CEA904B38B6B01B389694123247C01A0
:10AE800093E9190023A23B018329C4FF13850A001B
:10AE9000130A040093F91900B3E96901232E34FF62
:10AEA000EFB00FAC6FF01FF463C2690303A7C700D4
:10AEB00083A7870023A6E7002324F70093840B00D1
:10AEC0006F000019130700009307000093F61600A7
:10AED0006398062C832484FFB3849B4003AA440018
:10AEE000137ACAFF330A2A0163820720B309470194
:10AEF0006316F60E93070B0163CAF91E03A78400BD
:10AF000083A7C4001306C9FF138A84002326F70011
:10AF100023A4E70013074002636AC70A93063001BF
:10AF200093070A0063F2C6028327040023A4F400F7
:10AF30008327440023A6F4009307B00163EAC70403
:10AF400013048400938704010327040023A0E7006F
:10AF50000327440023A2E7000327840023A4E7007B
:10AF6000B3876401B38969412324FC0093E9190084
:10AF700023A2370183A7440093F71700B3E96701C1
:10AF800023A2340113850A00EFB08F9D6FF09FE577
:10AF90008327840023A8F4008327C40023AAF40095
:10AFA0006308E60013040401938784016FF0DFF95E
:10AFB000832704011304840123ACF4000327C4FF96
:10AFC0009387040223AEE4006FF01FF8930504009A
:10AFD00013050A00EFF09FCC6FF09FF863C869116A
:10AFE00003A7C70083A787001306C9FF1385840042
:10AFF00023A6E7002324F70003A7840083A7C40047
:10B000002326F70023A4E7009307400263EAC70C56
:10B01000130730016372C7020327040023A4E4006E
:10B020000327440023A6E4001307B001636CC7069E
:10B030001304840013850401832704002320F500F2
:10B04000832744002322F500832784002324F5006E
:10B0500003A74400B38669411306F0001377170075
:10B06000B38734016374D622B369EB0023A23401A1
:10B07000B385640193E6160023A2D50003A7470019
:10B080009385850013850A001367170023A2E70044
:10B09000EF804FC513850A00EFB08F8C138A8400B0
:10B0A0006FF05FD40327840023A8E4000327C400C3
:10B0B00023AAE4006308F600130404011385840145
:10B0C0006FF09FF7832704011385040213048401A2
:10B0D00023ACF4008327C4FF23AEF4006FF0DFF548
:10B0E00093050400EFF09FBB6FF09FF6634A6A0B75
:10B0F00083A7C40003A784001306C9FF1385840037
:10B100002326F70023A4E7009307400263E4C7085F
:10B11000130730016372C7020327040023A4E4006D
:10B120000327440023A6E4001307B0016366C702A7
:10B130001304840013850401832704002320F500F1
:10B14000832744002322F500832784002324F5006D
:10B1500093090A006FF0DFEF0327840023A8E400BF
:10B160000327C40023AAE4006308F60013040401C3
:10B17000138584016FF05FFC8327040113850402AB
:10B180001304840123ACF4008327C4FF23AEF4002E
:10B190006FF09FFA93050400EFF05FB06FF05FFB74
:10B1A00013850A00EFA05F84130A0500E30C05DC99
:10B1B0008327C4FF130785FF93F7E7FFB387FB00DF
:10B1C000639AE7008329C5FF93F9C9FFB389290171
:10B1D0006FF0DFCE1306C9FF9307400263EEC70886
:10B1E000130730016374C708032704002320E50018
:10B1F000032744002322E5001307B001636AC70256
:10B2000013078400930785008326070023A0D70037
:10B210008326470023A2D7000327870023A4E70043
:10B220009305040013850A00EF80CFAB6FF09FD524
:10B23000032784002324E5000327C4002326E50018
:10B240006308F60013070401930705016FF0DFFBA5
:10B2500083270401130784012328F5008326440172
:10B2600093078501232AD5006FF01FFA9307050085
:10B27000130704006FF05FF993050400EFF01FA2BD
:10B280006FF01FFA930909006FF05FC3B3E9E9009B
:10B2900023A2340103A747001367170023A2E70086
:10B2A0006FF05FDF130101FF232481001384050089
:10B2B00083A5050023229100232611009304050095
:10B2C00063840500EFF01FFE930504000324810052
:10B2D0008320C10013850400832441001301010170
:10B2E0006F804FA0B727008183A787986384A7103A
:10B2F0008327C504130101FE232C8100232A91001A
:10B3000023282101232E11002326310113040500D7
:10B310009304000013090008639A070683250404B8
:10B320006386050013050400EF80CF9B83258414FA
:10B330009304C414639005088325440563980508A5
:10B3400083278403638A07088327C4031305040043
:10B35000E78007008325042E638005081305040099
:10B36000032481018320C1018324410103290101B8
:10B370008329C100130101026FF0DFF2B38595004C
:10B3800083A50500639E0500938444008325C404BF
:10B39000E39624FF13050400EF80CF946FF01FF8AD
:10B3A00083A9050013050400EF80CF93938509005E
:10B3B0006FF05FFDE38295F803A905001305040013
:10B3C000EF804F92930509006FF0DFFE1305040034
:10B3D000EF804F916FF0DFF68320C10103248101DC
:10B3E00083244101032901018329C10013010102C2
:10B3F00067800000678000003367B5009303F0FFAB
:10B400001377370063100710B7877F7F9387F7F7AD
:10B410000326050083A60500B372F6003363F60029
:10B42000B382F200B3E26200639272106316D60830
:10B430000326450083A64500B372F6003363F60089
:10B44000B382F200B3E26200639E720C6316D6060A
:10B450000326850083A68500B372F6003363F600E9
:10B46000B382F200B3E262006398720C6316D604F2
:10B470000326C50083A6C500B372F6003363F60049
:10B48000B382F200B3E262006392720C6316D602DA
:10B490000326050183A60501B372F6003363F600A7
:10B4A000B382F200B3E26200639C720A13054501A5
:10B4B00093854501E30ED6F4131706019397060111
:10B4C000631EF7001357060193D706013305F740B3
:10B4D0009375F50F6390050267800000135707010D
:10B4E00093D707013305F7409375F50F6394050073
:10B4F000678000001377F70F93F7F70F3305F740D6
:10B50000678000000346050083C60500130515008B
:10B51000938515006314D600E31606FE3305D64066
:10B52000678000001305450093854500E31CD6FCA9
:10B5300013050000678000001305850093858500D2
:10B54000E312D6FC13050000678000001305C50058
:10B550009385C500E318D6FA130500006780000044
:10B560001305050193850501E31ED6F813050000B8
:10B570006780000083278600130101FD232E31011F
:10B580002326110223248102232291022320210356
:10B59000232C4101232A5101232861012326710113
:10B5A00023248101232291012320A1019309060074
:10B5B00063840712832A0600130A0500138405001A
:10B5C000130B000013090000930B3000130C200034
:10B5D00063000908032D84006360A90D8357C4002C
:10B5E00013F70748630A070A83240400832504012C
:10B5F000B38CB4408324440113871C003307270114
:10B60000B3849B02B3C4840363F4E400930407008F
:10B6100093F70740638207109385040013050A001F
:10B62000EFA08FBC130D0500631C05029307C0003B
:10B630002320FA008357C4001305F0FF93E70704A3
:10B640002316F40023A4090023A209006F00400977
:10B6500003AB0A0003A94A00938A8A006FF05FF7E0
:10B660008325040113860C00EFF0CFD58357C40067
:10B6700093F7F7B793E707082316F4002328A401EC
:10B68000232A9400330D9D01B38494412320A40107
:10B6900023249400130D09006374A901130D0900FC
:10B6A0000325040013060D0093050B00EFF00FDFD8
:10B6B00083278400B387A7412324F4008327040051
:10B6C000338DA70183A789002320A4013389274153
:10B6D00023A42901E31E09F623A209001305000093
:10B6E0008320C10203248102832441020329010231
:10B6F0008329C101032A8101832A4101032B01010E
:10B70000832BC100032C8100832C4100032D0100F9
:10B7100013010103678000001386040013050A006B
:10B72000EFF0CFE2130D0500E31A05F483250401C1
:10B7300013050A00EF701FDB6FF05FEF83D7C500C2
:10B74000130101ED2322911223202113232C4111F7
:10B75000232861112326111223248112232E311153
:10B76000232A51112326711123248111232291119F
:10B770002320A111232EB10F93F70708130A050008
:10B7800013890500130B060093840600638C0702DF
:10B7900083A705016398070293050004EFA0CFA4D7
:10B7A0002320A9002328A900631A05009307C000DD
:10B7B0002320FA00130CF0FF6F00502F93070004B2
:10B7C000232AF900B7170081938787AA2324F1025F
:10B7D000B7170081938747C2232AF100B71700816A
:10B7E000930BC104938747C12320710523240104CF
:10B7F00023220104938D0B00232801002324010040
:10B8000023260100232E0100130C0000232CF1003D
:10B8100013040B009306500283470400638407005F
:10B820006392D70AB30964416386090483278104BC
:10B8300023A06D0123A23D01B38737012324F10426
:10B840008327410493067000938D8D009387170022
:10B850002322F10463DEF6001306010493050900B8
:10B8600013050A00EFF01FD1E31C0522938D0B0096
:10B87000330C3C0183470400E386072A9306140037
:10B88000A30D01021304F0FF93090000130D000043
:10B89000930AA000930C900003C60600138B1600B9
:10B8A0001305A0051308A002930606FEE36CD50A53
:10B8B0008327810293962600B386F60083A60600AE
:10B8C00067800600130414006FF01FF5B7060081AF
:10B8D0009387C63A2328F10093760D02638C06689D
:10B8E0009384740093F484FF03A3040083AA4400A8
:10B8F000938C840093761D00638E0600B36653011B
:10B90000638A060093060003230ED102A30EC10230
:10B91000136D2D00137DFDBF6F00C02F13050A00AE
:10B92000EF90DFEF8327450013850700232EF100FA
:10B93000EFB09F992326A10013050A00EF901FEE98
:10B94000832785002324F1008327C100638C07002F
:10B95000832781006388070083C60700638406008D
:10B96000136D0D4093060B006FF01FF38346B10378
:10B97000E39A06FE93060002A30DD1026FF09FFE2C
:10B98000136D1D006FF01FFE83A904009384440013
:10B99000E3DA09FCB3093041136D4D006FF09FFCF1
:10B9A0009306B0026FF05FFD03460B0093061B0089
:10B9B0006310060503A404001386440063540400C6
:10B9C0001304F0FF93040600138B06006FF09FF939
:10B9D000330454039386160003C6F6FF3304B40001
:10B9E000930506FDE3F6BCFE138B06006FF0DFEB5C
:10B9F000130400006FF0DFFE136D0D086FF09FF66B
:10BA000093060B0093090000B3895903130606FD42
:10BA100093861600B309360103C6F6FF930506FDAB
:10BA2000E3F4BCFE6FF05FFC03460B009306800658
:10BA30006318D600130B1B00136D0D206FF09FF2DF
:10BA4000136D0D046FF01FF203460B009306C00642
:10BA50006318D600130B1B00136D0D026FF09FF0DF
:10BA6000136D0D016FF01FF083A60400938C44004A
:10BA7000A30D01022306D10813041000930A00004D
:10BA80009304C1086F00801C136D0D0193760D02A5
:10BA9000638006069384740093F484FF03A3040078
:10BAA00083AA4400938C8400E3DC0A0833036040DB
:10BAB000B336600033085041B30AD8409306D00231
:10BAC000A30DD102930610001306F0FF6306C44EC7
:10BAD00013060D00B3655301137DFDF7639E054CFE
:10BAE0006304046613061000639CC64C6F00900646
:10BAF00093760D01938C44006388060003A3040031
:10BB0000935AF3416FF05FFA93760D0403A3040098
:10BB10006388060013130301135303416FF05FFEA4
:10BB200093760D20E38E06FC131383011353834198
:10BB30006FF01FFD13760D0283A60400938444006A
:10BB4000630A06009357FC4123A0860123A2F60056
:10BB50006FF01FCC13760D016306060023A086014B
:10BB60006FF01FCB13760D04630606002390860149
:10BB70006FF01FCA93770D20E38207FE23808601B2
:10BB80006FF01FC9136D0D0193760D0263840602D9
:10BB90009384740093F484FF03A3040083AA4400F5
:10BBA000938C8400137DFDBF93060000A30D01025A
:10BBB0006FF09FF193760D01938C4400638606002D
:10BBC00003A304006F00000193760D046388060050
:10BBD00003D30400930A00006FF0DFFC93760D207E
:10BBE000E38006FE03C304006FF0DFFEB786FFFFAD
:10BBF00093C60683231ED10203A30400B706008167
:10BC00009387C63A938C4400930A0000136D2D006D
:10BC10002328F100930620006FF05FF9A30D0102C5
:10BC20009306F0FF938C440083A404006304D42C97
:10BC3000130604009305000013850400EFA00FC253
:10BC4000930A000063040500330495402322510148
:10BC500063D48A00232281008346B10363880600EF
:10BC600083274100938717002322F10093772D004B
:10BC70002320F10263880700832741009387270070
:10BC80002322F10093774D082322F10263940706E3
:10BC900083274100B386F940635ED0041308000196
:10BCA00093087000832781010326410483258104C2
:10BCB00023A0FD001306160013858D00634ED84A9D
:10BCC00023A2DD00B386B6002324D1042322C104BD
:10BCD00093067000930D050063DEC6001306010491
:10BCE0009305090013050A00EFF0DF88631A055A6F
:10BCF000938D0B008346B103638806041306B103DA
:10BD000023A0CD00130610008326410423A2CD00FA
:10BD100003268104938616002322D10413061600FD
:10BD20002324C10413067000938D8D00635ED6003A
:10BD3000130601049305090013050A00EFF09F8321
:10BD400063100556938D0B00832701026388070457
:10BD50001306C10323A0CD0013062000832641044F
:10BD600023A2CD0003268104938616002322D1044A
:10BD7000130626002324C10413067000938D8D0042
:10BD8000635ED600130601049305090013050A003B
:10BD9000EFF04FFE63160550938D0B008327410291
:10BDA000930600086394D70683274100B386F940C1
:10BDB000635ED004130800019308700083274101DB
:10BDC000032641048325810423A0FD0013061600E9
:10BDD00013858D006346D83E23A2DD00B386B600EE
:10BDE0002324D1042322C10493067000930D05007F
:10BDF00063DEC600130601049305090013050A005B
:10BE0000EFF04FF7631E0548938D0B00B38A8A400D
:10BE1000635E5005130800019308700083274101F9
:10BE2000832641040326810423A0FD009386160087
:10BE300093858D00634A583D23A25D01B38ACA00F1
:10BE4000232451052322D10413067000938D05008D
:10BE5000635ED600130601049305090013050A006A
:10BE6000EFF04FF1631E0542938D0B008326810492
:10BE700023A28D0023A09D003384860083264104E5
:10BE80002324810413067000938616002322D10414
:10BE900013878D00635ED600130601049305090025
:10BEA00013050A00EFF00FED631C053E13870B002E
:10BEB00093774D00639A07388327410063D4F900D4
:10BEC0009389070083278104330C3C01638C0700AE
:10BED000130601049305090013050A00EFF08FE92A
:10BEE0006310053C2322010493840C00938D0B0006
:10BEF0006FF01F9213850400EFB00FBD130405000F
:10BF0000930A00006FF09FD4136D0D0193760D021C
:10BF1000638006029384740093F484FF03A30400F7
:10BF200083AA4400938C8400930610006FF01FC80E
:10BF300093760D01938C44006386060003A30400EE
:10BF40006F00000193760D046388060003D304009C
:10BF5000930A00006FF05FFD93760D20E38006FEEC
:10BF600003C304006FF0DFFEB70600819387063C31
:10BF70006FF05F9693760D01938C44006386060004
:10BF800003A304006F00000193760D04638806008C
:10BF900003D30400930A00006FF0DF9593760D2021
:10BFA000E38006FE03C304006FF0DFFE13060D00FE
:10BFB000930610006FF01FB2130610006386C63898
:10BFC000130620006386C6149306010F9395DA01C9
:10BFD00013767300135333001306060333E365002F
:10BFE00093DA3A00A38FC6FEB36553019384F6FF3C
:10BFF0006396050293751D00638A0500930500038F
:10C000006306B600A38FB4FE9384E6FF9307010F87
:10C01000930A0400338497406FF05FC39386040053
:10C020006FF0DFFA93770D4093080000130E010FB5
:10C030002322F100130503001306A000930600005D
:10C0400093850A00232611039304FEFF2322C103D4
:10C0500023206102EF00D017032E41028328C10282
:10C060008327410013050503A30FAEFE9388180034
:10C0700003230102638E07048327810083C6070020
:10C08000639816059307F00F6384F80463960A001B
:10C090009307900063FE67028327C1008325C101D7
:10C0A00023206102B384F440138607001385040043
:10C0B000EFB04FA383278100930800000323010200
:10C0C00083C6170063860600938717002324F100B8
:10C0D000130503001306A0009306000093850A00D1
:10C0E0002322110323206102EF00404B03230102AE
:10C0F0008328410263960A0093079000E3F867F0F3
:10C1000013030500938A0500138E04006FF09FF25D
:10C110009304010F832701019376F3009384F4FFC6
:10C12000B386D70083C60600135343002380D40090
:10C130009396CA0133E3660093DA4A00B36653016B
:10C14000E39A06FC6FF09FEC9304010FE39006EC7A
:10C1500013761600E30C06EA93060003A307D10E3C
:10C160006F00C01F6300061C2306C108A30D010257
:10C17000938C04006FF05F909385050123A20D015D
:10C180002324B1042322C10463D6C8021306010488
:10C190009305090013050A002326D102EFF08FBD95
:10C1A000631005108326C10213850B0093087000ED
:10C1B00013080001938606FF930D05006FF09FAEF4
:10C1C0009385050123A20D012324B1042322C10478
:10C1D00063D6C802130601049305090013050A007B
:10C1E0002320D102EFF00FB9631C050A8326010258
:10C1F00013850B009308700013080001938606FF57
:10C20000930D05006FF09FBB1306060123A20D01DD
:10C210002324C1042322D10463D2D80213060104CB
:10C220009305090013050A00EFF0CFB4631A050661
:10C2300093850B009308700013080001938A0AFF8E
:10C24000938D05006FF09FBD832741003384F94033
:10C25000E35480C693040001930A70000326810111
:10C2600083274104832681042320C7009387170076
:10C2700063CE8406B3868600232287002324D1045C
:10C280002322F10413077000E358F7C213060104D8
:10C290009305090013050A00EFF0CFADE30E05C0CA
:10C2A0008357C90093F70704639607D08320C11210
:10C2B0000324811213050C00832441120329011267
:10C2C0008329C111032A8111832A4111032B0111F2
:10C2D000832BC110032C8110832C4110032D0110DE
:10C2E000832DC10F1301011367800000938606019F
:10C2F000232297002324D1042322F104130787006B
:10C3000063DEFA00130601049305090013050A0011
:10C31000EFF04FA6E31605F813870B00130404FF94
:10C320006FF0DFF383278104E38C07F61306010423
:10C330009305090013050A00EFF0CFA36FF05FF635
:10C340009306F0FFE314D4C6E39E0ACC9306900054
:10C35000E3EA66CC13030303A307610E9304F10E13
:10C360006FF0DFCA130101FE232C8100232A910004
:10C3700023282101232E1100232631011309050052
:10C3800093840500130406006308050083278503D2
:10C3900063940700EF601FE9832784012324F400DE
:10C3A0008357C40093F787006388070A8327040133
:10C3B0006384070A8317C40093F9F40F93F4F40F0E
:10C3C000139727016356070A8327040103250400F6
:10C3D0003305F54083274401634AF50093050400C3
:10C3E00013050900EF605FCA631005088327840006
:10C3F000130515009387F7FF2324F4008327040017
:10C40000138717002320E40023803701832744018A
:10C41000638CA7008357C40093F71700638E07004F
:10C420009307A000639AF400930504001305090024
:10C43000EF609FC5631A05028320C10103248101B7
:10C440001385040003290101832441018329C100CC
:10C450001301010267800000930504001305090021
:10C46000EF609F8EE30805F49304F0FF6FF0DFFCAC
:10C4700037270000B3E7E7002316F40083274406BC
:10C4800037E7FFFF1307F7FFB3F7E7002322F406B0
:10C490006FF09FF3B7270081138605009305050011
:10C4A00003A587986FF01FECB727008183A78798B3
:10C4B000130101FE232C8100232A9100232E110059
:10C4C000130405009384060083A7470363980504BB
:10C4D00063960700B72700819387078183A7070E1C
:10C4E0009386040013060000930541001305040021
:10C4F000E78007009307F0FF6318F50023A004000E
:10C500009307A0082320F4008320C10103248101A4
:10C510008324410113010102678000006396070034
:10C52000B72700819387078183A7070E93860400AE
:10C530006FF0DFFBB7270081930606001386050026
:10C540009305050003A587986FF01FF6B7270081B4
:10C5500083A7879883A7470363960700B7270081BF
:10C560009387078103A3070E670003006384050216
:10C570009307F00F63FAC7009307A0082320F50084
:10C580001305F0FF678000002380C500130510002D
:10C590006780000013050000678000009387050096
:10C5A0001308060093880600130305006396062807
:10C5B00037170081130747D763F6C50EB70601008A
:10C5C0006378D60C9306F00FB3B6C6009396360088
:10C5D000B358D6003307170103470700B306D70047
:10C5E000130700023307D740630C0700B397E70037
:10C5F000B356D5003318E600B3E5F6003313E50073
:10C600001355080133F7A502131608011356060146
:10C6100093560301B3D5A50213170701B366D700DC
:10C62000B307B6021387050063FEF600B386060162
:10C630001387F5FF63E8060163F6F6001387E5FF4D
:10C64000B3860601B386F640B3F7A60213130301BF
:10C6500013530301B3D6A6029397070133E3670090
:10C66000B305D60213850600637CB300330368006C
:10C670001385F6FF636603016374B3001385E6FF59
:10C68000131707013367A700930500006F00400EE2
:10C69000B708000193060001E36C16F393068001CE
:10C6A0006FF01FF3631606009306100033D8C6021E
:10C6B000B70601006372D80C9306F00F63F406010D
:10C6C00093088000B35618013307D700834607004C
:10C6D00013070002B38616013307D7406318070A11
:10C6E000B3870741930510001356080193180801FA
:10C6F00093D808019356030133F7C702B3D7C70293
:10C7000013170701B366D7003385F80213870700B4
:10C7100063FEA600B38606011387F7FF63E80601F0
:10C7200063F6A6001387E7FFB3860601B386A6402B
:10C73000B3F7C6021313030113530301B3D6C602A2
:10C740009397070133E36700B388D8021385060087
:10C75000637C1301330368001385F6FF63660301EE
:10C76000637413011385E6FF131707013367A700EE
:10C770001305070067800000B70600019308000159
:10C78000E362D8F4930880016FF0DFF33318E80018
:10C79000B3D5D7003313E500B356D50013550801C0
:10C7A000B397E70033F7A502B3E8F6009317080143
:10C7B00093D7070113D60801B3D5A50213170701B4
:10C7C0003367C700B386B70213860500637ED700C0
:10C7D000330707011386F5FF636807016376D70007
:10C7E0001386E5FF33070701B306D74033F7A602E8
:10C7F0009398080193D80801B3D6A602131707012E
:10C80000B385D702B36717011387060063FEB7002D
:10C81000B38707011387F6FF63E8070163F6B700E4
:10C820001387E6FFB3870701B387B7409315060167
:10C83000B3E5E5006FF05FEB63E6D518370701005D
:10C8400063F4E6041308F00F3337D80013173700EA
:10C8500037180081130848D7B3D5E600B385050122
:10C8600003C80500930500023308E800B3850541BD
:10C870006396050213071000E3ECF6EE3335C500AE
:10C88000134715006FF0DFEEB70500011307000135
:10C89000E3E0B6FC130780016FF09FFB33570601FE
:10C8A000B396B600B366D70093DE060133D707010F
:10C8B000B378D703B397B700335805013363F80053
:10C8C0009397060193D70701135803013316B60057
:10C8D0003357D7039398080133E80801338FE702F1
:10C8E000130E0700637EE8013308D800130EF7FF2C
:10C8F0006368D8006376E801130EE7FF3308D800B9
:10C900003308E841B378D8033358D8039398080123
:10C91000B38E07039317030193D70701B3E7F8001A
:10C920001307080063FED701B387D7001307F8FF8A
:10C9300063E8D70063F6D7011307E8FFB387D70092
:10C94000131E0E01B387D741B70E01003367EE0007
:10C950001388FEFF337307019358070133780601EC
:10C9600013560601330E03033388080393560E0152
:10C970003303C30233030301B3866600B388C802DE
:10C9800063F40601B388D80113D60601B308160173
:10C9900063E61703E39A17CFB70701009387F7FF02
:10C9A000B3F6F60093960601337EFE003315B5000C
:10C9B000B386C60193050000E37CD5DA1307F7FFC1
:10C9C0006FF09FCC93050000130700006FF05FDA53
:10C9D00093080600138706009307050013880500D7
:10C9E000639C0622B7160081938646D763FCC50C6C
:10C9F00037030100637E660A1303F00F6374C300FC
:10CA0000130780003353E600B386660003CE0600AA
:10CA100013030002330EEE003303C341630C030023
:10CA2000B3956500335EC501B31866003368BE0078
:10CA3000B317650013D608013377C80213950801B0
:10CA40001355050193D607013358C8021317070180
:10CA5000B366D7003308050363FA0601B3861601EF
:10CA600063E6160163F40601B3861601B386064138
:10CA700033F7C6029397070193D70701B3D6C602CF
:10CA8000B306D50213150701B367F50063FAD700A3
:10CA9000B387170163E6170163F4D700B387170163
:10CAA000B387D74033D56700930500006780000047
:10CAB0003703000113070001E36666F413078001E2
:10CAC0006FF05FF46316060013061000B3581603E8
:10CAD0003706010063F2C80A1306F00F63741601EB
:10CAE0001307800033D6E800B386C60003CE0600E5
:10CAF00013030002330EEE003303C341631803082F
:10CB0000B385154113D70801139508011355050185
:10CB100013D60701B3F6E502B3D5E50293960601F5
:10CB2000B3E6C600B305B50263FAB600B3861601D4
:10CB300063E6160163F4B600B3861601B385B6400A
:10CB4000B3F6E5029397070193D70701B3D5E50242
:10CB5000B305B50213950601B367F50063FAB70094
:10CB6000B387170163E6170163F4B700B3871701B2
:10CB7000B387B7406FF01FF33706000113070001BA
:10CB8000E3E2C8F6130780016FF0DFF5B3986800A1
:10CB900033D7C501B3176500335EC50113D508014E
:10CBA000B376A702B3956500336EBE009395080176
:10CBB00093D5050113560E013357A702939606012C
:10CBC000B3E6C6003387E50263FAE600B3861601D2
:10CBD00063E6160163F4E600B38616013386E64089
:10CBE000B376A602131E0E01135E0E013356A60283
:10CBF000939606013386C502B3E5C60163FAC50004
:10CC0000B385150163E6150163F4C500B38515010D
:10CC1000B385C5406FF01FEFE3EAD5E837070100A1
:10CC200063FCE604930EF00F33B7DE0013173700F2
:10CC300037130081B3D8E600130343D7B3886800E5
:10CC400083CE0800130E0002B38EEE00330EDE41D9
:10CC5000631E0E0263E4B600636AC500B307C540F5
:10CC6000B385D5403335F5003388A54013850700DB
:10CC7000930508006FF09FE3B70800011307000158
:10CC8000E3E816FB130780016FF09FFA3357D601D4
:10CC9000B396C601B366D70013D8060133D7D501C2
:10CCA00033730703B395C501B357D501B3E7B70095
:10CCB0009395060193D5050193D807013316C60154
:10CCC0003315C5013357070313130301B368130169
:10CCD000338FE5021303070063FEE801B388D80031
:10CCE0001303F7FF63E8D80063F6E8011303E7FFD7
:10CCF000B388D800B388E84133FF0803B3D80803EA
:10CD0000131F0F01338815039395070193D5050170
:10CD1000B365BF009387080063FE0501B385D500A6
:10CD20009387F8FF63E8D50063F605019387E8FF72
:10CD3000B385D50013130301370F01003363F300EC
:10CD40009307FFFFB378F300B38505411353030145
:10CD500013580601B377F6003387F802B307F302DE
:10CD6000B388080333030303B388F800135807019B
:10CD7000330818016374F8003303E3019357080183
:10CD800033836700B70701009387F7FF3378F80014
:10CD9000131808013377F7003307E80063E66500EE
:10CDA000639E6500637CE5003306C7403337C700E8
:10CDB0003307D7003303E340130706003307E5408A
:10CDC0003335E500B3856540B385A540B397D501FC
:10CDD0003357C70133E5E700B3D5C5016FF01FCD69
:10CDE000130101FF83270500832E4500032F8500D3
:10CDF0000327C50003A3050083A2450083AF850078
:10CE000083A8C500F3262000B785000093560701CC
:10CE10009385F5FF131E0701139608011358F701B8
:10CE2000B3F6B60013D70801135E0E0113560601C0
:10CE30003377B70093D8F801639EB600B3E5D70106
:10CE4000B3E5E501B3E5C50163920508631CD70AA4
:10CE50006F008000631AB700B3655300B3E5F501B6
:10CE6000B3E5C50063960504130510006316D702E9
:10CE70006394670263925E026310FF03631ECE0039
:10CE800063041803631A070033E5D7013365E5012E
:10CE90003365C5013335A00013010101678000002F
:10CEA000736018006F000006130500006FF0DFFECE
:10CEB000B78500009385F5FF6390B60433E5D7018D
:10CEC000B366E501B3E6C6016388060213150E01D9
:10CED00013550541E35605FCB78700009387F7FF1C
:10CEE00013051000E31AF7FAB3675300B3E7F7012D
:10CEF000B3E7C700E38207FA13160601135606418B
:10CF0000E35006FA130510006FF01FF9130101FF3B
:10CF1000832F050003284500832E85008327C50045
:10CF200083A2050083A8450003AF850003A6C500C2
:10CF300073272000B785000093D607019385F5FF7E
:10CF400013930701131E060113570601B3F6B6002B
:10CF50001353030193D7F701135E0E013377B70024
:10CF60001356F6016390B602B3E50F01B3E5D501A0
:10CF7000B3E565006384050C736018001305E0FFDA
:10CF80006F00000D631AB700B3E55800B3E5E50183
:10CF9000B3E5C501E39205FE6394060A33E50F018C
:10CFA0003365D5013365650013351500631A070035
:10CFB000B3E55800B3E5E501B3E5C50163820506B5
:10CFC00063020508631606081305F0FF6F004008AA
:10CFD000130500006FF0DFFD6348D70663DAE60053
:10CFE0001305F0FF63860706130510006F00400667
:10CFF000636C6E04631CC3036368DF05631CDF039B
:10D0000063E408056394080163E0F205E36A18FD30
:10D0100013050000639E080363FC5F026FF05FFC72
:10D0200063040502130500006F008002E36AC3FB7E
:10D030006FF05FFFE3E6EEFB6FF0DFFEE306D7F491
:10D04000E30807F8E38AC7F813051000E39E07F624
:10D050001301010167800000130101FF832F050008
:10D0600003284500832E85008327C50083A2050081
:10D0700083A8450003AF850003A6C50073272000E1
:10D08000B785000093D607019385F5FF1393070139
:10D09000131E060113570601B3F6B600135303011E
:10D0A00093D7F701135E0E013377B7001356F601DD
:10D0B0006390B602B3E50F01B3E5D501B3E56500B2
:10D0C000638A050C73601800130520006F000005CB
:10D0D000631AB700B3E55800B3E5E501B3E5C50150
:10D0E000E39205FE639A060A33E50F013365D50125
:10D0F0003365650013351500631A0700B3E5580062
:10D10000B3E5E501B3E5C50163880506631C0500C9
:10D110006380C70213051000639807001301010123
:10D1200067800000E31C06FE1305F0FF6FF01FFF91
:10D13000E342D7FE63DAE6001305F0FFE38007FE63
:10D14000130510006FF09FFDE3666EFC631CC303C4
:10D15000E362DFFD631CDF03E3EE08FB6394080179
:10D16000E3EAF2FBE36A18FD13050000E39808FB0D
:10D17000E3F65FFA6FF05FFCE30E05F813050000BD
:10D180006FF0DFF9E36AC3FB6FF05FFFE3E6EEFBEE
:10D190006FF0DFFEE300D7F4E31C07F61305000091
:10D1A0006FF0DFF5130101F42328210B2324410B39
:10D1B0002322510B2320610B232C8109232A91095F
:10D1C00013090500232E110A232C810A232A910A10
:10D1D0002326310B232E71092328A1092326B10907
:10D1E00003A5050083A7450083A6850083AAC50083
:10D1F000832C0600032B4600032C8600032AC6005E
:10D20000F32420003786000013970A0193D90A01FE
:10D21000135707011306F6FF232651072320A10603
:10D220002322F1062324D1062328A102232AF10276
:10D23000232CD102232EE102B3F9C90093DAFA01BB
:10D2400063800906638EC916370501003367A7009E
:10D25000232EE102130601039307C10303A707006E
:10D2600083A6C7FF9387C7FF1317370093D6D6014E
:10D270003367D70023A2E700E312F6FE83270103FA
:10D2800037C5FFFF13051500939737002328F102D8
:10D29000B389A900930B0000130400006F008014F1
:10D2A00033E6A7003366D6003366E6006306062041
:10D2B0006300070613050700EF300065930645FF7E
:10D2C00093D7564093F6F601638E06061307C0FF08
:10D2D0003387E70213030103130800029395270025
:10D2E0003308D8401307C7003307E3006314E3088B
:10D2F00013070108B305B700032701039387F7FF5E
:10D30000B316D70023A8D5FA9306F0FF6F00000AE2
:10D31000638A060013850600EF30005F13050502DF
:10D320006FF0DFF9638A070013850700EF30C05DF7
:10D33000130505046FF09FF8EF30005D1305050637
:10D340006FF0DFF71306C0FF3386C7021307C10370
:10D3500093063000B305C70083A505009386F6FF4A
:10D360001307C7FF2322B700E3D6F6FE9387F7FF24
:10D370006FF09FF90326C7FF83280700330EB7001D
:10D3800033560601B398D800336616012320CE0029
:10D390001307C7FF6FF09FF51397270013060103CC
:10D3A0003307E600232007009387F7FFE396D7FEB5
:10D3B000B7C9FFFF93891901B389A9406FF09FEDA9
:10D3C000B3E7A700B3E7D700B3E7E700638C070E26
:10D3D0001317070113570741930B30001304000183
:10D3E000E34C07EA13150A013787000093570A0137
:10D3F000135505011307F7FF232641072320910743
:10D40000232261072324810723209105232261051C
:10D41000232481052326A104B3F7E700135AFA0158
:10D420006386070A6384E71C370701003365E5005C
:10D430002326A104930501041307C10483260700D2
:10D440000326C7FF1307C7FF939636001356D6016E
:10D45000B3E6C6002322D700E392E5FE03270104CA
:10D4600037C5FFFF13051500131737002320E1040C
:10D47000B387A70093060000B38737012324F10088
:10D48000938717002322F10093972B00B3E7D7006F
:10D490009387F7FF1306E00033C74A016366F61A65
:10D4A0003716008193972700130686D3B387C700EA
:10D4B00083A707006780070093090000930B100003
:10D4C0006FF09FDD930B20006FF01FDDB3679B01B2
:10D4D000B3E78701B3E7A70063800714630E050471
:10D4E000EF308042130645FF135756401376F6017E
:10D4F000630006089306C0FFB306D70213030104B6
:10D5000013080002931527003308C8409386C6000D
:10D51000B306D3006316D30893070108B385B70099
:10D52000832701041307F7FF3396C70023A0C5FC28
:10D530009306F0FF6F00400A630A0C0013050C000D
:10D54000EF30803C130505026FF0DFF9630A0B0032
:10D5500013050B00EF30403B130505046FF09FF8F7
:10D5600013850C00EF30403A130505066FF09FF766
:10D570001306C0FF3306C7029307C10493063000A9
:10D58000B385C70083A505009386F6FF9387C7FF81
:10D5900023A2B700E3D6E6FE1307F7FF6FF05FF9AB
:10D5A00083A7C6FF83A80600338EB600B3D7070152
:10D5B000B398C800B3E717012320FE009386C6FF87
:10D5C0006FF05FF59317270013060104B307F60009
:10D5D00023A007001307F7FFE316D7FEB7C7FFFF27
:10D5E00093871701B387A7406FF0DFE8336B9B0188
:10D5F000336B8B01336BAB0093062000E30E0BE61D
:10D60000131505011355054193063000E34605E661
:10D61000130400016FF05FE693070000930610000B
:10D620006FF09FE513040001B7870000232EF1047B
:10D63000232C0104232A0104232801049387F7FFE4
:10D64000130700006F00101983250103032E010446
:10D65000370801001306F8FF93D3050193570E0115
:10D66000B3F5C500337ECE00B386B702338AC50357
:10D67000B388C3033385160193560A01B386A60007
:10D68000B389F30263F41601B3890901032341044A
:10D6900013D80601B3F6C600337ACA009396060182
:10D6A000B3864601935F03013373C3002326D10081
:10D6B0002320D106B308B302B386BF0233866302C8
:10D6C0003385C60093D60801B386A600B38BF30357
:10D6D00063F6C60037060100B38BCB0013D60601F4
:10D6E000B70E01002320C1001386FEFF33F5C600EC
:10D6F000B3F8C8001315050133051501B306A800DA
:10D700002320D1028326410393D2060133F6C600BB
:10D71000B308C603338AC20313D80801B386C7020D
:10D72000B3864601B306D800338F570263F446012F
:10D73000330FDF0113D80601370A01003308E8016F
:10D74000930EFAFF130B080033F8D601B3F8D80193
:10D750001318080133081801B30E6602B388620279
:10D7600093DA0E01B386CF02B3861601B386DA00D0
:10D77000338F5F0263F41601330F4F0193D8060114
:10D78000B388E801B70A0100232811019388FAFF42
:10D79000B3F61601B3FE1E0193960601B38DD601B2
:10D7A00083268104B3F8160193DE0601338AB8029A
:10D7B000338C1303935C0A01338FBE02330F8F0146
:10D7C000338FEC01B386D30363748F01B3865601A4
:10D7D000935A0F01B386DA00370D0100232AD100D6
:10D7E0009306FDFF337FDF00337ADA00131F0F014A
:10D7F000330F4F01032A8103232CE101B376DA00B2
:10D80000135F0A01330ACF03B38AC603B38CD7026E
:10D81000B38C4C0113DA0A01330A9A01B30CCF031B
:10D82000338CE70363749A01330CAC01935C0A01F7
:10D83000338C8C01232E8101370C0100130DFCFF6A
:10D84000337AAA01B3FAAA01131A0A01B30C5A01D6
:10D85000032A0102B3894901032A010033B5A90053
:10D86000B3890901330AAA00B30B7A01338C6B0127
:10D8700033B80901B30A0C0133B80A01333C6C0117
:10D8800033680C01B3BBAB00B30B780103288101F3
:10D89000338ABA01B33DBA0103250101330A0A01F3
:10D8A00033380A01232C010103284101B38BAB005B
:10D8B0002320310123223107832981013385BB01D4
:10D8C00033080501B30A3801B33DB5018329C1010D
:10D8D00003254101330A9A01338C3A013338A800F9
:10D8E000B33C9A0103258101B3099C01138B090004
:10D8F00083290101B3BAAA000325C101B3BB3B01CF
:10D90000B36A5801B3EDBB01333CAC00B33C9B019F
:10D91000B38D5D01B36C9C0133859D01232AA10069
:10D920000325C1042324410713580501337DA501B4
:10D930003305BD02B38AA303935B0501B305B802A7
:10D94000B3855501B385BB00B383030363F655016B
:10D95000370C0100B383830193DA0501B3837A00A6
:10D96000370C0100832AC103232E71009303FCFFAF
:10D97000B3F575003375750093950501B3F37A001F
:10D98000B385A50013D50A01B38BA702B38AC303DD
:10D99000B387770293DD0A01330EC503B387C7014E
:10D9A000B387FD0063F4C701B38B8B01370C010013
:10D9B000930DFCFF13DE0701B3F7B701330E7E01B1
:10D9C00093970701B3FDBA012320C103B38DB701BB
:10D9D000338EC802B38A1203935C0E01B387CE0262
:10D9E000B3875701B387FC00B38BD20363F45701AD
:10D9F000B38B8B0193DA0701B3897A01B70B01006E
:10DA0000938AFBFFB3F75701337E5E0193970701BB
:10DA1000B387C7012328F100B30A6F022322310321
:10DA2000B3876602B38CDF0213DE0701B38C5C019F
:10DA3000330E9E01338CEF0363745E01330C7C0163
:10DA4000935A0E01338C8A01B70A0100938AFAFFB8
:10DA5000337E5E01131E0E01B3F75701B307FE00BC
:10DA60008329C101032E4101B30ABB00B3B5BA003B
:10DA7000B30C3E0183290102338EBC00B38ABA0184
:10DA8000B3BDBA01B30B3E01B389BB0123263103F9
:10DA900083290101032B4102B335BE00B38A3A0149
:10DAA000B3B93A0123243103B389BB01B3896901B6
:10DAB000032B810223283101B38AFA00B38969015B
:10DAC000032E0102138B0900B3B7FA00B389890151
:10DAD000232A3101B389F900B3BBCB01232C3101D7
:10DAE000032EC1028329C10123265107B33DBE0184
:10DAF000B3BC3C01032E010183294102B3EDBB01FC
:10DB0000B3E5BC00B33B3E01032E410183298102F2
:10DB1000B385B501333C8E01032E8101B33D3B013A
:10DB2000B3EDBB01B337FE00B367FC00B38DB501A5
:10DB3000B38DFD00B38BD802330C1F0393D50B01BB
:10DB4000B387DE02B3878701B387F500338EEE0318
:10DB500063F68701B7050100330EBE0093D50701B8
:10DB6000370C0100338EC5019305FCFFB3F7B700F6
:10DB7000B3F5BB00B38CA20393970701B385B7003D
:10DB8000B30BCD023306C80293D70B0133069601BF
:10DB9000B387C700B382020363F49701B3828201A3
:10DBA00013D60701370C0100B30256001306FCFF21
:10DBB000B3F7C7009397070133F6CB003386C7004E
:10DBC000B38BAF02B3876302B38F7F0293DC07018D
:10DBD00033036502B38F6F00B38FFC0163F46F00F2
:10DBE000B38B8B0113D30F01370C0100B30B7301FF
:10DBF0001303FCFFB3FF6F00939F0F01B3F76700A0
:10DC00003383FF00B30CAF03B30FDD02B306D802BA
:10DC100093D70F01B3869601B387D700330F0F0355
:10DC200063F49701330F8F0193D60701370C01007E
:10DC3000338FE6019306FCFFB3F7D70093970701F4
:10DC4000B3F6DF00B386D700B38FAE02B3871303FA
:10DC5000B38E7E0293DC0701B3081503B38E1E0159
:10DC6000B38EDC0163F41E01B38F8F0193D80E01D4
:10DC7000B388F80123281101B7080100938FF8FF3A
:10DC8000B3FEFE01B3F7F701939E0E01B38EFE00C3
:10DC900083278101B38DCD0133BECD01B387B7009A
:10DCA000B3B5B700338CBD00B387C70033B6C70028
:10DCB000B30C5C00B389CC00B3876700B3887901EB
:10DCC000138B09002328F106B3B767003383F800EC
:10DCD0003336CB00B335BC00B3B25C00B3E2C20054
:10DCE000B337F300B365BE00B3B87801B3E8F8000A
:10DCF000B3855500B309D300B3851501B385E5019C
:10DD0000B3B6D9003386D50033BFE50183250101C1
:10DD1000B336D600B387D901B366DF00232AF106F4
:10DD2000330FB600B3B7D7013306FF00333FBF0050
:10DD3000B385A303B337F600336FFF00330DA5039C
:10DD400093D70501B3037802B383A3013305A80277
:10DD5000338877006376A801B70801003305150101
:10DD6000B377F80193970701B3FFF5011358080142
:10DD7000B38FF7013308D8008327C1008326010041
:10DD80003306F6013308E801B33FF601B3E9D700E3
:10DD90003308F8013305A800336A3A01939ADA0090
:10DDA000232EA106232CC10633EA4A01930701065C
:10DDB0009305010783A6C70003A6070193874700C1
:10DDC00093D636011316D600B3E6C60023AED7FEAF
:10DDD000E392F5FE83268106832A01068327C10686
:10DDE000232CD10483264106333A4001336A5A0179
:10DDF000232AD104232EF104232841059396B7004A
:10DE000063D40614131AFA01930701059305C1059B
:10DE100083A6070003A647009387470093D6160002
:10DE20001316F601B3E6C60023AED7FEE392F5FE65
:10DE30008327C105333A400193D71700232EF104FD
:10DE40008327010533EA4701232841058326410042
:10DE5000B74700009387F7FFB387F600635AF026B1
:10DE60008326010513F676006302061013052000D1
:10DE7000032641058325C105136414006386A40E9F
:10DE8000130530006388A40C6392040E13F5F600AA
:10DE900013084000630C050D938646002328D10427
:10DEA00093B646003386C600B336D600232AC10493
:10DEB000032681053386C600B336D600B386B60086
:10DEC000232CC104232ED1046F00400A13870A00BB
:10DED000832701032328F10483274103232AF10424
:10DEE00083278103232CF1048327C103232EF1040C
:10DEF000930720006382FB54930730006386FBF294
:10DF000093071000E394FBF4232E0104232C010457
:10DF1000232A0104232801046F00005013070A007C
:10DF200083270104938B06002328F10483274104EF
:10DF3000232AF10483278104232CF1048327C104BD
:10DF4000232EF1046FF0DFFA832781002322F100F2
:10DF50006FF0DFEF631C0700938686002328D1044F
:10DF600093B686006FF01FF4E31807FE8326C10501
:10DF70001396B60063500602B707F0FF9387F7FFCA
:10DF8000B3F6F600232ED10483264100B7470000E4
:10DF9000B387F600930601051305C10503A6060025
:10DFA00083A5460093864600135636009395D50107
:10DFB0003366B60023AEC6FEE312D5FEB786000078
:10DFC0009386E6FF63C6F60A8326C10593D636001C
:10DFD000232ED1048326C1059397170137060180AC
:10DFE0002316D1068326C10693D717011306F6FF21
:10DFF00093970701B3F6C600B3E7F60093971700AF
:10E000001317F70193D717000328010503254105CE
:10E010008325810533E7E7006304040073201400BF
:10E020008320C10B0324810B2322A9002320090193
:10E030002324B9002326E900130509008324410B9A
:10E040000329010B8329C10A032A810A832A410A71
:10E05000032B010A832BC109032C8109832C41095D
:10E06000032D0109832DC1081301010C67800000F5
:10E0700093072000638AF404930730006384F4025A
:10E0800063940402B7870000232E0104232C0104AB
:10E09000232A0104232801049387F7FF1364540003
:10E0A0006FF05FF3E30007FE9307F0FF232EF10408
:10E0B000232CF104232AF1042328F104B78700005C
:10E0C0009387E7FF6FF09FFDE30007FE6FF09FFB74
:10E0D00013051000639007088326010503264105F8
:10E0E0008325810513F876000325C105630E080416
:10E0F000130820001364140063860405130830001D
:10E10000638A04036392040413F8F6009308400042
:10E11000630C18039386460093B646003306D60078
:10E12000B336D600B385D500B3B6D5003305D500D8
:10E130006F008001631A07009386860093B68600FD
:10E140006FF0DFFDE31A07FE135545011345150077
:10E150001375150093061000B387F64013064007A9
:10E16000634EF62413DE57409306000093F7F70141
:10E170001306000093152600631AC6036394070470
:10E1800093083000130801053386C840B308B8006F
:10E1900083A808009387170013084800232E18FF50
:10E1A000E356F6FE930540006F00800B130801054F
:10E1B000B305B80083A5050013061600B3E6B60044
:10E1C0006FF05FFB130601083306B600032606FD59
:10E1D000130300023303F34033166600B3E6C600B0
:10E1E00013060105B305B6001306300093080000BE
:10E1F0003306C6419385450063C4C80293050108F0
:10E20000131626003386C5008325C105B3D7F50054
:10E210002328F6FC93074000B387C7416FF09FF8AF
:10E22000939E280013080105B30ED80103AF050023
:10E2300003A8C5FF93881800331F6F003358F800F8
:10E240003368E80123A00E016FF0DFFA1396270070
:10E25000130801053306C800232006009387170022
:10E26000E396B7FE03260105B336D000B3E6C60039
:10E270002328D10413F67600630E0604130620004B
:10E280000328C10513641400638AC40A130630000E
:10E29000638AC4066390040413F6F600630CF60266
:10E2A00083254105938646002328D10493B6460072
:10E2B000B385B600B3B6D500232AB1048325810502
:10E2C000B385B600232CB104B3B5D500B3870501DF
:10E2D000232EF1048327C1059396C70063DC06084B
:10E2E000232E0104232C0104232A010423280104E2
:10E2F0001364140093071000E30E05CC136424008C
:10E300006FF05FCDE31807FC032641059386860076
:10E310002328D10493B686003386C600B336D600D0
:10E32000232AC104032681053386C600232CC10499
:10E330003336D600B30706016FF09FF9E30C07F8F8
:10E340008327410593868600032681052328D1046F
:10E3500093B68600B387F600B3B6D700232AF1043C
:10E36000B387C600232CF104B3B7D700B3870701E6
:10E370006FF01FF6930701059305C10583A60700FB
:10E3800003A647009387470093D636001316D6019D
:10E39000B3E6C60023AED7FEE392F5FE8327C105A0
:10E3A00093D73700232EF10493070000E30405C23E
:10E3B00093761400E38006C26FF05FF403264105F4
:10E3C00083270105B3E7C70003268105B3E7C7002C
:10E3D0000326C105B3E7C700638E0702232E01049D
:10E3E000232C0104232A01042328D10493072000AD
:10E3F00013641400638EF402930730006382F40206
:10E4000093075000638204028327010593D73700E6
:10E410002328F10413642400930700006FF09FBBCE
:10E42000E31407FE930790002328F1046FF0DFFD4B
:10E43000E31A07FE6FF05FFDB7870000232E01048B
:10E44000232C0104232A0104232801049387F7FFC6
:10E450006FF05FB8130101FA232C8104232A910481
:10E46000232E1104232821052326310523244105C9
:10E4700023225105232061059304050083A605008E
:10E4800003A7450083A7850003A4C500832E0600CB
:10E49000032E4600832886000328C6007329200027
:10E4A000232CF1022324F100931704019319140083
:10E4B00093D70701232E81022328D102232AE102C8
:10E4C0002320D1002322E1002326F10093D9190152
:10E4D0001354F401930501001303C10083270300C3
:10E4E0000327C3FF1303C3FF939737001357D701C5
:10E4F000B3E7E7002322F300E39265FE83260100E1
:10E5000093170801232C110393963600232C110135
:10E5100093D7070193181800232AC103232E010360
:10E52000232AC1012320D1002328D1032328D1018C
:10E53000232EF10093D818011358F8011305010197
:10E54000130EC10183270E000327CEFF130ECEFF4B
:10E55000939737001357D701B3E7E7002322FE0054
:10E56000E312C5FF03270101B78700009387F7FF78
:10E57000131737002328E1006390F8020326810176
:10E5800083274101B3E7C7000326C101B3E7C700F2
:10E59000B3E7E70063940700134818003386194176
:10E5A000E31E882A635CC038639408100328410185
:10E5B000832581010323C101B368B800B3E8680073
:10E5C000B3E8E800639C0804378700001307F7FFEF
:10E5D00003284100032581008325C1009307000023
:10E5E0006312E6023367A8003367B7003367D700CA
:10E5F000630A0700B7070400B3F7F50093B71700E5
:10E60000939747002324A1022320D1022322010350
:10E610002326B102130506006F00C0449307F6FFDE
:10E6200063900706032641003387E600B336D70020
:10E630003305C800B307D500B3B6D7002322F102D3
:10E64000832781003336C500B366D6002320E1025C
:10E650003387F5003306D700B337F7000327C1002F
:10E66000B336D600B3E7D7003303E3002324C10257
:10E67000B38767002326F102130510006F00002105
:10E68000378700001307F7FF6304E6006F10C077B9
:10E6900003284100032581008325C1009307000062
:10E6A0003367A8003367B7003367D7006FF05FF4B4
:10E6B000B78700009387F7FF6396F90403254100AD
:10E6C000832581000326C100930700003367B5004E
:10E6D0003367C7003367D700630A0700B707040032
:10E6E000B377F60093B71700939747002322A10250
:10E6F0002320D1022324B1022326C102138509005D
:10E700006F0040368327C10137070800B3E7E700F1
:10E71000232EF1009307400763D4C7006F10806F6A
:10E720009307060013D357401306000093F7F70131
:10E73000130700009316270063186702639007040D
:10E74000930530003387E540B305DE0083A505005F
:10E7500093871700130E4E00232EBEFEE356F7FEDE
:10E76000930640006F00800AB306D50083A606001A
:10E77000130717003366D6006FF0DFFB13070104A1
:10E780003307D700032707FD93080002B388F8403A
:10E79000331717013366E60013073000B306D500C0
:10E7A0001308000033076740938646006344E8027D
:10E7B00093060104131727003387E6008326C1015F
:10E7C000B3D7F6002328F7FC93074000B3876740D0
:10E7D0006FF01FF983A5C6FF83AE0600131E280045
:10E7E000B3D5F500B39E1E01330EC501B3E5D501C7
:10E7F0002320BE00130818006FF01FFB139727009B
:10E800003307E5002320070093871700E398D7FE1E
:10E81000832701013336C00033E6C7002328C10037
:10E8200083260100832701010327410083258101FD
:10E83000B387F600B3B6D7002320F1028327410146
:10E840000325C101B307F7003386D70033B7E700CC
:10E85000B337D600B367F700032781008326C100D2
:10E860002322C102B305B7003386F50033B7E500B4
:10E87000B337F600B386A6003367F7003387E600A8
:10E880002324C1022326E102138509008327C10244
:10E890001397C700634407006F1040333707F8FF32
:10E8A0001307F7FFB3F7E7002326F10283270102DE
:10E8B000130515009305C1021397F7019307010291
:10E8C00083A6070003A647009387470093D6160048
:10E8D0001316F601B3E6C60023AED7FEE392F5FEAB
:10E8E0008327C1021306000093D717002326F102E5
:10E8F000B337E00003270102B367F7002320F102DA
:10E90000B78700009387F7FF631AF56C630C0972F1
:10E91000930730006312F972630604729307F0FFE5
:10E92000378500002326F1022324F1022322F1027D
:10E930002320F1021305E5FF6F00C0716304063266
:10E940003385384163940912032E41000328810066
:10E95000832EC10033660E013366D6013366D600BE
:10E96000631C0604B78700009387F7FF0328410163
:10E97000832581018326C1016312F502B367B800C4
:10E98000B3E7D700B3E7E700638A07003706040060
:10E9900033F6C60013361600131646002320E10294
:10E9A000232201032324B1022326D102630405306C
:10E9B000930706006F00000B9307F5FF639C0704A5
:10E9C00003264101B386E60033B7E600B305CE0067
:10E9D000B387E50033B7E7002322F10283278101E3
:10E9E00033B6C5003367E6002320D102B306F80032
:10E9F0003386E6003337E600B3B7F600B3E7E70047
:10EA00000327C1012324C102B38EEE00B387D701CF
:10EA10006FF05FC6B78600009386F6FF6304D500EB
:10EA20006F10C04003284101832581010326C101E5
:10EA300093070000B366B800B3E6C600B3E6E6008D
:10EA4000638A0600B7070400B377F60093B7170090
:10EA5000939747002320E102232201032324B102DC
:10EA60002326C102130600006F008039B78700001B
:10EA70009387F7FF6396F8040325410183258101FD
:10EA80000326C10193070000B366B500B3E6C600D4
:10EA9000B3E6E600638A0600B7070400B377F60022
:10EAA00093B71700939747002322A1022320E10286
:10EAB0002324B1022326C102138508006FF09FFAB8
:10EAC0008327C10037070800B3E7E7002326F100DA
:10EAD0009307400763D4A7006F1000369307050023
:10EAE0001307000233C6E70293060000B3E7E7020C
:10EAF000130700006340C7041307060063540600B1
:10EB00001307000013152600639207041307300053
:10EB10003306C7403307A300032707009387170076
:10EB200013034300232EE3FEE356F6FE13063000E4
:10EB30006F00000B131527003385A5000325050082
:10EB400013071700B3E6A6006FF0DFFA13172700CC
:10EB5000130801043307E800032707FC130E000223
:10EB6000330EFE403317C701B3E6E600130730004B
:10EB70003385A500130300003307C7401305450084
:10EB80006344E30213050104131727003307E5006C
:10EB90000325C100B357F5002320F7FC930740007D
:10EBA000B387C7406FF09FF80328C5FF032F050008
:10EBB000931E23003358F800331FCF01B38ED501C5
:10EBC0003368E80123A00E01130313006FF01FFB4D
:10EBD000139727003387E50023200700938717004A
:10EBE000E358F6FE83270100B336D000B3E6D70022
:10EBF0002320D1008326010183270100032741013F
:10EC000083258100B387F600B3B6D7002320F10235
:10EC1000832741000325C100B307F7003386D700DF
:10EC200033B7E700B337D600B367F7000327810196
:10EC30008326C1012322C102B305B7003386F50044
:10EC400033B7E500B337F600B386A6003367F700A5
:10EC50003387E6002324C1022326E102138508003E
:10EC60006FF0DFC2B787000013851900938FE7FFAD
:10EC7000B37FF5010323410103288101032EC10164
:10EC800083254100032F8100832EC10063940F2C44
:10EC900033E5E5013365D5013365D500639A091C79
:10ECA0006318050C2320E1022322610223240103BF
:10ECB0002326C10303250102832541028326810205
:10ECC0000327C102B367B500B3E7D700B3E7E70096
:10ECD000E38A0772232AB1022328A102232CD1023E
:10ECE000232EE102930501039307C10303A7070045
:10ECF00083A6C7FF9387C7FF1317170093D6F601A4
:10ED00003367D70023A2E700E392F5FE83270103D0
:10ED10009397170013F77700E308076C1307200099
:10ED20008326C10313661600E30EE96A1307300059
:10ED3000E302E96AE31A096A13F7F7009305400052
:10ED4000E304B76A9387470093B74700032741035B
:10ED50003387E7003337F70083278103B307F700D2
:10ED6000B3B7E700B387D700232EF1026F00D06757
:10ED7000B3670301B3E7C701B3E7E700639C07008C
:10ED80002320D1022322B1022324E1032326D1032D
:10ED90006FF05FF23387E600B336D7003303B3007A
:10EDA000B307D300B3B6D7003333B3003363D30014
:10EDB000B305E8012322F102B38765002324F102A1
:10EDC000B3B5E501B3B76700B3E7F500330EDE0175
:10EDD000B387C7012320E1021397C70063460700EA
:10EDE0002326F1026FF01FED3707F8FF1307F7FF37
:10EDF000B3F7E7002326F102130510009307000084
:10EE00000327010293767700E38C066693062000C1
:10EE10008328C10293E71700E308D9629306300004
:10EE2000E308D95E631209049376F7009305400066
:10EE3000638CB60203284102130747002320E10236
:10EE400013374700330807013337E8002322010353
:10EE50000328810233080701232401033338E80023
:10EE6000B30618012326D102E31206626F00506236
:10EE70009387F7FF6396F908631405006F1040004D
:10EE8000B7070400B3F7FE0093B717009397470046
:10EE90006390380BB3680301B3E8C801B3E8E80036
:10EEA000E388087C9316DE00E3D8067C630405063D
:10EEB000378700002326E1022324010223220102D6
:10EEC00023200102130501021307C1028326070054
:10EED0008325C7FF1307C7FF9396360093D5D50147
:10EEE000B3E6B6002322D700E312E5FE03270102B2
:10EEF00013040000131737002320E1026F00800283
:10EF00006396F800930700006FF0DFF893070000A6
:10EF1000631005022320E10223226102232401035E
:10EF20002326C103378500001305F5FF6FF05FED61
:10EF300033680301336EC8013367EE00E31A07F646
:10EF40002320D1022322B1022324E1032326D1036B
:10EF50006FF05FFD3387E6003303B300B336D700AD
:10EF60002320E1023307D300B336D7003333B30095
:10EF7000B366D3003308E8013303D800B336D300B7
:10EF80003338E8013368D800330EDE013308C80196
:10EF90002322E102232461022326010393070102B5
:10EFA0009305C10203A7070083A647009387470084
:10EFB000135717009396F6013367D70023AEE7FE89
:10EFC000E392F5FEB78700009387F7FF630CF50027
:10EFD0008327C10293D717002326F102930700006D
:10EFE0006FF01FE2630E0902930730006314F90209
:10EFF000630804029307F0FF378500002326F1021F
:10F000002324F1022322F1022320F1021305E5FF5C
:10F010006F00000293072000E31EF9FCE30C04FCE0
:10F0200023260102232401022322010223200102BC
:10F03000930750006FF0DFDC93072000E310F98E98
:10F04000E30E048C23260102232401022322010261
:10F0500023200102130600006FF09FFD6356C028B5
:10F060006392080C03284101832581010323C10118
:10F07000B368B800B3E86800B3E8E800638608D472
:10F080009307F6FF639A0706832841003387E6401B
:10F0900033B6E6003385084133BEA8003305C540CA
:10F0A0002320E1022322A1021306000063F6E600FA
:10F0B000330618411336160003288100B366C601D3
:10F0C0003306B8403335C8003306D6402324C10286
:10F0D00063860600B387054193B717000327C10075
:10F0E000B3E7A70033076740B307F7402326F102D1
:10F0F000130510006F00001D378700001307F7FF8E
:10F100006308E6D8130740076352F704930710001B
:10F11000232E0100232C0100232A01002328F100C3
:10F120006F008012B78700009387F7FF6388F9D8D4
:10F130008327C10137070800B3E7E700232EF1005A
:10F1400093074007E3C4C7FC9307060013D3574057
:10F150001306000093F7F70113070000931627002A
:10F160006318670263900704930530003387E54016
:10F17000B305DE0083A5050093871700130E4E002C
:10F18000232EBEFEE356F7FE930640006F00800A72
:10F19000B306D50083A60600130717003366D60012
:10F1A0006FF0DFFB130701043307D700032707FDC8
:10F1B00093080002B388F840331717013366E6005E
:10F1C00013073000B306D50013080000330767406B
:10F1D000938646006344E802930601041317270050
:10F1E0003387E6008326C101B3D7F6002328F7FC56
:10F1F00093074000B38767406FF01FF983A5C6FFF0
:10F2000083AE0600131E2800B3D5F500B39E1E0181
:10F21000330EC501B3E5D5012320BE001308180045
:10F220006FF01FFB139727003307E500232007002B
:10F2300093871700E398D7FE832701013336C00078
:10F2400033E6C7002328C10083264100832501003F
:10F2500003270101832741013387E540B387F64047
:10F2600033B6F600B3B6E500B386D7402322D10209
:10F270002320E1029306000063F4E50093B6170033
:10F28000B3E6C60003278101032681003307E64069
:10F29000B307D7402324F102B335E600130600007C
:10F2A00063840600133617008327C1000327C101BA
:10F2B0003366B60013850900B387E740B387C740BC
:10F2C0002326F1028327C1021397C700E3500710DA
:10F2D000370708001307F7FFB3F7E7002326F1020B
:10F2E000930905006F00C067630806343385384111
:10F2F00063900914032E410003268100032FC100EF
:10F30000B36ECE00B3EEEE01B3EEDE00639C0E04EE
:10F31000B78700009387F7FF832841018325810188
:10F320008326C101130600006312F502B3E7B8009B
:10F33000B3E7D700B3E7E700638A070037060400A6
:10F3400033F6C60013361600131646002320E102DA
:10F35000232211032324B1022326D102130408001F
:10F360006FF0CFE49307F5FF639A07068328410106
:10F37000B306D740B335D7003385C84133B3A800AF
:10F380003305B5402320D1022322A10293050000BA
:10F390006376D700B3051E4193B51500832881011C
:10F3A000B3E66500B385C84033B5B800B385D54032
:10F3B0002324B10263860600B307164193B71700F2
:10F3C0000327C101B3E7A700130408003307E7418F
:10F3D000B307F7402326F1026FF09FD1B7860000F4
:10F3E0009386F6FFE316D526832841018325810104
:10F3F0000326C10193070000B3E6B800B3E6C600D8
:10F40000B3E6E600638A0600B7070400B377F600A8
:10F4100093B71700939747002320E102232211039B
:10F420002324B1022326C102130408006FF08FE3E6
:10F43000B78700009387F7FF6396F804032541011F
:10F44000832581010326C10193070000B366B5003F
:10F45000B3E6C600B3E6E600638A0600B707040019
:10F46000B377F60093B71700939747002322A102C2
:10F470002320E1022324B1022326C10213850800C0
:10F480006FF09FFA8327C10037070800B3E7E70052
:10F490002326F10093074007E3C0A71C930705004C
:10F4A0001307000233C6E70293060000B3E7E70242
:10F4B000130700006340C7041307060063540600E7
:10F4C000130700001315260063920704130730008A
:10F4D0003306C7403307A3000327070093871700AD
:10F4E00013034300232EE3FEE356F6FE130630001B
:10F4F0006F00000B131527003385A50003250500B9
:10F5000013071700B3E6A6006FF0DFFA1317270002
:10F51000130301043307E300032707FC930E0002E3
:10F52000B38EFE403317D701B3E6E6001307300071
:10F530003385A500130E00003307C74013054500AF
:10F540006344EE0213050104131727003307E50097
:10F550000325C100B357F5002320F7FC93074000B3
:10F56000B387C7406FF09FF80323C5FF832F0500C3
:10F57000131F2E003353F300B39FDF01338FE501D8
:10F580003363F30123206F00130E1E006FF01FFB87
:10F59000139727003387E500232007009387170080
:10F5A000E358F6FE83270100B336D000B3E6D70058
:10F5B0002320D10083264101832501010327010077
:10F5C000832741003387E540B387F64033B6F60022
:10F5D000B3B6E500B386D7402322D1022320E1024F
:10F5E0009306000063F4E50093B61700B3E6C60087
:10F5F00003278100032681013307E640B307D74084
:10F600002324F102B335E6001306000063840600EC
:10F61000133617008327C1010327C1003366B600E4
:10F6200013850800B387E740B387C7402326F1025C
:10F63000130408006FF01FC9B787000093851900F5
:10F640001385E7FFB3F5A500032F41010323410014
:10F65000032E8100832EC100832F81018322C101EB
:10F6600063920524B365FF013365C301B3E555001B
:10F670003365D501B3E5E5003365D500639C09101A
:10F68000631405022320E1022322E1032324F10372
:10F690002326510213040800639E05E01304E9FFCA
:10F6A000133414006FF00FE1639A05002320D10298
:10F6B000232261022324C1036FF04FEDB387E6409C
:10F6C000B308E34133B5F600B3351301B388A8405E
:10F6D0002320F102232211031305000063F6F60034
:10F6E00033056F4013351500B303FE413365B50094
:10F6F000338AA34023244103B33A7E0093090000D8
:10F700006304050093B91300B3855E40B3E9590162
:10F71000B38535412326B1021395C5006352050612
:10F72000B306D74033036F40B337D700B307F34076
:10F730002322F1022320D102333F6F009307000000
:10F740006374D7009337130033EFE701338ECF4153
:10F75000B3BFCF01330EEE412324C1039307000052
:10F7600063040F0093B71300B38ED241B3E7F701E0
:10F77000B387FE402326F102130408006FF08FD3F5
:10F78000B3E71701B3E74701B3E7B700639407D2C4
:10F790006FF0DFF09387F7FF930301026394F9069C
:10F7A000630E056EB7070400B3F7FE0093B71700AA
:10F7B00093974700639E380D638A056C9396D20039
:10F7C00063DA066C6308050A378700002326E10226
:10F7D0002324010223220102232001021307C10274
:10F7E000832607008325C7FF1307C7FF93963600BC
:10F7F00093D5D501B3E6B6002322D700E392E3FE0A
:10F800006FF0CFEE6396F800930700006FF0DFFA19
:10F81000631E0506639E0504B78700002326F102D8
:10F820002324010223220102232001029307C102A3
:10F8300003A7070083A6C7FF9387C7FF13173700E7
:10F8400093D6D6013367D70023A2E700E392F3FEF5
:10F8500083270102378500001304000093973700C7
:10F860002320F1021305F5FF930700016FF04FD934
:10F87000930700002320E1022322E1032324F10364
:10F8800023265102130408006FF0CFE9930700000C
:10F89000E39C05F22320D102232261022324C10329
:10F8A0006FF0CFEAB387E640B308E34133B5F60023
:10F8B000B3351301B388A8402320F102232211039A
:10F8C0001305000063F6F60033056F40133515008D
:10F8D000B303FE413365B500B38AA340232451032B
:10F8E000333B7E00130A00006304050013BA1300C3
:10F8F000B3855E40336A6A01B38545412326B10270
:10F900001395C500635E050AB306D74033036F4005
:10F91000B337D700B307F3402322F1022320D102EB
:10F92000333F6F00930700006374D70093371300D1
:10F93000338ECF4133EFE701B3BFCF01330EEE413A
:10F940002324C10363040F0013B61300B38ED24106
:10F950003366F601B38ECE402326D103130408008C
:10F960000325C10263080506EF00107A130545FF61
:10F97000930600023368D502B347D502630808082E
:10F980001307C0FF1303010293952700B3860641B6
:10F990003387E7021307C7003307E3006310E30A66
:10F9A00013070104B305B700032701029387F7FF8C
:10F9B0003318070123A005FF9306F0FF6F00800BAB
:10F9C000B3E71701B3E75701B3E7B700E39A07F8C6
:10F9D0006FF0DFCC0325810263080500EF00D072D1
:10F9E000130505026FF09FF8032541026308050027
:10F9F000EF009071130505046FF05FF70325010216
:10FA0000EF009070130505066FF05FF61306C0FF58
:10FA10003386C7021307C10293063000B305C7003F
:10FA200083A505009386F6FF1307C7FF2322B700BF
:10FA3000E3D6F6FE9387F7FF6FF01FF80326C7FFA4
:10FA400083280700330EB7003356D600B398080159
:10FA5000336616012320CE001307C7FF6FF01FF493
:10FA600013972700130601023307E600232007003F
:10FA70009387F7FFE396D7FE634E35133305354181
:10FA80001305150093070002B348F50213080000A0
:10FA9000130700003365F5026342170593860800DB
:10FAA00063D408009306000013972800631605042A
:10FAB0009307300093060102B3881741B387E6002D
:10FAC00083A70700130515009386460023AEF6FEB4
:10FAD000E3D6A8FE130730006F00000C9317270031
:10FAE00093060102B387F60083A7070013071700E8
:10FAF0003368F8006FF05FFA9307010493962600CD
:10FB0000B386D70083A706FE93050002B385A54000
:10FB1000B397B7003368F800930701023387E70013
:10FB20009307300013060000B387174113074700FF
:10FB30006344F6021307010493972700B307F70005
:10FB40000327C1023355A70023A0A7FE13054000D9
:10FB5000330515416FF01FF81313260093060102B9
:10FB600033836600032E07008326C7FF13061600A3
:10FB7000331EBE00B3D6A600B3E6C6012320D300D1
:10FB80006FF0DFFA9317250093060102B387F600A2
:10FB900023A0070013051500E356A7FE0327010263
:10FBA000B337000113060000B367F7002320F1020A
:10FBB0006FF04F908327C1023707F8FF1307F7FF55
:10FBC000B3F7E7003385A9402326F10213060000AE
:10FBD0006FE0DFDD631A04009387870093B7870027
:10FBE0006FF0CF96E31A04FE0327C10393070600C4
:10FBF000130500001357470113471700137617002A
:10FC00006FF00FA093070600130500006FE09FE55B
:10FC1000631C04A483254102130787002320E1020B
:10FC200013378700B305B70033B7E5002322B102CD
:10FC300083258102B305B7002324B102B3B5E500E3
:10FC4000B38615016FF00FA2630004A28326410260
:10FC500013078700832581022320E10213378700E1
:10FC6000B306D70033B7E6002322D102B306B700AC
:10FC70002324D102B3B6E600B38616016FF08F9E3F
:10FC80006308060013F717006304070093E72700D3
:10FC90000327C1029316C70063D20602B78600008D
:10FCA000130515009386F6FF6306D510B706F8FF17
:10FCB0009386F6FF3377D7002326E102130701026C
:10FCC0009305C10283260700032647001307470058
:10FCD00093D636001316D601B3E6C600232ED7FE00
:10FCE000E392E5FE0327C1023786000093563700F2
:10FCF0002326D1021307F6FF631AE502832541028A
:10FD0000032701023367B700832581023367B700F9
:10FD10003367D700630C07002326C10223240102A6
:10FD20002322010223200102130400000327C10241
:10FD30001315150113551501231EE10213170501B3
:10FD40000325C103B70601809386F6FF3375D500FE
:10FD50003365E500131515001314F4011355150050
:10FD600003280102832541020326810233658500B1
:10FD70006384070073A017008320C1050324810555
:10FD800023A6A40023A0040123A2B40023A4C4003A
:10FD90001385040003290105832441058329C10437
:10FDA000032A8104832A4104032B01041301010661
:10FDB00067800000630E0902130730006314E90234
:10FDC000630804021307F0FF378500002326E102D1
:10FDD0002324E1022322E1022320E1021305E5FFAF
:10FDE0006F00000213072000E31EE9FCE30C04FC93
:10FDF00023260102232401022322010223200102DF
:10FE000093E757006FF09FEB130740076344F70039
:10FE10006FE05F9193071000232E0100232C010057
:10FE2000232A01002328F1006FE09F9F130740075A
:10FE30006344F7006FE0DFCA930710002326010038
:10FE400023240100232201002320F1006FE09FDA28
:10FE5000130740076356F7E49307100023260100B9
:10FE600023240100232201002320F1006FF08FF4EE
:10FE70006302058A6FF0CF8C930700016FF00F8348
:10FE800093070000639838896FF0CF87E3060598E1
:10FE90006FF05FA0930700016FF0DF92E39C38974B
:10FEA0006FF09F96130101FE032305008327450091
:10FEB000032685000328C50073272000374700006C
:10FEC000931618009318080193D51601232061009A
:10FED0002322F1002324C1002326010123286100ED
:10FEE000232AF100232CC1009306E7FF93D80801D1
:10FEF00063C6B602639C0500B3E76700B3E7C700BB
:10FF0000B3E7170113050000638E07041308100000
:10FF100013050000732018006F00C0049306D7017A
:10FF20001358F80163D4B604370500801345F5FF74
:10FF30003305A800630608141307E701130800013E
:10FF4000E39AE5FC135716019398F800B36817017C
:10FF5000E39208FCB3E767001316F600B367F600F8
:10FF60006390070A13010102678000009306F706F9
:10FF7000B7070100B386B640B3E7F80013060101E6
:10FF800013D75640232EF10093F6F6019308000094
:10FF900093050000130E0600032506009385150047
:10FFA00013064600B3E8A800E318B7FE13162700AF
:10FFB000639C0604930701023386C700832706FF6C
:10FFC000130610002328F100930730003387E74021
:10FFD0006314C70013062000130740009317260080
:10FFE000B307FE0023A0070013061600E318E6FE81
:10FFF00003250101630408003305A040E38408F6EB
:02000004800179
:10000000130810006FF01FF1930501023386C5003D
:10001000832506FF13050002130330003305D54086
:100020003303E34013071700B395A5001317270008
:10003000930E0102B3E8B8003387EE009305000089
:1000400063C065021386150013070102939525000E
:10005000B305B700B3D7D70023A8F5FE6FF0DFF7DD
:10006000832507FF832E06FFB395A500B3DEDE00D0
:10007000B3E5D5012328B100930510006FF05FFCB4
:10008000130800016FF01FE9130101FD2322910203
:100090002326110223248102232021039304050037
:1000A000638C051493D7F54133C4B7003304F4408F
:1000B0001305040013D9F501EF00100537470000C0
:1000C0001307E7013307A74013051505232881000F
:1000D000232A0100232C0100232E01009375F50132
:1000E000638005049307F0059306300063CCA700F6
:1000F00093060002B386B640B356D400232ED10037
:10010000930620001386F6FF9307010293962600BC
:10011000B386D7003314B40023A886FE6F00000511
:1001200093575540130630003306F64093060102FC
:10013000131626003386C600832606FF130620000A
:10014000232ED1009306F00563C2A6029306200079
:10015000B386F6409396260093070102B386D70034
:1001600083A706FF13061000232CF1009306F0FF6F
:100170009317260093050101B387F50023A007001C
:100180001306F6FFE316D6FE8327C10113171701E6
:10019000135717012316F100931707010327C10016
:1001A000B70601809386F6FF3377D7003367F700F1
:1001B00093171700032701011319F9018320C102C6
:1001C00023A0E400032741010324810293D71700F1
:1001D00023A2E40003278101B3E7270123A6F4004B
:1001E00023A4E400138504000329010283244102AF
:1001F0001301010367800000232E0100232C01005E
:10020000232A01002328010013070000130900001E
:100210006FF09FF7130101FD2322910223261102A3
:100220002324810293040500F327200093574601FD
:100230001317C60093F7F77F1357C700938617006D
:100240002328B100232AE100232E0100232C0100E2
:1002500093F6E67F1354F601638E0602B74600005C
:10026000938606C013D54500B387D7009356470041
:100270001317C7013367A7009395C501232ED1003B
:10028000232CE100232AB10023280100930600005B
:100290006F00C0133365B7006398070E9306000024
:1002A00063060512630E070413050700EF00C0651F
:1002B00013061503135756401376F6016308060418
:1002C0009306C0FFB306D702130301019307000290
:1002D00013182700B387C7409386C600B306D30020
:1002E0006312D308930701023388070183270101B2
:1002F0001307F7FF3396C7002328C8FE6F00C0031B
:10030000EF008060130505026FF09FFA1306C0FF2F
:100310003306C7029306C10193073000B385C600B8
:1003200083A505009387F7FF9386C6FF23A2B60037
:10033000E3D6E7FE1307F7FF9306F0FF93172700B6
:1003400013060101B307F60023A007001307F7FF08
:10035000E316D7FEB74700009387C7C0B387A7400F
:100360006FF0DFF283A5C6FF83A80600338E060177
:10037000B3D5F500B398C800B3E515012320BE003E
:100380009386C6FF6FF0DFF5630C050A9317C7016C
:1003900013D64500B3E7C700B7060800B376D70009
:1003A000232CF10013574700B78700003367F7008D
:1003B00093B616009395C50193964600232AB10083
:1003C00023280100232EE1009387F7FF0327C101B3
:1003D00093971701370601802316E1000327C10018
:1003E00093D717011306F6FF939707013377C700DA
:1003F000B367F700939717001314F40193D717000E
:10040000032801010325410183258101B3E787000A
:100410006384060073A016008320C10203248102B6
:1004200023A2A40023A0040123A4B40023A6F40063
:100430001385040083244102130101036780000037
:10044000B78700009387F7FF6FF05FE4130101FDAA
:100450008326050003274500832785000326C50062
:10046000F3252000232CF1002324F1029317060129
:1004700013131600232EC10093D707011356F6015C
:100480002328D1002320D102232AE1002322E102E4
:100490002326F1021353130113050600130E010264
:1004A0009306C10283A7060003A7C6FF9386C6FF73
:1004B000939737001357D701B3E7E70023A2F6005D
:1004C000E312DEFE83280102B78E000093071300BB
:1004D000139838001387EEFF23200103B3F7E700DA
:1004E000638E072AB7C7FFFF938707403303F300E4
:1004F0009307E07F63DA6710638405069307300093
:10050000639AF504630E06049307F0FF1303E07F7C
:100510009308F0FF13070000130850009306200013
:1005200013681800638ED538930630006384D5387D
:10053000639A053893F6F700130E40006384C639BA
:1005400093864700B3B7F600B388F8009387060098
:100550006F00403793072000E398F5FAE30606FAA8
:10056000930700001303F07F930800001308500066
:1005700013978800635E0700130313001307F07FCF
:100580006308E334370780FF1307F7FFB3F8E80089
:100590009396D80193D73700B3E7F6009306F07F20
:1005A00013D73800631ED300B3E7E700130700003A
:1005B0006388070037070800930700001305000051
:1005C0001317C7001373F37F131343011357C700A7
:1005D0001315F5013367670013860700B366A7009C
:1005E0002324C1002326D10087378100630408003B
:1005F000732018002734F100032581008325C100F2
:1006000013010103678000006354600683288102A0
:100610000327C1028327410293D6C801131747005D
:100620003367D70093964700B3E6060193D7C70117
:1006300093984800B336D000B3E71701B3E6F6004D
:100640002322E1022320D1028327010283284102D1
:1006500063080316130700001308000093F67700E1
:10066000E39E06EAE30607F0137718006F00802583
:100670009307C0FC635CF300232201029307100080
:100680002320F102130300006FF01FFC8327C10237
:100690003707080013080E00B3E7E7002326F1022E
:1006A0009307D003B387674013DF5740930E0000D2
:1006B00093F7F701130700008328080013071700BA
:1006C00013084800B3EE1E01E318EFFE13172F00C6
:1006D0006396070413083000330FE8413388E600BF
:1006E00003280800938717009386460023AE06FF71
:1006F000E356FFFE93064000139727003307EE00F2
:100700002320070093871700E398D7FE03270102F1
:10071000B337D001B367F7006FF09FF6930601037C
:10072000B386E60083A606FF130300023303F340FB
:10073000B3966600B3EEDE00B306EE00130730009A
:10074000930800003307E7419386460063C4E8023C
:1007500093060103131727003387E6008326C1029F
:10076000B3D7F6002328F7FE93074000B387E7418D
:100770006FF05FF803A8C6FF83A20600939F2800CE
:100780003358F800B3926200B30FFE01336858008B
:1007900023A00F01938818006FF01FFB83274102ED
:1007A00083268102032EC10233E7D7003367C701D6
:1007B000B368070163160306B337100193080000FE
:1007C00033E7F8006300070E93D6F701139718007C
:1007D0003307D7009396170013F376001308000031
:1007E00063060302130820006380050B1308300022
:1007F0006380050913081000639A050013F3F600DF
:10080000130E400093B6C6FF631AC3071357870140
:100810001347170013771700130300006FF01FE44E
:10082000638A0806938EFEFF13080000631AD30143
:100830003708040033780E011338180013184800E5
:100840001397460093D7C70193D6C601131E4E00D7
:10085000B3E7E700B3E6C60137074000B3E8E600B8
:1008600093F787FF1303F07F130700006FF01FDF7C
:1008700013081000E31C06F893B686FF93C6160013
:100880003307D7006FF09FF813081000E30006F855
:100890006FF09FFE930700001303F07F1308000022
:1008A0006FF01FCD930700009308000013030000B2
:1008B0006FF0DFFE63180600938687006FF09FC815
:1008C000E31C06FEE30607CA136828006FF05FCA40
:1008D000930700006384050213073000639AE50064
:1008E000630E06009307F0FF1303E07F6F00000123
:1008F00013072000E398E5FEE30606FE13685800A0
:10090000938807006FF0DFC8B7070100637AF5022C
:100910009307F00FB3B7A7009397370013070002B0
:100920003307F740B357F50037150081130545D756
:10093000B387A70003C507003305A7406780000001
:100940003707000193070001E36AE5FC9307800184
:040950006FF0DFFC69
:02000004810079
:10000000300000003100000032000000330000002A
:10001000340000003500000036000000370000000A
:10002000380000003900000061000000620000009C
:10003000630000006400000065000000660000002E
:1000400048656C6C6F2066726F6D205F636C6F73B8
:10005000650A000073745F6D6F64653A20000000EC
:1000600073745F6465763A200000000073745F6902
:100070006E6F3A200000000073745F7569643A2067
:100080000000000073745F6769643A20000000009C
:1000900073745F726465763A2000000073745F7356
:1000A000697A653A2000000073745F626C6B736953
:1000B0007A653A200000000073745F626C6F636BB6
:1000C000733A200048656C6C6F2066726F6D205F1C
:1000D0006973617474790A0048656C6C6F2066728C
:1000E0006F6D205F6C7365656B0A000048656C6C12
:1000F0006F2066726F6D205F726561640A00000098
:100100003000000031000000320000003300000029
:100110003400000035000000360000003700000009
:10012000380000003900000061000000620000009B
:10013000630000006400000065000000660000002D
:100140000A00000030000000310000003200000012
:1001500033000000340000003500000036000000CD
:100160003700000038000000390000006100000086
:1001700062000000630000006400000065000000F1
:100180006600000074657374696E675F746D630A5E
:10019000000000000A000000746573745F646976F3
:1001A000657267656E63650A0000000074657374AC
:1001B0005F737061776E0A0030000000310000004C
:1001C0003200000033000000340000003500000061
:1001D0003600000037000000380000003900000041
:1001E0006100000062000000630000006400000085
:1001F00065000000660000007072696E74663A2047
:100200004E65776C6962204D61696E2025640A0035
:10021000E00E0080F4200080F4200080F40E0080C6
:10022000F4200080F4200080F42000808C0E0080F8
:10023000F4200080F4200080FC0E00801C0F008061
:10024000F4200080140F0080240F0080F420008030
:100250007C0F0080840F0080840F0080840F00805A
:10026000840F0080840F0080840F0080840F008042
:10027000840F0080840F0080F4200080F420008030
:10028000F4200080F4200080F4200080F42000801E
:10029000F4200080C0130080F4200080141000803F
:1002A00000130080C0130080C0130080C0130080C2
:1002B000F4200080F4200080F4200080F4200080EE
:1002C000B40F0080F4200080F42000805C1D0080CA
:1002D000F4200080F4200080F4200080041E0080C0
:1002E000F4200080501E0080F4200080F420008064
:1002F000B81E0080F4200080F4200080F4200080EC
:10030000F4200080F4200080F4200080F42000809D
:10031000F4200080C0130080F420008014100080BE
:1003200004130080C0130080C0130080C01300803D
:10033000BC0F00800413008004100080F4200080B3
:10034000E80F0080F4200080F01C0080601D008019
:10035000CC1D008004100080F4200080041E00806A
:10036000D80E0080541E0080F4200080F42000800D
:10037000101F0080F4200080D80E00802020202054
:10038000202020202020202020202020303030302D
:10039000303030303030303030303030494E460040
:1003A000696E66004E414E006E616E003031323330
:1003B00034353637383961626364656600000000A1
:1003C000303132333435363738394142434445468B
:1003D00000000000300000000000000000000000ED
:1003E0000000000000000000000000007665924A56
:1003F0004A803F154CC99A97208A025260C42575DD
:10040000326A52CE9A32CE284DA7E45D3DC55D3B9F
:100410008B9E925A6C52CE508BF1283D0D65170C75
:100420007581867576C9484D669CF85850BC545CF9
:1004300065CCC6910EA6AEA019E3A3461E85B7EA09
:10044000FE981B90BBDD8DDEF99DFBEB7EAA514330
:1004500035023701B1366C336FC6DF8CE980C9478E
:10046000BA93A841F850FB256BC7716BBF3CD5A66A
:10047000CFFF491F78C2D3400000000000000000F9
:1004800020F09DB5702BA8ADC59D6940000000000F
:1004900000000000000000000004BFC91B8E3440B3
:1004A000000000000000000000000000000000202C
:1004B000BCBE194000000000000000000000000069
:1004C00000000000409C0C40000000000000000004
:1004D000000000000000000000C80540000000000F
:1004E00000000000000000000000000000A002402A
:1004F00000000000000000000000000000000000FC
:100500000080FF3FFFFFFEFFFCFFF8FFF0FFE0FF72
:10051000C0FF80FF00FF00FE00FC00F800F000E0DC
:1005200000C00080000000003020FCCFC3A1238168
:10053000E32DDE9FCED2C804DDA6D80A6482CBD2DA
:10054000EAF2D4122549E42D36344F53AECE6B2552
:100550003FF598F6D36B5801A687BDC057DAA58240
:10056000A6A2B53231E7D404F2E332D332711CD201
:1005700023DB32EE49905A393EA20853FBFE551157
:1005800091FA39197A63254331C0AC3C6DE2DEDB68
:100590005DD0F6B37CACA0E4BC647C46D0DD553EB7
:1005A000202A2462B347D798233FA5E939A527EA33
:1005B0007FA82A3F5B0BF24A81A5ED18DE67BA944B
:1005C0003945AD1EB1CF943F71BFB3A9897968BEDB
:1005D0002E4C5BE14DC4BE9495E6C93F4D3D3D7C3C
:1005E000BA362B0DC2FDFCCE61841177CCABE43F53
:1005F00055C1A8A44E401361C3D32B6519E2581707
:10060000B7D1F13F0AD7A3703D0AD7A3703D0AD7EF
:10061000A3703D0AD7A3F83FCDCCCCCCCCCCCCCC6E
:10062000CCCCCCCCCCCCCCCCCCCCFB3F204E614E7B
:1006300020000000202D496E66696E6974792000E3
:1006400020496E66696E6974792000004E614E0023
:1006500045256400000000000500000019000000AE
:100660007D00000000000000000000000000F03FDE
:10067000000000000000244000000000000059407D
:100680000000000000408F40000000000088C340D0
:1006900000000000006AF8400000000080842E4145
:1006A00000000000D01263410000000084D7974191
:1006B0000000000065CDCD41000000205FA0024297
:1006C000000000E876483742000000A2941A6D420C
:1006D000000040E59C30A2420000901EC4BCD642FF
:1006E00000003426F56B0C430080E03779C34143AA
:1006F00000A0D8855734764300C84E676DC1AB4320
:10070000003D9160E458E143408CB5781DAF15443D
:1007100050EFE2D6E41A4B4492D54D06CFF0804418
:10072000F64AE1C7022DB544B49DD9794378EA442D
:10073000BC89D897B2D29C3C33A7A8D523F64939B7
:100740003DA7F444FD0FA5329D978CCF08BA5B25D9
:10075000436FAC642806C80A0080E03779C3414380
:10076000176E05B5B5B89346F5F93FE9034F384D17
:10077000321D30F94877825A3CBF737FDD4F1575C3
:1007800040750080948700809487008054750080B5
:10079000948700809487008094870080EC740080A8
:1007A00094870080948700805C7500807C75008051
:1007B0009487008074750080847500809487008021
:1007C000DC750080E4750080E4750080E4750080CD
:1007D000E4750080E4750080E4750080E4750080B5
:1007E000E4750080E4750080948700809487008021
:1007F000948700809487008094870080948700808D
:1008000094870080247A008094870080747600802A
:1008100064790080247A0080247A0080247A008021
:10082000948700809487008094870080948700805C
:10083000147600809487008094870080FC83008079
:10084000948700809487008094870080A48400802F
:1008500094870080F08400809487008094870080D3
:10086000588500809487008094870080948700805A
:10087000948700809487008094870080948700800C
:1008800094870080247A00809487008074760080AA
:1008900068790080247A0080247A0080247A00809D
:1008A0001C760080687900806476008094870080E0
:1008B00048760080948700809083008000840080C8
:1008C0006C8400806476008094870080A48400801B
:1008D00038750080F48400809487008094870080BD
:1008E000B08500809487008038750080202020200B
:1008F00020202020202020202020202030303030B8
:10090000303030303030303030303030D8960080B9
:10091000D09E0080D09E0080EC960080D09E00800B
:10092000D09E0080D09E008088960080D09E00805F
:10093000D09E0080F49600800C970080D09E0080AE
:100940000497008014970080D09E008064970080F8
:100950006C9700806C9700806C9700806C9700808B
:100960006C9700806C9700806C9700806C9700807B
:100970006C970080D09E0080D09E0080D09E00802A
:10098000D09E0080D09E0080D09E0080D09E0080AF
:10099000D09E0080D09E0080D4970080F497008085
:1009A000D09E0080D09E0080D09E0080D09E00808F
:1009B000D09E0080D09E0080D09E0080D09E00807F
:1009C000D09E0080D09E0080F0980080D09E008055
:1009D000D09E0080D09E008088990080D09E0080AC
:1009E000749C0080D09E0080D09E0080D49C0080AB
:1009F000D09E0080D09E0080D09E0080D09E00803F
:100A0000D09E0080D09E0080D09E0080D09E00802E
:100A1000D09E0080D09E0080D4970080F897008000
:100A2000D09E0080D09E0080D09E00809497008051
:100A3000F8970080C4970080D09E0080B497008013
:100A4000D09E0080A0980080F49800805899008083
:100A5000C4970080D09E008088990080D096008046
:100A6000789C0080D09E0080D09E008038960080C8
:100A7000D09E0080D09600802020202020202020A2
:100A800020202020202020203030303030303030E6
:100A9000303030303030303043000000504F534958
:100AA000580000002E0000006CB9008064C1008076
:100AB00064C1008080B9008064C1008064C100808E
:100AC00064C100801CB9008064C1008064C10080E2
:100AD00088B90080A0B9008064C1008098B9008006
:100AE000A8B9008064C10080F8B9008000BA008015
:100AF00000BA008000BA008000BA008000BA00800E
:100B000000BA008000BA008000BA008000BA0080FD
:100B100064C1008064C1008064C1008064C1008041
:100B200064C1008064C1008064C1008064C1008031
:100B300064C1008068BA008088BA008064C1008007
:100B400064C1008064C1008064C1008064C1008011
:100B500064C1008064C1008064C1008064C1008001
:100B600064C1008084BB008064C1008064C10080D7
:100B700064C100801CBC008064C1008008BF00808C
:100B800064C1008064C1008068BF008064C10080CF
:100B900064C1008064C1008064C1008064C10080C1
:100BA00064C1008064C1008064C1008064C10080B1
:100BB00064C1008068BA00808CBA008064C1008083
:100BC00064C1008064C1008028BA00808CBA0080B3
:100BD00058BA008064C1008048BA008064C10080B7
:100BE00034BB008088BB0080ECBB008058BA00801A
:100BF00064C100801CBC008064B900800CBF008010
:100C000064C1008064C10080CCB8008064C10080F1
:100C100064B90080202020202020202020202020B7
:100C20002020202030303030303030303030303004
:100C30003030303000202020202020202020282884
:100C4000282828202020202020202020202020208C
:100C500020202020208810101010101010101010CC
:100C600010101010100404040404040404040410FC
:100C7000101010101010414141414141010101018A
:100C80000101010101010101010101010101010154
:100C90001010101010104242424242420202020260
:100CA0000202020202020202020202020202020224
:100CB00010101010200000000000000000000000D4
:100CC0000000000000000000000000000000000024
:100CD0000000000000000000000000000000000014
:100CE0000000000000000000000000000000000004
:100CF00000000000000000000000000000000000F4
:100D000000000000000000000000000000000000E3
:100D100000000000000000000000000000000000D3
:100D200000000000000000000000000000000000C3
:100D3000000000000000000020DF008020DF0080B5
:100D40001CDF0080D0DE0080D0DE008024D6008052
:100D50001CDF0080D0DE008024D60080D0DE008042
:100D60001CDF0080CCDE0080CCDE0080CCDE00808A
:100D700028D60080000102020303030304040404D4
:100D80000404040405050505050505050505050517
:100D900005050505060606060606060606060606F7
:100DA00006060606060606060606060606060606E3
:100DB00006060606070707070707070707070707C7
:100DC00007070707070707070707070707070707B3
:100DD00007070707070707070707070707070707A3
:100DE0000707070707070707070707070707070793
:100DF0000707070708080808080808080808080877
:100E00000808080808080808080808080808080862
:100E10000808080808080808080808080808080852
:100E20000808080808080808080808080808080842
:100E30000808080808080808080808080808080832
:100E40000808080808080808080808080808080822
:100E50000808080808080808080808080808080812
:100E60000808080808080808080808080808080802
:040E7000080808085E
:040E7400E00F00810A
:100E7800000000000000F03F0000000000002440D7
:080E88000000000000005043CF
:100E90001000000000000000017A5200017C0101F6
:100EA0001B0D02001000000018000000F0B600FF4B
:100EB0003404000000000000100000002C000000BE
:0C0EC00010BB00FF100400000000000048
:100ED0000000008104000081080000810C000081F6
:100EE0001000008114000081180000811C000081A6
:100EF0002000008124000081280000812C00008156
:100F00003000008134000081380000813C00008105
:100F10000001008104010081080100810C010081B1
:100F20001001008114010081180100811C01008161
:100F30002001008124010081280100812C01008111
:100F40003001008134010081380100813C010081C1
:100F500044010081480100814C0100815001008161
:100F600054010081580100815C0100816001008111
:100F700064010081680100816C01008170010081C1
:100F800074010081780100817C0100818001008171
:100F9000050000000500000005000000050000003D
:100FA000B8010081BC010081C0010081C401008141
:100FB000C8010081CC010081D0010081D4010081F1
:100FC000D8010081DC010081E0010081E4010081A1
:100FD000E8010081EC010081F0010081F401008151
:100FE00000000000CC120081341300819C130081AA
:100FF00000000000000000000000000000000000F1
:1010000000000000000000000000000000000000E0
:1010100000000000000000000000000000000000D0
:1010200000000000000000000000000000000000C0
:1010300000000000000000000000000000000000B0
:1010400000000000000000000000000000000000A0
:101050000000000000000000000000000000000090
:101060000000000000000000000000000000000080
:101070000000000000000000000000000000000070
:10108000000000000000000001000000000000005F
:101090000E33CDAB34126DE6ECDE05000B00000024
:1010A0000000000000000000000000000000000040
:1010B0000000000000000000000000000000000030
:1010C0000000000000000000000000000000000020
:1010D0000000000000000000000000000000000010
:101410000814008108140081101400811014008148
:1014200018140081181400812014008120140081F8
:1014300028140081281400813014008130140081A8
:101440003814008138140081401400814014008158
:101450004814008148140081501400815014008108
:1014600058140081581400816014008160140081B8
:101470006814008168140081701400817014008168
:101480007814008178140081801400818014008118
:1014900088140081881400819014008190140081C8
:1014A0009814008198140081A0140081A014008178
:1014B000A8140081A8140081B0140081B014008128
:1014C000B8140081B8140081C0140081C0140081D8
:1014D000C8140081C8140081D0140081D014008188
:1014E000D8140081D8140081E0140081E014008138
:1014F000E8140081E8140081F0140081F0140081E8
:10150000F8140081F8140081001500810015008195
:101510000815008108150081101500811015008143
:1015200018150081181500812015008120150081F3
:1015300028150081281500813015008130150081A3
:101540003815008138150081401500814015008153
:101550004815008148150081501500815015008103
:1015600058150081581500816015008160150081B3
:101570006815008168150081701500817015008163
:101580007815008178150081801500818015008113
:1015900088150081881500819015008190150081C3
:1015A0009815008198150081A0150081A015008173
:1015B000A8150081A8150081B0150081B015008123
:1015C000B8150081B8150081C0150081C0150081D3
